:020000040800F2
:10000000405500200D0200081502000817020008E4
:10001000190200081B0200081D0200080000000071
:100020000000000000000000000000003102000895
:100030002102000800000000C9020008D9020008DF
:1000400027020008270200082702000827020008EC
:1000500027020008270200082702000827020008DC
:1000600027020008270200082702000827020008CC
:1000700027020008270200082702000827020008BC
:1000800027020008270200082702000827020008AC
:10009000270200082702000827020008270200089C
:1000A000270200082702000827020008270200088C
:1000B000270200082702000827020008270200087C
:1000C000270200082702000827020008270200086C
:1000D000270200082702000827020008270200085C
:1000E000270200082702000827020008270200084C
:1000F000270200082702000827020008270200083C
:10010000270200082702000827020008270200082B
:10011000270200082702000827020008270200081B
:10012000270200082702000827020008270200080B
:1001300027020008270200082702000827020008FB
:1001400027020008270200082702000827020008EB
:1001500027020008270200082702000827020008DB
:1001600027020008270200082702000827020008CB
:1001700027020008270200082702000800000000EC
:1001800027020008270200082702000827020008AB
:10019000270200082702000827020008270200089B
:1001A000C19800082702000855220008270200080D
:1001B000270200082702000827020008270200087B
:1001C000270200082702000827020008270200086B
:1001D000270200082702000827020008270200085B
:1001E000270200082702000827020008270200084B
:1001F0002702000827020008DFF80CD000F006F9FB
:1002000000480047892E01084055002006488047D5
:1002100006480047FEE7FEE7FEE7FEE7FEE7FEE7EB
:10022000FEE7FEE7FEE7FEE709A90008F90100087E
:100230001EF0040F0CBFEFF30880EFF30980816913
:1002400011F8021C91BB01B590E80F10E047BDE822
:1002500000508CE80300244B93E80600914208BF4D
:10026000704741B91EF0100F10D12049086820F0E6
:10027000010008600AE02CE9F00F1EF0100F08BF23
:100280002CED108AC1F838C081F822E01A6092F88B
:100290002210906B61F0FF0E1EF0100F08BFB0EC43
:1002A000108AB0E8F00F80F309887047104A13688D
:1002B0009942FAD801B552F821C00FC8E047BDE80D
:1002C0000050CCF80000704701B500F0F3FCBDE829
:1002D0000140EFF3098CBEE701B500F065FFBDE812
:1002E0000140EFF3098CB6E7A417002034EF00E0DB
:1002F000143201082DE9F05F0546002092469B4626
:1003000088460646814640241BE02846414647462B
:10031000224600F06BF853465A46C01A914110D35A
:1003200011461846224600F052F82D1A67EB0108D4
:100330004F4622460120002100F049F817EB000942
:100340004E41201EA4F10104DFDC484631462A4616
:100350004346BDE8F09F10B5441A0346944209D2C3
:100360008418114403E011F8013D04F8013D521EC8
:10037000F9D210BD40EA0104A40703D009E010C976
:10038000121F10C3042AFAD203E011F8014B03F83C
:10039000014B521EF9D210BDD2B201E000F8012B80
:1003A000491EFBD270470022F6E710B513460A46F5
:1003B00004461946FFF7F0FF204610BD034611F82A
:1003C000012B00F8012B002AF9D118467047202A8A
:1003D00004DB203A00FA02F1002070479140C2F19C
:1003E000200320FA03F3194390407047202A04DBCE
:1003F000203A21FA02F00021704721FA02F3D0409E
:10040000C2F120029140084319467047064C074D3F
:1004100006E0E06840F0010394E8070098471034D4
:10042000AC42F6D3FFF7ECFEC05D0108E05D0108C9
:1004300070B58C1810F8015B15F0070301D110F8A6
:10044000013B2A1106D110F8012B03E010F8016BD3
:1004500001F8016B5B1EF9D12B0705D40023521E56
:100460000DD401F8013BFAE710F8013BCB1A921CBE
:1004700003E013F8015B01F8015B521EF9D5A142BC
:10048000D8D3002070BD10B5930712D400F10C032F
:10049000D00718D153E8000F084203D1BFF32F8FC4
:1004A000002005E020EA010243E8002404B1F1E75E
:1004B00010BDC068D20700EA010315D1002B18BF98
:1004C00010BD002010BD53E8000F00EA01028A426F
:1004D00003D0BFF32F8F002005E020EA010243E89C
:1004E000002404B1EFE710BD8B4218BF002010BDFF
:1004F00010B500F1280151E8002F12B9BFF32F8F7A
:1005000004E0531E41E8003404B1F4E78AB12C3012
:1005100001210BE0821CD2E84F3FC2E8441F04B126
:10052000F9E713F0FF0F08BF10BD0830006800287E
:10053000F0D1002010BD84465CF8303F93B110B577
:100540004FF0000E05E0CB78D4789C420FD2536870
:1005500096461A46002AF6D10022C1E9012E00F182
:100560002C0207E00022C1E90122C1620AE0C1E9D0
:10057000012E0832BEF1000F116018BF0EF1040CFD
:10058000BDE81040CCF80010283050E8001F4A1C8D
:1005900040E8002303B1F8E77047D1E9012C02F1EC
:1005A0000803002A08BF00F12C03C3F800C0D1E9FA
:1005B00001210B1D002908BF00F130031A607047AC
:1005C00001480068704700BF10E000E0074801786C
:1005D000012905D10021017005484FF080610160BB
:1005E0000448016841F00101016070473851002062
:1005F00004ED00E010E000E04FF0FF307047000035
:1006000040B10B490968B1FBF0F0411E0020B0EB8E
:10061000116F02D04FF0FF307047064AFF2313706E
:10062000054A0623136051600449906008707047C2
:100630008813002023ED00E010E000E03851002096
:1006400010B5930712D400F12803D00718D153E84E
:10065000000F084203D1BFF32F8F002005E020EAEE
:10066000010243E8002404B1F1E710BD806AD2071B
:1006700000EA010315D1002B18BF10BD002010BDEA
:1006800053E8000F00EA01028A4203D0BFF32F8F24
:10069000002005E020EA010243E8002404B1EFE76E
:1006A00010BD8B4218BF002010BD000080B5124A5B
:1006B0004FF0000E02F1440C624606E01A699142C6
:1006C0000BD3891A03F10C029E461368002BF5D157
:1006D0000022C0E902E2016106E0C0E902E3016133
:1006E00098601A69511A1961BEF1000F18BF0EF116
:1006F0000C0CCCF8000080BD90170020EFF30581B2
:1007000029B9EFF3108111B9EFF3118111B16FF035
:1007100005007047DFF804C000DF70478913000848
:10072000EFF3058129B9EFF3108111B9EFF31181CE
:1007300009B100207047DFF808C000DF704700BF34
:100740009D130008EFF3148010F0010F08D0EFF3B1
:10075000058028B9EFF3108010B9EFF3118010B1C4
:100760000448007A7047DFF808C000DF704700BF18
:100770000914000890170020EFF3058028B9EFF363
:10078000108010B9EFF3118010B10348C0687047B2
:10079000DFF808C000DF704790170020151400082C
:1007A000EFF3058028B9EFF3108010B9EFF3118053
:1007B00010B16FF005007047DFF804C000DF70472C
:1007C00021140008EFF3058028B9EFF3108010B969
:1007D000EFF3118010B16FF005007047DFF804C02F
:1007E00000DF704799150008F8B50546EFF305805E
:1007F00014460E4628B9EFF3108010B9EFF31180BC
:1008000000B36FF003001DB313BB0EB329780829A2
:100810001ED1687898B12846FFF76AFE074677B17F
:100820006A6A07F10C013046FFF795FD0CB1F878C4
:1008300020703846FD6000F085FA002008E06FF077
:10084000020005E0DFF80CC028463146224600DFF2
:1008500001B0F0BD25160008EFF305832BB9EFF3C7
:10086000108313B9EFF311830BB100207047DFF849
:1008700008C000DF704700BF151700082DE9F041E0
:100880000646EFF3058090460D4628B9EFF3108039
:1008900010B9EFF3118038B36FF003070EB303BB49
:1008A000FDB1307808281CD17078C0B106F10C0079
:1008B00000F0F9F8044694B1726A04F10C0029467C
:1008C000FFF749FD40F20710002720802046A7705F
:1008D00084F80380C4E9015600F034FA01E06FF0B7
:1008E00002073846BDE8F081DFF80CC030462946E3
:1008F000424600DFBDE8F0814D180008EFF30582A5
:100900002AB9EFF3108212B9EFF3118212B16FF02E
:1009100005007047DFF804C000DF704715190008B4
:10092000EFF3058129B9EFF3108111B9EFF31181CC
:1009300009B100207047DFF808C000DF704700BF32
:10094000AD190008EFF3058129B9EFF3108111B952
:10095000EFF3118111B16FF005007047DFF804C0AB
:1009600000DF7047191A0008F8B504466078A8B18E
:10097000A76810E095F82320696AAF682046FFF762
:1009800082FD06463EB1284600F049FB2846314626
:10099000002200F0EFFB3D46002DEBD1F8BDB0B5D5
:1009A0000023D0B3C9B3032A37D886460F315EF887
:1009B000084F21F0070CDEF804102346A3EB0E04C9
:1009C00021F00305641B644505D21C689E46002C7B
:1009D000F1D1002321E0D0E9004363444360204487
:1009E00050F8044C9C423EBF08384360DEF80410C7
:1009F00069B1DEF8000021F0030141F80E004CEA75
:100A0000020071444860CEF800108E4603E04CEAC4
:100A10000200CEF804000EF108031846B0BD80B500
:100A2000002218B311B300F10803A1F1080C4FF034
:100A3000000E1A46624505D013689646002BF8D181
:100A4000002213E051F8043C4268BEF1000F23F08D
:100A50000303A2EB030242604FF0010219BFDCF86E
:100A60000000CEF80000002041F8040C104680BDC4
:100A700008B1420702D00022104670470022182910
:100A8000FAD311F00703F7D11022C0E90012014494
:100A9000A1F108038360002341F8083C81684A60A3
:100AA0000122C360E8E708B3B0B5014604C951E8C4
:100AB000003F9A4202D8BFF32F8F04E05C1C41E84C
:100AC000004505B1F3E701688B42BDE8B0400DD2A7
:100AD00000F1140151E8000F10B9BFF32F8F04E0AB
:100AE000026841E8002303B1F4E770470020704733
:100AF000B0B510B3C2688A421FD802698A421CD9B5
:100B0000021D52E8003F13B9BFF32F8F04E05C1EB3
:100B100042E8004505B1F4E793B1143002680A6079
:100B2000BFF35F8F50E8002F0B689342F6D140E887
:100B3000001404B1F2E70020B0BD6FF00300B0BDB7
:100B40006FF00200B0BD84460020BCF1000F18BF5A
:100B5000002921D002B3FBB180B54FF0000E02FB9B
:100B60000130CCE9001ECCE90223CCE90403481E85
:100B7000C1F1010E194600FB02FC04E088180EF1D9
:100B8000010E08600146BEF1000FF7D1002043F8C6
:100B90000C000120BDE880407047F8B5044660783D
:100BA00000285ED0A078A8B3E5686878002858D0FF
:100BB00028462146FFF7F1FC002005F10C062146EE
:100BC00060703046FFF794FFA868002849D040784D
:100BD000932846D13046FFF766FF0446002C40D0EC
:100BE000284600F0F5F9002100220646002700F013
:100BF000C1FA304600F050FA06466A6A04F10C0069
:100C0000B168FFF7A8FB40F207102080A770F068DA
:100C1000E07027E0A568687818B3A86810B340783A
:100C200083281FD1284600F0D3F900210022064670
:100C3000002700F09FFA304600F02EFA06466A6A56
:100C400004F10C01B068FFF786FBF06808B1E178A9
:100C50000170677005F10C002146BDE8F840FFF710
:100C600047BFF8BD28462146BDE8F840FFF763BC02
:100C70002DE9F041044600274FF0010815E0E8781F
:100C80006C69000711D52F76A86870B1284600F06E
:100C90009FF900210022064600F06CFAEE60F06A2F
:100CA000C5E90470F56285F818802546002DE6D167
:100CB000BDE8F081F8B5224C4FF6FF7604F15605F9
:100CC00004F15A0727E0D7E85F1F4A1C904200D87A
:100CD0000022C7E8532F03B1F5E788B2E16D51F860
:100CE0002000002826D001780139062913D8DFE832
:100CF00001F0041207120A0D1000216E88470AE065
:100D0000616E884707E0A16E884704E0E16E88477E
:100D100001E0216F8847B4F85400D5E85F1F11B98E
:100D2000BFF32F8F04E04A1EC5E8532F03B1F4E749
:100D30003142C8D10020BDE8F84000F0EDB800BF56
:100D40009017002070B501461948B0F8542000F102
:100D50005603D3E85F4FA24202D8BFF32F8F04E0BF
:100D6000651CC3E8565F06B1F3E7A3B293421AD2FB
:100D700000F15803D3E85F4F651CAA4200D8002554
:100D8000C3E8565F06B1F5E7C36DA2B243F822107F
:100D9000417A002919BF0121817206484FF0805124
:100DA00008BF016070BD0220BDE8704012F09CB821
:100DB0009017002004ED00E0012141700C4990F9EA
:100DC00020C001F11C021346194651F8082F4AB100
:100DD00092F920106145F6DC02F10C01C0E9022312
:100DE000986002E00022C0E902230860704700BF5B
:100DF0009017002080B54A1C1AD0224A4FF0000EEE
:100E000002F12C0C624606E0DA69914227D3891A76
:100E100003F110029E461368002BF5D1C161002139
:100E2000BEF1000FC0E9041E18BF0EF1100C25E042
:100E30001449002201F1300C634611461A6802F190
:100E40001003002AF9D14FF0FF320029C2614FF0A0
:100E50000002C0E9042118BF01F1100C0EE0BEF140
:100E6000000FC0E9043EC16118BF0EF1100CCCF8B0
:100E7000000003F1140CDA69511AD961CCF80000B2
:100E800080BD00BF90170020C36941695A1C11D072
:100E9000DFF848C021B9DCF82C20824218BF704727
:100EA000026922B15161D1691944D161416939B1F5
:100EB0000A610EE0094A31B9136B834203D07047CF
:100EC000CCF82C20704703690BB15961416919B105
:100ED0000B61002141617047136370479017002038
:100EE000B0B50C4DEC6A1CB1E0690138E06100D08E
:100EF000B0BD204600F093F8204600F0C3F8246906
:100F00002CB1E0690028F4D00020606100E00024EA
:100F1000EC62B0BD90170020B0B505461548002D15
:100F20004469017A0DD0022906D12CB194F9200030
:100F300095F92010814213DC2846BDE8B04000F04E
:100F4000A1B8022914D19CB1456A8DB194F9200051
:100F500095F920108142D8BFB0BD284600F05FF857
:100F60002046FFF729FF2846BDE8B04000F0DEB874
:100F7000B0BD00BF9017002010B50446002060707F
:100F8000A07810F0020F0DD0C00605D40F48216BD9
:100F9000406FFFF744FD05E00C48216BD0F884005A
:100FA000FFF7A6FDA078C00708BF10BD0749D1F81C
:100FB000880020B12146BDE81040FFF799BDD1F867
:100FC00080002146BDE81040FFF729BD90170020A2
:100FD0000146886830B18268002A8A6000D0D160FA
:100FE0000021C1607047C9B191F920C000F1080229
:100FF00006E093F9202062450ADB03F10802184657
:101000001368002BF5D10022C1E90220083004E06A
:10101000C1E90230816003F10C0001607047C168D2
:1010200031B182688A60826802B1D1600021C160FA
:101030007047B0B50446254603E02878012803D15F
:10104000ED68002DF9D1B0BD2046FFF7E8FF284636
:101050002146BDE8B040FFF7C6BF10B50446607832
:10106000332818BF10BD94F82320616A2046FFF78B
:10107000E7FA014629B120460022BDE8104000F001
:1010800079B810BD01460120487002481C30FFF7B6
:10109000AABF00BF9017002090F822104022806B5A
:1010A00002EA810181F06001084470470748416904
:1010B00039B1086B8A6B824204D90068044A9042B5
:1010C00000D17047012011F00FBF00BF9017002022
:1010D000A52E5AE2B0B5114DA86A08B101240AE064
:1010E0000F480021826D0F4800F08AFD0446002C55
:1010F000AC6218BF01240A48416E61B1A96C51B9B4
:10110000C26D0948002100F07BFD0028A86418BFCB
:1011100001202040B0BD2046B0BD00BF9017002088
:101120004C5D0108EB2E01081912000802214170E4
:1011300001498861FFF7BABF9017002010B50C4C29
:101140008446207A02281CBF002010BD636900205D
:101150006BB1626A5AB1184683F801C0FFF74AFEC4
:1011600004F11C00FFF734FFFFF7E0FF012010BD82
:1011700090170020B0B504461546402294F822008E
:1011800002EA8000A26B80F0600011502046FFF759
:101190007BFE20461DB1BDE8B040FFF7BDBEBDE8F7
:1011A000B040FFF76FBF0000B0B5FFF709FA194D67
:1011B000E968286D01310028E96000D08047FFF719
:1011C0008FFE0020FFF7A8FE296C11B3AA69A86B57
:1011D00090421CBFC5E90E21B0BDE96B11B10139C8
:1011E000E96316D1297A022913D16C6A8CB190F87F
:1011F000200094F8201081420BD12046FFF70FFF0A
:10120000A86BFFF73FFF2046FFF790FF286CC5E96A
:101210000E40B0BD90170020BCB50D480821D0E9A4
:101220001820FFF719FB0B4D0028E8640ED00A497F
:101230006C462965214600224FF0FF33FFF7D4FAB0
:1012400010B9DDE900108847E86CF3E7BCBD00BFCA
:101250004C5D0108901700205D12000870B5144D18
:101260006C6C1CB320690126013820611CE02069E8
:10127000E0B9E06808B1A1688160686404F1180110
:1012800000220023E86CFFF7F9FA18B10320214689
:1012900011F02AFEE078012804D161692046FFF7A9
:1012A00005FA00E066706C6C002CE0D170BD00BFE8
:1012B00090170020DFF804C000DFFEE7D51A000811
:1012C000EFF305822AB9EFF3108212B9EFF311821E
:1012D000F2B1B0B56FF00304C0B1002916DB02789B
:1012E000012A13D1427842F00402042A02D16FF09D
:1012F00002040BE000F1280252E8003F43EA010437
:1013000042E8004505B1F7E7FFF71CFD2046B0BDF8
:10131000DFF804C000DF70473D1B0008EFF30583D2
:101320002BB9EFF3108313B9EFF3118313B16FF0FF
:1013300005007047DFF804C000DF7047A91B0008F4
:10134000EFF3058028B9EFF3108010B9EFF31180A7
:1013500008B100207047DFF808C000DF704700BF09
:10136000F51B0008EFF305832BB9EFF3108313B9D6
:10137000EFF311830BB100207047DFF808C000DFE6
:10138000704700BF011C0008014629B180B5132039
:10139000FFF7D4FEBDE880400020704710B501463D
:1013A00049B188680C6870B182070FD1CA68002102
:1013B000102A15D222E000241149D1F8900038B14A
:1013C000FFF771FB0AE0C8680028F5D0002115E09E
:1013D000D1F8800010210122FFF7E1FA60B101216C
:1013E000817040F20311074A01800021C0E90141E8
:1013F000C16003494A6600E000200146084610BD6E
:1014000090170020690900080148007A704700BF62
:10141000901700200148C068704700BF9017002057
:101420002DE9F843DFF8648198F80800012800F0FE
:10143000A580002840F0A480554F4FF0FF30796D13
:101440004829C0F09F80FC68002C00F09B803D8AFA
:10145000002D00F0978008F108009C21FEF7A3FF03
:10146000A8F85450C8F85C40B868D7E90B41C8F8F0
:1014700040002046FFF7FCFA08B1C8F88040D7E9E1
:101480000541DFF81091D7E907562046C847D8F83C
:1014900080100028284618BF2146C8F8741031462D
:1014A000C847D8F88010002818BF2946C8F8781017
:1014B000D7E909412046C847D8F88010002818BF4E
:1014C00021467C6BC8F87C1044B12168D4E9022322
:1014D0002046FFF738FB08B1C8F88440BC6B44B124
:1014E0002168D4E902232046FFF72DFB08B1C8F894
:1014F0008840FC6B44B12168D4E902232046FFF701
:1015000022FB08B1C8F88C403C6C44B12168D4E996
:1015100002232046FFF717FB08B1C8F890407C6C07
:1015200044B12168D4E902232046FFF70CFB08B13F
:10153000C8F89440BC6C44B12168D4E90223204629
:10154000FFF701FB08B1C8F89840FC6C44B1216872
:10155000D4E902232046FFF7F6FA08B1C8F89C4008
:101560003C6D44B12168D4E902232046FFF7EBFA31
:1015700008B1C8F8A040012088F80800002001E068
:101580004FF0FF3001B0BDE8F08300BF901700209E
:101590004C5D0108710A0008B0B51E4C207A012884
:1015A0001CD1FFF797FDC8B11B48FF211B4D81756A
:1015B000817D026881F0FF01C2F30222B1FA81F15C
:1015C000C1F120018A4228BF511CFE2202FA01F11A
:1015D000C17468681249FFF713F810B14FF0FF307B
:1015E000B0BDFFF709F82061FEF7F0FF04F11C0021
:1015F000FFF7EEFC0028F1D0FFF798FD2878C00730
:101600000CBF0320022080F31488022020720020E7
:10161000B0BD00BF901700200CED00E04C5D01084C
:10162000D90200082DE9F84304461E4690460F46AD
:101630006FF00305002C67D0002F65D020780828B4
:1016400062D1607800285BD02046FEF751FF8146CA
:10165000B9F1000F42D020464946FEF79EFF626A6C
:1016600009F10C013846FEF776FEB8F1000F04F1DF
:101670000C064FF0000549461CBF99F8030088F896
:10168000000089F801503046FFF732FAA068D8B35D
:101690004078932837D13046FFF705FA06460025F3
:1016A00096B32046FFF794FC002101220746FFF77E
:1016B00061FD3846FFF7F0FC0746626A06F10C0050
:1016C000B968FEF748FE40F2071031463080B57029
:1016D000F868F0702046FEF72EFF15E086B18320F3
:1016E0003146FFF72BFD40B1094841692046FFF71D
:1016F0007AFCEFF30980C0E902786FF0010503E09E
:101700006FF0020500E00025284601B0BDE8F08337
:10171000901700202DE9F84F04460D46002764B1CC
:101720005DB105F10F01B4FA84F021F00306B6FAB9
:1017300086F10844202804D20027384601B0BDE8CD
:10174000F08F06FB04F872B1D2F808A01368D2E952
:101750000490BAF1000F11D05FEA8A71ECD1D16820
:101760003429E9D30DE000234FF0000935490093F7
:10177000D1F8A00078B1FFF796F912E0D1680029FE
:10178000DAD1B9F1000F31D000274045D5D319F097
:1017900003002DD0D1E7D1F8800034210122FFF7DA
:1017A000FEF882464FF0010BB9F1000F12D1BAF1E9
:1017B000000F0FD0234F41460022F86FFFF7EFF8DC
:1017C0008146B9F1000F07D048464146FEF7EBFDD0
:1017D00057461AE057461AE0BBF1000F14D0D7F86D
:1017E000A00060B15146FFF783F90DE00028A3D1B6
:1017F000BAF1000FBAD000934FF0000BD4E7D7F83E
:1018000080005146FFF70BF900274BF0020B002F29
:101810003FF493AF4FF48470009987F802B03246DA
:101820004B4638800020C7E90110C7E90950C7E9D5
:101830000B0007F10C002146FFF785F9014802492A
:1018400001677AE7901700209B0B00082DE9F84309
:101850000546994690460E466FF00307002D52D07C
:10186000002E50D0287808284DD16878002848D01C
:10187000A868D0B14078832817D12846FFF7A8FB85
:101880000021012204460027FFF774FC2046FFF7E1
:1018900003FC04466A6A3146A068FEF75CFDE06816
:1018A00088B380F8008000272DE005F10C00FFF7D9
:1018B000FAF804468CB16A6A04F10C003146FEF76E
:1018C0004AFD40F207100027214620802846A770D5
:1018D00084F80380FEF72FFE15E0B9F1000F10D059
:1018E00093204946FFF72AFC40B109484169284640
:1018F000FFF779FBEFF30980C0E902686FF0010799
:1019000001E06FF00207384601B0BDE8F08300BF88
:101910009017002070B5044623480E4645695DB314
:101920003CB32078042824D16078C8B3207E30B33B
:10193000E17811F0010F02D0E268AA422CD07EB308
:1019400088070AD5E06895F9201090F920208A428E
:1019500003DA80F82010FFF76CFB53203146FFF7C5
:10196000EDFB18B120462946FFF73DFB6FF0010063
:1019700070BD6FF0030070BD4FF0FF3070BDE560CB
:101980000021E86A0028C4E9041000D00461EC6278
:1019900001202076002070BDFF2801D00130F8E73B
:1019A0006FF0020070BD00BF9017002070B558B1F5
:1019B000D0E90065846884B1A10711D1C168002015
:1019C0001C2938BF70BD16E0002500261149D1F84A
:1019D000940038B1FFF767F80AE0C0680028F5D036
:1019E000002070BDD1F880001C210122FEF7D7FF36
:1019F000044664B10120A0704FF482701121208050
:101A000004F10800E5706660FEF7CDFC00E00024FC
:101A1000204670BD9017002070B504462C484069E0
:101A200070B154B12178042907D1617811B1E1680E
:101A3000814209D06FF0020404E06FF0030401E07A
:101A40004FF0FF34204670BD217E0029F2D00139CD
:101A500011F0FF0F217601D00024F3E7616909B18D
:101A600022690A61236900F12C052A46002B18BF60
:101A700003F114021160E178890711D590F8211063
:101A800009E093682BB193F920304DB2AB42C8BF47
:101A9000194602F114052A68002AF2D180F82010B4
:101AA000A06878B12046FFF793FA0021002205468E
:101AB0000026FFF75FFBE560E86AC4E904600120E7
:101AC000EC62207600200024FFF726FABAE700BF78
:101AD00090170020B0B5184D6C6964B3287A0228BD
:101AE00029D1686A38B3E06AFFF7C2F8A06918B173
:101AF00000210022FFF73EFBEFF30980A06305F110
:101B00001C00FFF765FAFFF711FB00206861E07821
:101B1000C00701D0A06920B12046BDE8B040FFF762
:101B20002BBA0020E06004206070686B0028A06081
:101B300000D0C4606C63B0BD90170020B0B50546FE
:101B40006FF003045DB1002909DB2878012806D174
:101B5000687840F00400042803D16FF002042046A6
:101B6000B0BD05F1280050E8002F42EA010440E82A
:101B7000004303B1F7E768783328F0D195F82320C4
:101B8000696A2846FEF75CFD01460029E7D095F812
:101B900023000C46012280075CBF686A21EA00042A
:101BA0002846FFF7E7FADAE7F8B505461048144685
:101BB0000E46476997B1002D13DB38462946324659
:101BC000FEF73EFD90B97CB13320214687F82360B3
:101BD0007D62FFF7B3FA6FF0010007E04FF0FF30CE
:101BE00004E06FF0030001E06FF0020001B0F0BD0F
:101BF0009017002001484069704700BF90170020EF
:101C00002DE9FE4F8046B8F1000F21D06AB102F1F4
:101C1000100A9AE88006D2E900439568B5B1A80792
:101C200016D1D068442813D317E04FF0180A0023C8
:101C300000274FF000090024644A0293D2F888007C
:101C4000CDE90014C8B1FEF72EFF1CE0D06820B12A
:101C50000026304603B0BDE8F08F37B10026B9F159
:101C6000000FF6D017F00700F3D1BAF1000F38D00B
:101C7000AAF101003728EBD835E0D2F880004421E2
:101C80000122FEF78CFE05464FF0010B67B95DB1EE
:101C9000B9F1000F0AD04D4849460022406FFEF7C7
:101CA0007EFE074687B911E02E463EE04748484988
:101CB000D0F88400D1F854900028ECD0FEF7F3FE61
:101CC00007461FB14BF0100B2E462CE0BBF1000F66
:101CD0001CD03E49D1F88800E0B12946FEF708FF44
:101CE0001DE04FF0180AB9F1000F06D00026B9F137
:101CF000480FAED319F00700ABD1002D3FF49CAFD5
:101D0000CDE9001402934FF0000BBFE74FF0000B3A
:101D1000002707E0D1F880002946FEF780FE002763
:101D20004FF0010B00264BF0020B002E3FF491AF59
:101D300040F2011086F802B0182130800298F0704D
:101D40000198706006F10800FEF72DFB07EB090112
:101D5000FD2086F821A086F820A086F82200002029
:101D6000403986F82F00C6F82B00C6F82700C6F8C1
:101D70002300C6E90C79C6E90E181649009D3960A2
:101D80001349097849070AD511213A1D4FF0CC3380
:101D9000A1EB990101E008C201310029FBD1B16B2F
:101DA000002202E041F8220001320D2AFAD10A4A4B
:101DB0004FF080700D62C1E90D28C86303480749E0
:101DC00001663046FFF7A8F843E700BF90170020F0
:101DD0004C5D0108A52E5AE2B51200085B10000800
:101DE00049490A6822F440320A600A6843681A4383
:101DF0000A6001684A6822F480724A6001684A6891
:101E0000036942EA03224A6001684A6822F040728C
:101E10004A6001684A6883681A434A6001688A68B0
:101E200022F400628A6001688A68C3681A438A6083
:101E3000816A6FF07062D14214D001688A6822F022
:101E400070628A6001688A68836A1A438A600168DE
:101E50008A6822F040528A6001688A68C36A1A431D
:101E60008A6009E001688A6822F070628A6001680D
:101E70008A6822F040528A6001688A6822F0020271
:101E80008A6001688A68836942EA43028A60016A5B
:101E900089B101684A6842F400624A6001684A6890
:101EA00022F460424A6001684B68426A521E43EA6B
:101EB00042324A6004E001684A6822F400624A60E3
:101EC0000168CA6A22F47002CA620168CB6A828B16
:101ED000521E43EA0252CA6201688A6822F4007202
:101EE0008A6001688A68036B42EA43228A6001685B
:101EF0008A6822F480628A6001688A68406942EADE
:101F0000802088607047000004230140002800DC26
:101F10004042704770B51B481949016000F1340117
:101F200002220A6007244C6004238B60CC600A61A3
:101F30004A618A61002444608460C3602021016199
:101F4000402141614FF4C0718161C461910201621D
:101F5000490041628462002100F05EF809490948A5
:101F6000343106F0C1FB084D10B10120287000E0AB
:101F70002C7040F2036000F009F8287870BD000072
:101F8000400100A040490020781300202DE9F843CB
:101F900081460027009701251E4C256010266660AB
:101FA000A560E7604FF6FF7821464246A1F1500058
:101FB00006F0D0FB012005F0FBF8022020606660EF
:101FC000A560E7602146A1F15000424606F0C2FB41
:101FD0000320206066600820A060E7602146A1F130
:101FE0005000424606F0B6FB4FF40C7300930420F9
:101FF00020606660A560E3602146A1F15000424682
:1020000006F0A8FBA4F150004946BDE8F84306F0ED
:102010008EBB00009049002030B587B004464E4981
:10202000086840F001000860086800F001000190B5
:1020300049490839086840F480000860086800F4DD
:1020400080000190086840F008000860086800F00F
:1020500008000190086840F010000860086800F06F
:1020600010000190086840F020000860086800F047
:1020700020000190086840F040000860086800F007
:1020800040000190086840F080000860086800F097
:1020900080000190086840F480700860086800F4CF
:1020A0008070019002200390012004900325059583
:1020B0000C2006904CF203700290284802A905F00B
:1020C00089F84FF683700290254802A905F082F83E
:1020D0004FF63F000290234802A905F07BF848F232
:1020E00037100290204802A905F074F84FF62C70C2
:1020F00002901E4802A905F06DF840F2FF600290C0
:102100001B4802A905F066F81A4900224A6080209F
:1021100088608000C86040000861800048618000DD
:102120008861CA61C00008624A628D62CA620A633D
:102130001148086021638C63084604F029FD0D48AE
:1021400004F05AFD00220F21382005F0F9FC382058
:1021500005F0E8FC07B030BD38380240000C024002
:10216000001002400014024000180240001C02400F
:102170000020024080480020106402400120704787
:1021800010B500240448012105F014F9012800D1FC
:102190000124204610BD00000000024000B587B0B9
:1021A0000A48016841F001010160006800F0010087
:1021B00001900120029000200390049002A904489D
:1021C00005F008F807B0002000BD000030380240DC
:1021D00000000240F0B5BFF34F8FBFF36F8F1B4974
:1021E00000200860BFF34F8FBFF36F8F184E316828
:1021F00041F400313160BFF34F8FBFF36F8F14494B
:1022000070310860BFF34F8F081F0068C0F34E3174
:102210000E4A43F6FF771032C0F3C905284607EA95
:10222000411343EA80741460401E441CF9D1491ED6
:10223000481CF3D1BFF34F8F306840F480303060DA
:10224000BFF34F8FBFF36F8FF0BD000050EF00E082
:1022500014ED00E002490220096888607047000020
:10226000484E00200168CAB2103A1823B2FBF3F2BC
:10227000064B9B5CC365032A6FF3090102D9091D54
:10228000816500E08165806D7047000018320108AB
:10229000014610B500208A6A4FF0C0748B69002B8C
:1022A0000ED0B3F5005F1AD062B3012A2AD0022AF9
:1022B00028D0032A03D1C96AC90100D5012010BD65
:1022C0001AB1012A06D0022AF9D1C96AC901F6D584
:1022D000012010BDC96AA142FBD1012010BD52B13D
:1022E000012A0AD0022A06D0032AF7D1C96AA142DC
:1022F000F4D1012010BD012010BDC96AC901FBD570
:10230000012010BD012010BD10B5029C42EA8111D0
:1023100041EA032141EA0441C16610BD1CB5012810
:1023200008D84878152200900B780021064804F060
:10233000F9FE1CBD0A5C0346CDE9002102483922A2
:10234000002104F09BFE1CBDA04E0020FEE730B52E
:10235000D1E901230D681A43D1E9033423431A4319
:102360004B691A438B691A43D1E90734496A012D35
:1023700008D005686FF30E051A4322430A432A4327
:1023800002600BE0056825F4F845234329430B431D
:1023900041686FF30E010A4303604260002030BDC4
:1023A000426942EA410141610020704708B5D1E924
:1023B00000231A438B68C9685B1E5B0143EA412115
:1023C0000A43009200990161002008BDF0B54B68F6
:1023D0000C685B1E4D69641E44EA03148B686D1E15
:1023E0005B1E44EA0326CB680C6989695B1E641E88
:1023F000491E012A0DD0826802F0704246EA03337A
:1024000043EA044343EA055343EA0161114381600F
:1024100010E08268084F3A401B0343EA0553134318
:10242000C26802F0704246EA044444EA0161114382
:102430008360C1600020F0BDFF0F0FFF2DE9F04762
:10244000044640688EB00027804601F049FC0090A9
:10245000B0F87CA0D0F86890D0F88060D0F88850B0
:10246000C06D00B10768684601F090FC05E069683E
:1024700020468847002843D12D68002DF7D12068D9
:10248000172853D00CDC0F283DD004DC0B2877D064
:102490000D2825D18BE0112810D0142820D13BE045
:1024A000262846D004DC1E2851D0202818D18AE0E6
:1024B0002A2816D0B0F5107F12D128E04046E568F2
:1024C00001F00EFC0290697A39B9297A012904D108
:1024D00030F87C1F41F48071018002A801F056FCA5
:1024E00075E0404601F0FCFB0090E16811B1C0F8D6
:1024F000841002E0D0F88400E060684601F046FCF9
:102500000EB0BDE8F087D7B34046B8475FE021463C
:1025100040460EF031FFF3E705A9404600F001FB0D
:10252000E0680699016007994160E9E7C4F80C90FA
:10253000E6E7E0680228E3D1CDF83080E0680D904E
:1025400027200A900AA9A0680AF00CF8D8E7E068EA
:10255000012804D00021404600F0B1FAD0E730460F
:1025600009F0C7F868B1304609F068FA304608F05B
:1025700099FF98B10121304608F09EFA0EE026E05E
:102580002FE0484609F0AEFA0646404601F0A8FBA7
:102590000090C0F88060684601F0F8FB01214046D9
:1025A00000F08DFA002EABD10020E060A8E75FEAD2
:1025B0000A700CD4E068C06848B1007A38B140466F
:1025C00009F03CFA03E0214640460EF01CFC21468F
:1025D000404608F0DCF9002892D0204608F082FC42
:1025E0008EE7404601F07CFB0090703001F0E4FA89
:1025F000684673E7F0B587B01D46DDE90D73044604
:1026000000200C9ECDE90304CDE90510CDE90002C0
:1026100002903A463146284600F002F807B0F0BD75
:102620002DE9F04F8BB09846DDE9155691468A4664
:102630008346149F1A9C02F0DBF93348603445F45A
:102640008055CDE90204CDE9007543464A4651461E
:10265000584608F08FFB04004FD001F041FB3022B8
:102660000490179908F0C8FA0498282227493430B2
:10267000FDF771FE04981999244F4166A0F87C601B
:102680000026C0F88060C666083FC0F88860796898
:10269000C16504A801F07AFB05A9204600F041FAC3
:1026A0001B4841F2827103960094CDE90110BDF9F7
:1026B0001E00BDF91A10BDF91C20431ABDF91800FF
:1026C0005B1C121A521C08F055FB064678684168DC
:1026D00020468847204601F003FB0490866604A844
:1026E00001F054FB42F20400054202D1204608F0FA
:1026F000ABFC2046189900F0F1F903F009F90BB092
:102700002046BDE8F08F00003D240008EC140020B6
:10271000DD2C00082DE9F041044694B0006800F07B
:10272000B7F908B1D94D01E0D84D2C3560681528AE
:102730001ED00CDC0B281FD004DC00287ED005281E
:102740007DD12FE10E287BD01228F9D141E1162846
:1027500006D0172808D0182808D01C28F0D109E086
:10276000E86914B0BDE8F081286AFAE7686AF8E71A
:10277000A86AF6E76869F4E720680B901C200C90C3
:10278000206801F0ADFA0390016D0BA8884706465A
:1027900003A801F0FBFA022E0FDB95E807008DE895
:1027A0000700D4E904023346A16903F0B3FC2069B1
:1027B0008719A069A0EB06082CE0286802F0B9FD93
:1027C0002169E8690A18521E606901F09DFEA2693C
:1027D000E869111A491C606901F096FED4E9040702
:1027E0007F1C394601F0E0FE3946A06901F0DCFEAD
:1027F000686802F09EFD20693946401C01F0D4FE55
:10280000A0693946401E01F0CFFEA0692769A0F1FA
:102810000208BF1C286802F08CFD424639466069F8
:1028200001F072FE686802F084FD60694246394634
:10283000401C01F069FE686A022802E015E1B0E080
:1028400000E10BDDA86802F074FD61696A6A881C0A
:102850008B180146424638465B1E27E0296AB14282
:1028600026DD6069022E074600F1020801DB3744CD
:1028700001E007F10207206901DB304401E000F1CB
:10288000020022693B460A444146A2F1010201F0DE
:102890004BFF022E02DBA069821B01E0A269921E9F
:1028A000A069E9693B46401A4146401C01F03CFFE3
:1028B000022E02DB6069064401E06669B61CE76926
:1028C00028687F1E02F035FD3A463146206901F046
:1028D000DBFE3A463146A06901F0D6FEE76968683A
:1028E000BF1E02F026FD20693A463146401C01F029
:1028F000CBFEA0693A463146401E01F0C5FEE869AC
:10290000022802DC286A022823DDA86A022802DDE8
:10291000E1690F1A01E0E769BF1EA86802F009FD2E
:10292000E969022909DD20693B46421800F1020CE1
:1029300031466046521E01F0F7FE286A022808DD83
:10294000A269E8693B46101A3146401C921E01F00C
:10295000EBFE286802F0EDFCD4E90620216901F0C5
:10296000D3FD686802F0E5FCD4E906202169401E29
:10297000491C521E01F0C8FDA86A022811DDA16998
:102980002669E469A1F10208271AA41EB61C7F1C5F
:10299000A86802F0CEFC234642463946304601F094
:1029A000C3FE71E0208A00B2ADF81400A18A09B21A
:1029B000ADF81610228B12B2ADF81820A38B1BB203
:1029C000ADF81A302C69ED68CDE9005401F036FD00
:1029D0005AE0208A298B0844ADF81400A08AADF88B
:1029E0001600208B298B401AADF81800A08BADF88B
:1029F0001A00206801F074F90390006FF0B1022012
:102A000002F02EFD039890F87C10C1F3C00100EB9A
:102A10008100006C02F08DFC0398406B02F0A6FC74
:102A20000398006F01F05CF903990990B1F95A20FD
:102A300005A901F09DFC09A801F0A8F903A801F07F
:102A4000A5F921E0208AADF81400A08AADF816009F
:102A5000208BADF81800A08BADF81A00A86802F022
:102A600068FC05A801F08CFE0EE0206801F038F942
:102A7000039030F85A1F41F00C01018003A801F0C7
:102A800085F9206809F086F800206AE644160020DF
:102A900038B505004FF000040FD001F0A9FF28461B
:102AA00001F01EF9009090F87C00000700D5012489
:102AB000684601F06BF902F02BFF204638BD70B577
:102AC0000D46040009D001F093FF294620460FF07F
:102AD0009DF8BDE8704002F01BBF70BD7CB50D468F
:102AE00004001DD001F084FF204601F0F9F80090A9
:102AF000006F0190684601F049F9294601A803F0EA
:102B0000E9FD58B1204601F0EBF80090019901670A
:102B1000684601F03BF9204608F09CFD02F0F8FE03
:102B20007CBD2DE9F34F85B000270C46B8460598CB
:102B300001F0D6F80090C06D0121856805982A68DB
:102B4000904782462A6803210598904704902A6896
:102B500002210598904703902A6800210598904724
:102B60000646009809F0F2F98346009809F0F5F955
:102B70008146009890F83210890601D5B0F9588046
:102B800000F036F805460098C06E10B108F063FCFE
:102B9000074625806780A4F804A0049AABEB0200E6
:102BA00006EB0802401E2A4420813A44E280039B3F
:102BB000A9EB0302521E6281A4F80CA020827019B6
:102BC000E681401E6082684601F0E0F8B4F90C002E
:102BD0000190B4F91000029002AA01A9059800F032
:102BE00039F80198A0810298208207B0BDE8F08FE3
:102BF00010B50146002091F83220920607D5B1F9B0
:102C00005400002803D1486B01F08EFE801C10BDDB
:102C100070B58AB00C46054601F062F80990C06DA7
:102C2000866809A801F0B2F8009534B1012C06D0ED
:102C3000022C0BD0032C04D10AE0182000E016204F
:102C400001907168684688470AB070BD1520F7E7A3
:102C50001720F5E72DE9FC4117468846044601F0A8
:102C60003FF80090C16D056868468E6801F08EF8E7
:102C700032680021204690470646204608F0A2FA16
:102C800027E000BF01F02CF80190B0F900102AB243
:102C9000B0F90430891A9A1AB0F90230A3EB25432F
:102CA000B34210D190F82800000605D53868884254
:102CB00009DB491E396006E0D8F80000904202DCCA
:102CC000521CC8F8002001A801F060F8204608F066
:102CD00017FB0400D6D1BDE8FC8100002DE9F043CC
:102CE0000446406889B0054608F028FB814600F09C
:102CF000F7FF0290D0F84880D0F88070466E02A8A6
:102D000001F044F82068172852D008DC0E2839D08A
:102D10000F2811D014284BD015283CD148E01E288C
:102D20001DD01F2829D022283FD0312833D10020A0
:102D3000E06009B0BDE8F0831F494046884503D0F4
:102D400006F012FA01F052F9002EF2D0D4E9021284
:102D50002068CDE90405CDE9061204A81FE0E0686B
:102D60000028E6D02FB1AF4203D0384608F066FE07
:102D7000DFE7284608F0B6FEDBE72146484607F0C5
:102D800006FED6E7E0684168002904DD00680928EE
:102D9000EFD00A2805D05EB12046C4F80490B047B1
:102DA000C7E7284608F0D2FEC3E7C4F80C80C0E7A6
:102DB000204608F097F8BCE7785634FF1CB500248D
:102DC000019401AC009400F0E7F81CBD2DE9FF4F21
:102DD00083B0814606988A46A0EB0A08109E002020
:102DE0000090A2EB09043568934654EA080018D015
:102DF0002046FFF78BF807464046FFF787F88742E3
:102E00000BDA2046444680464846D146824658461C
:102E1000DDF818B0069001200090002C07DD204658
:102E200006E007B04846BDE8F04F00F03BB960420D
:102E3000A0420AD04846D9466442C8F100088346F9
:102E40004FF0FF37DDF818A000E001275148B8F136
:102E5000000F11D004EBD4714FEA610B01DACBF112
:102E6000000B4C480068807E88B3002F02DA30687F
:102E70002044306000257BE000990029016821D0C2
:102E8000897E11B10027804615E007B05A464946B1
:102E90005046BDE8F04F05F059BE28466D1C0EF0B7
:102EA00081FF38B9D8F8000009EB0701406E42688D
:102EB000504690477F1CA742EFDD6D1E356007B07E
:102EC000BDE8F08F8A7E1AB10027804617E019E02E
:102ED000486E5A465146036807B04846BDE8F04F71
:102EE000184728466D1C0EF05DFF38B9D8F8001061
:102EF00009EB0700496E4A68514690477F1CA7427C
:102F0000EFDDDAE700250FE008FB05B090FBF4F1F8
:102F100001EB0A00009951B11E4A09EB0501126844
:102F2000526E526890476D1CA542EDDDC7E7194906
:102F300009EB05030968496E4A6801461846F1E73E
:102F400008FB05B090FBF4F101EB0A00019030683A
:102F5000384430600EF026FF48B9009890B10D4813
:102F600009EB05010068406E4268019890476D1CAE
:102F7000A542E5DD3068002F01DA20443060C01B37
:102F800030609CE7034909EB05000968496E4A680F
:102F90000199EBE7201400202DE9FF470F46404937
:102FA0001646804609680C981D460A7E012A1CD0E8
:102FB000A8EB0600791B50EA01031CD0A2F101091D
:102FC0000FF012FE00F58060824603F03EFC00FB2D
:102FD00009F4504603F03EFC00FB09F1002C0CDA2A
:102FE000C4F50070801240420AE000903246394633
:102FF0004046FFF7EBFEBDE8FF8704F50074A01222
:10300000002904DAC1F5007189124C4202E001F591
:1030100000718C12002804DD411C01EBD1714910B4
:1030200003E000EBD0714910401E00EBD07042105D
:10303000002C04DD601C00EBD070401003E004EBBA
:10304000D4704010641E04EBD47308EB0104ADF897
:1030500000403C18ADF80240A8EB02045B10B21A25
:10306000ADF80440ADF808203144FC1AEA1AADF876
:103070000C102844ADF80A20ADF80E000023ADF87E
:1030800006401A460421684600F07AF83946404660
:103090000BF08EFF294630460BF08AFFABE70000AD
:1030A00020140020064A13681A7E012A05D0521EF9
:1030B00002EBD272521000F005B85A6E52681047F7
:1030C000201400202DE9F05F0646884640F2C32018
:1030D00002FB00F14FF47A7091FBF0F702FB02F172
:1030E00002EBD27001EB600B1446B118234A301B7F
:1030F0007F1C1268526E13680A46414698470125A4
:1031000038E000BF05FB05F004FB040159451CDD58
:10311000BC4219DD194B06EB050AA6EB05091B6835
:10312000AAF1010208EB04015B6E09F101001B68C2
:103130009847124BAAF10102A8EB04011B6809F1A0
:1031400001005B6E1B689847641E0C4B3219301BE4
:103150001B68924608EB05015B6E81461B68984729
:10316000064B5246A8EB05011B6848465B6E1B6880
:1031700098476D1CBD42C5DDBDE8F09F20140020BE
:103180002DE9FF4F43F6FF740F46664283B09B461E
:10319000814600210BE000BF09EB8100B0F902007D
:1031A000A04200DA0446B04200DD0646491CB9429E
:1031B000F2DB67480068406900280DD0B0F90610BE
:1031C0001A46A1EB0B01B14200DA0E46B0F902003B
:1031D000801AA04200DD0446B4E0DFF878A10020A8
:1031E0000546CAF8000088E0781E854201DA6B1CAB
:1031F00000E0002309EB850C09EB8302BCF9020017
:10320000B2F90210A04244D1A14215D139F92330BC
:10321000059A39F9251003EB020C4D4A05981268FE
:10322000084404EB0B01526E6045136801DA6246F4
:103230002AE00246604627E02846A4464FF00008F0
:103240007A1E0BE008B1401E00E0781E09EB8003F7
:10325000B3F90230634504D108F101089045F1DB70
:103260002346A34248D01A1B39F92500A1EB040CD0
:10327000059B92EA0C0F09D4354A184404EB0B0164
:103280001268526E13680246984735E009F018FA42
:1032900032E0A14230D001DBA04203DDA0422BDBB3
:1032A000A14229DCE04688420ADC0346A04223DC36
:1032B0000846A14220DBB8F900C0B2F9001008E0CE
:1032C0000B46A14218DCA04216DBB2F900C0B8F9E7
:1032D0000010E21AA1EB0C0151430029A0EB0302FC
:1032E00002DD01EB620102E0A1EB6201491CC01AA0
:1032F00091FBF0F06044C9E76D1CBD42FFF674AF6E
:103300000598009004EB0B000190002080460546D4
:1033100013E01149B8F1000F31F915A009D0009957
:1033200001EB0A0208440A490968496E0B680199D1
:10333000984788F0010850466D1C064909688D427F
:10334000E7DB641CB4427FF748AF07B0BDE8F08FFD
:1033500020140020F8160020205100200E4810B53F
:10336000006801F0DBFF0D48006801F0E2FF01207A
:1033700002F058F8002002F063F8002002F070F824
:10338000002001F0E7FF0648006801F0EFFFBDE80C
:103390001040002002F018B81C140020181400205F
:1033A0001414002033B583B004001BD001F020FBBF
:1033B000204600F095FC0190456E01A800F0E6FC67
:1033C000049800F08DFC00908460684600F0DEFCFC
:1033D000042204A9284600F0FBFC204608F03AF934
:1033E00002F096FA05B030BD2DE9F0410446002503
:1033F000D4E90007B0F5407F00D1012521463846C9
:1034000007F0C5FA064615B138460DF050FC002EFF
:103410002FD02068052806D00B280ED00F2806D004
:10342000262821D10EE038460DF041FC1CE038463C
:10343000E168BDE8F0410DF003BE3846BDE8F0415B
:103440000DF010BDE06805280ED1384607F0A8FF42
:10345000A168884205D0384607F092FFA1688842EB
:1034600002D160680DF038FF2046BDE8F04107F05A
:1034700039BDBDE8F081F0B585B00DF1280C9CE8B0
:10348000F0004FF0000C8DE8F01000F003F805B0EC
:10349000F0BD00002DE9F04F85B09846DDE90E56ED
:1034A00091468A468346109F129C01F0A1FA184863
:1034B0006C34CDE90204CDE9005643464A465146F4
:1034C000584607F057FC04001BD000F0BEFC054630
:1034D00000F0BBFC0646204600F002FC0490C0E968
:1034E00019560022119907F087FB049830220949E8
:1034F0003430FCF730FF0498A0F8787004A800F08E
:1035000045FC02F005FA05B02046BDE8F08F00004A
:10351000E93300081415002013B582B0044601F009
:1035200067FA204600F0DCFB009060B1406A00F0D2
:10353000D7FB01460190022303AA009800F087F808
:1035400001A800F023FC684600F020FC02F0E0F93E
:103550001FBD00002DE9F04385B01D4690460F4683
:10356000814601F045FA2C2000F0E0FA060025D053
:10357000780000F0DBFA04000FD0B8F1000F0CD097
:103580005DB1204600F0ACFB0F4B00906A001B6859
:1035900041469847684600F0F9FB304600F0A0FB32
:1035A0000A49029000F10C02446282E8A202084932
:1035B00001600849416002A800F0E8FB02F0A8F9A8
:1035C00005B03046BDE8F083E815002099040108F5
:1035D00001120108F50E0108F8B515460E46070060
:1035E0004FF0000415D001F003FA384600F078FBE4
:1035F0000090042D08D200EB8500446BB44203D048
:103600004663384608F026F8684600F0BFFB02F033
:103610007FF92046F8BDF8B50D4606004FF00004CE
:1036200013D001F0E5F9304600F05AFB009090F815
:103630006C40AC4204D080F86C50304608F00AF878
:10364000684600F0A3FB02F063F92046F8BD2DE9BF
:10365000F041044680681D4617460E46002826D0D5
:10366000D4E9040290420ED1521E6A4371193046C9
:10367000FCF771FE20692A46401E05FB00603946B2
:10368000FCF769FE0EE005FB0013401C20612A4692
:1036900039461846FCF75FFEE16819B12046BDE8DF
:1036A000F0410847A068BDE8F04100F002B8BDE86D
:1036B000F08110B58AB0044600F012FB09A904AAF3
:1036C000CDE9002105AB089006AA07A90CF077FB0D
:1036D00008A800F05BFB02A9204607F0BFFDBDF87B
:1036E000080007990844ADF80800BDF80A000699DB
:1036F0000844ADF80A00BDF80C000599401AADF871
:103700000C00BDF80E000499401AADF80E0002A995
:10371000204607F05FFF0AB010BD0000014AC2E971
:1037200000017047C0130020014AC2E90001704740
:10373000C8130020014AC2E900017047D0130020DD
:10374000014AC2E900017047BC1400202DE9F04F86
:10375000DFF828B191B04FF0FF35DBF80030B3F956
:1037600022100691DE69B3F92490F469A18981429F
:1037700006D8E289824203D3471AD4F8008012E0C7
:10378000D4E9018100296FD00A8882426CD84D8823
:10379000854269D3801A82B2486800EB8200B0F992
:1037A0000070B0F90250781C5ED0307EA17C10FB16
:1037B00001FA217CCDE90701B3F92A60304605F012
:1037C00039FDC0B20E90DBF8000007FB0A81A37C34
:1037D000826B0127CDE90412CDE90273C069089A12
:1037E000C17E807ECDE90001DDE90603494605F092
:1037F0004BF8681C18D046F0020005F01BFDDBF802
:103800000000A37C05FB0A81826BCDE90273CDE940
:103810000412C069089AC17E807ECDE90001DDE90D
:103820000603494605F030F8DBF800005D46C06944
:10383000417E007E814214D9022E12D086F004000F
:1038400005F0F8FC2868C069027EC37E12FB039174
:10385000437E857E089A06984B4412FB050205F0CC
:103860009FF90E9805F0E6FCDBF80000627C418CC5
:103870001144418411B0BDE8F08F000020140020F5
:1038800004480068C069C06909B1027C0A60407CD4
:103890007047000020140020022008807047C06993
:1038A00082898A4202D8C2898A4210D2806880B155
:1038B00002888A420DD843888B420AD3406800EBC5
:1038C0008100A0EB8200B0F90000002801DB01209C
:1038D00070470020704700002DE9F043304C03464C
:1038E00087B020681946B0F92A60C069C06900F045
:1038F00086F8002850D041680088181A01EBC005EE
:103900003046AF7805F096FC814620686A6801234E
:10391000816BCDE90237CDE90421C169CB7E8A7E76
:10392000CDE900230B7EB0F924102A78B0F92200EB
:1039300004F0AAFF2068C069417E027E91421FD92F
:10394000C07E11FB00F812FB00F7022E18D000F029
:1039500062FF064600F028FF01F0EBFC21682A78A0
:10396000CB69B1F92200DB7E12FB0302B1F924100E
:1039700001EB0803394405F013F9304601F0D9FC96
:10398000484605F057FC20686A78C369B0F92210F0
:103990009B7E12FB0311418407B0BDE8F083000059
:1039A0002014002030B50F4C05460B4620682946F0
:1039B000C069C06900F023F8002812D0416800886F
:1039C00024682A1A0120E46900EBC200085CA47E86
:1039D00010FB04F0002B04D011F8321011FB04F19D
:1039E000196030BD2014002001200880704700B508
:1039F000C06900F004F8002800D0012000BD06E0F6
:103A000002888A4202D842888A4202D2806800280C
:103A1000F6D170472DE9F0410025154E154C18E000
:103A20002069C5EB451700EB87007422001D316843
:103A3000FCF791FC2069002140F8271000EB87007B
:103A400000F10C018161011D0A1DC0E90F126D1CFE
:103A50004164A0688542E3DB0CF064FA2169C0EBA5
:103A6000401001EB8000001D3060BDE8F0810000D7
:103A7000201400200016002070B510490E48086080
:103A8000084602F01FFE0D4C143CA068C0EB40102D
:103A90008500284600F09EF8094B20612A461B68E5
:103AA000002198474FF0FF30206001F053FFBDE840
:103AB00070400CF037BA00001D10010814160020E9
:103AC000E4150020F8B50C0005460ED000F090FF7C
:103AD000204600F01BF8060010D000F001F9224645
:103AE000009025B12946074B03E00020F8BD064BA6
:103AF00000211B689847684600F048F901F008FF6C
:103B00003046F8BDE8150020E415002010B504008B
:103B100009D000F06DFF204608F038FE044601F0A1
:103B2000F7FE204610BD002010BD000038B5054648
:103B300000F05EFF2846FFF7E9FF04000AD000F01E
:103B4000CFF8064B00902A461B680021984768462C
:103B500000F01CF901F0DCFE204638BDE415002021
:103B6000024A106021F0030050607047E84F0020C7
:103B700010B5040011D000F03BFF0848042101EB10
:103B8000C401406B4158486808F0B8FD20460DF06C
:103B900079FFBDE8104001F0BBBE10BD284F0020EA
:103BA000002805D0034AD16B016001B14860D063A1
:103BB00070470000284F002010B5044600F018FFA1
:103BC0002068FFF7D5FF00202060BDE8104001F01D
:103BD0009FBE00002DE9F04104460CF0BDFB2848D3
:103BE000E41C24F00305016C2D1DA94200D90D46EB
:103BF000C46B13E054F8042CAA420ED184B121689E
:103C000009B162684A60616809B122680A60C26BE2
:103C1000A24231D12168C1632EE02468002CE9D191
:103C20008046816BC0680F1857F8040C3E1A306844
:103C300038B100200DF09AFF57F8040C3E1A306896
:103C4000D0B97068A84217DB3044441B3046241DAD
:103C50000DF044FFD8F80C10491BC8F80C10D8F828
:103C600014102944C8F814107068401B02D0314663
:103C700008F044FD44F8045C2046BDE8F0810000F3
:103C8000284F002010B500240CF066FB0C490F20D3
:103C900001EBC002526C1AB101EBC000406C08E0AD
:103CA000401EF5D508E04168A14200D90C46806865
:103CB00010B180680028F6D1A4F10C0010BD0000FE
:103CC000284F0020002138B10449042202EBC00033
:103CD000496B085841680C3908467047284F002046
:103CE0000549CA69521CCA61496B01EBC0010A78D7
:103CF000521C0A7000F062B8284F00207CB50646BE
:103D00000C460846FFF702FF050021D006B33046F7
:103D1000FFF7D8FFA04200DA044600F069FE28460B
:103D2000FFF7DEFF00903046FFF7DAFF094B019006
:103D300001461B68224600989847684600F026F81E
:103D400001A800F023F83046FFF712FF01F0E0FD74
:103D500028467CBDE815002010B500F049FEFFF7AD
:103D600091FF64220849B0F5800F04D990FBF2F46A
:103D7000086A444303E0096A4143B1FBF2F401F0ED
:103D8000C7FD204610BD0000284F00200A490268E8
:103D90004B6B52F8082C03EBC2021378022B03D3AF
:103DA000CB690BB15B1ECB611178491E11700021EC
:103DB0000160084670470000284F00200349042294
:103DC00002EBC000496B085808307047284F0020AC
:103DD0002DE9FC414FF000060B465FEA000834462F
:103DE0002BD032B111461846FFF76CFE060000D109
:103DF00001244046FFF774FF009007884568684635
:103E0000FFF7C4FFCCB9B9002846091DFFF776FFBC
:103E1000050015D0FFF764FF019040F8276001A866
:103E2000FFF7B4FF4046FFF75BFF00904560018855
:103E3000491C01806846FFF7A9FF2046BDE8FC81C8
:103E40003046FFF795FE0124F7E70820FFF76EBE26
:103E50007CB5050023D0FFF743FF00904068C0B158
:103E6000FFF73EFF0024019005E0019800EB84007D
:103E7000FFF7A2FE641C00980088A042F5DC01A8B0
:103E8000FFF784FF0098001DFFF796FE00990020C1
:103E900008806846FFF77AFF2846FFF769FE7CBD79
:103EA00038B5002430B1FFF71BFF00900488684646
:103EB000FFF76CFF204638BD38B50D46002448B1E9
:103EC000FFF70EFF2946009000F006F8044668460A
:103ED000FFF75CFF204638BD38B50D460188002449
:103EE000A94209D9406838B1FFF7FAFE009050F8AE
:103EF00025406846FFF74AFF204638BD70B50C469E
:103F0000054600F0ABFDC1B223462846BDE870402F
:103F1000002200F001B80000F0B52D271C68B0F1B8
:103F2000004F08D0002600280DDA651C1D602770A0
:103F30004042012408E0651C01261D606FF000402E
:103F40002770491E01E00024091BC9B22AB3491E8B
:103F5000C9B222E00C46491EC9B2944205D1124CA6
:103F600027781C68651C1D602770104C54F8215080
:103F700090FBF5F4E4B20A2C11D804FB150011B93A
:103F80000EB1641CE4B20A2C02D10124491CC9B24E
:103F90001D686F1C30341F602C700029DAD119683D
:103FA00000200870F0BD00000C140020C032010891
:103FB00010B5C2B2CBB2D21A00D5524293B25B4313
:103FC000C0F30722C1F30724121B00D55242000C94
:103FD00092B2A0EB114002FB023200B2002801DADB
:103FE000404200B280B200FB002010BD10B500219D
:103FF000084600F0AFFC43F6FF725042BDE81040A7
:1040000013460146AFF300802DE9FC411C461546DE
:104010000E46074600F0ECFC042005F00BF9804644
:1040200012484069C16C006D0F4406440D440444BD
:10403000ADF80070ADF80450ADF80260ADF8064080
:10404000684607F091FF07E023462A463146384686
:1040500004F0A6FD07F03CFF0028F5D1404605F02E
:10406000E9F801F055FCBDE8FC8100000C140020CB
:10407000B0F90630B0F90420B0F90210B0F9000030
:10408000FFF7C2BF2DE9F0411C4616460D46074614
:10409000022B02DB0020BDE8F0811C20FFF79AFD17
:1040A0000028F8D00DB105610AE0094A52F8241041
:1040B00009B905E011460A68002AFBD109690161C6
:1040C00084618682002101604160C0E90217E2E755
:1040D0005414002070B51D46FFF7D4FF040009D02A
:1040E00000F00EF8E068006820B90348006800EBB3
:1040F00085008465204670BD20140020FFF750BD68
:1041000070B5C0B38269022A36DA2149531C0C7893
:104110009C4200DA0B701F4C54F8221019B944F875
:10412000220032E019464B68002BFBD106E0CB6839
:10413000C5681B682D68AB4203DD09680029F6D10C
:104140001AE0C1B1CB68C6681B683668B3420CD1AF
:10415000838A012B05D008E01946DB681B68AB4257
:1041600003DB0B68002BF7D129B14B6833B1186022
:104170004A68426004E0FFE7012070BD44F8220075
:104180004860884200D100210160002070BD00001D
:104190007A1400205414002010B503E00468FFF7DF
:1041A000AFFF20460028F9D110BD000010B50C4B20
:1041B0008269002153F82240844205D1046843F803
:1041C0002240026802B1516042680AB1036813607C
:1041D00002680AB1436853600160416010BD00008D
:1041E0005414002000207047022801DB0020704793
:1041F000054951F8200004E0C16809680029F6D09B
:1042000000680028F8D17047541400202DE9FC47BD
:1042100006005FD000F0ECFB00F016FB3C4C814642
:104220002068B0F9228000F061FB216807468A8C83
:10423000D01B888441E000BF47F6FF71304602F092
:10424000C7F882460146304602F098F821680546D4
:1042500091F82C0000F00300012841D002283BD047
:1042600000204A8C101A4884ADF800006A1E1044E1
:10427000ADF80400888CADF80200A9F101010844F2
:10428000ADF806006A465146304601F005FD21684A
:10429000BDF8020088845146304601F027FA0644F2
:1042A00030780A281ED00D281CD0BDF800002168E7
:1042B00028444884307818B1761C30780028BBD167
:1042C0002068818C39448184818D21F003018185AE
:1042D00001F01EFBBDE8FC8705EBD5704010C0E780
:1042E0002846BEE7206890F82C1001F00301012950
:1042F0000BD0022909D0018C418431780A29D9D107
:10430000828C02EB09018184D4E7A0F82280F4E7D3
:104310002014002070B514460D46064600F068FBD8
:1043200005480068458484843046FFF76FFFBDE888
:10433000704001F0EDBA0000201400202DE9F0419A
:1043400007460A4815460E460068B0F92C0040F0B2
:10435000020001F075F804462A4631463846FFF758
:10436000D9FF2046BDE8F04101F06AB820140020D2
:1043700047F6FF73AFF300802DE9FC411F469046DE
:104380000D4606004FF000041AD000F031FB65B175
:10439000284607F06FFC040007D00246294668460D
:1043A00002F088F8684607F065FC3B46424629461D
:1043B000304601F0C9FC204607F05CFC01F0A8FA89
:1043C000BDE8FC812DE9F04F87B09B46DDE91098F0
:1043D00092460C46054600F00BFB16480168C86C77
:1043E000096D47190E1900EB0A0501EB0B04ADF836
:1043F0001070ADF81450ADF81260ADF8164004A876
:1044000007F0B2FD88B1DFF830B04FF0000ACDE917
:104410000098CDE902BA2B462246394630460AF0CA
:1044200020FB07F055FD0028F1D101F071FA07B02B
:10443000BDE8F08F201400204D8B00082DE9F04FCF
:1044400087B09B46DDE9109892460C46054600F081
:10445000CFFA16480168C86C096D47190E1900EBB0
:104460000A0501EB0B04ADF81070ADF81450ADF86F
:104470001260ADF8164004A807F076FD88B1DFF8A9
:1044800030B04FF0010ACDE90098CDE902BA2346D9
:104490002A46314638460AF0E4FA07F019FD0028AA
:1044A000F1D101F035FA07B0BDE8F08F20140020FB
:1044B0008D8A00082DE9FE4F9846DDE90D6514460A
:1044C0008A4683460C9F00F093FA0E480068C16C40
:1044D00001EB0409016D002001EB080407F044FD25
:1044E0000AE00097CDE9016523464A465146584601
:1044F0000AF062FB07F0ECFC0028F2D1BDE8FE4FA9
:1045000001F006BA201400202DE9FC4114460D46A6
:10451000064600F06DFA114F3968C86C096D054404
:1045200004440E44ADF80050ADF80440ADF802600C
:10453000ADF80660684607F017FD08E038682246C7
:104540003146406E03682846984707F0C1FC0028B2
:10455000F4D101F0DDF9BDE8FC8100002014002059
:104560002DE9F0411C4615460E46074600F040FA7C
:104570000C480168C86C096D074405440E440C449E
:10458000002007F0F1FC07E023462A463146384672
:10459000FEF714FC07F09CFC0028F5D1BDE8F041C3
:1045A00001F0B6B9201400207CB50C46064600F098
:1045B0001FFA0F4D2868C16C006D0E440444ADF81D
:1045C0000460ADF80060ADF80640ADF80240684602
:1045D00007F0CAFC07E028682146406E4268304672
:1045E000904707F075FC0028F5D101F091F97CBDEA
:1045F000201400202DE9FC411C4616460D460746B6
:1046000000F0F6F91A480168087ECA6C096D174473
:104610000D440C44401E391A1644ADF800103118F0
:10462000ADF80410291A2044ADF80600ADF80210C8
:10463000684607F099FC15E032462946384604F0F2
:1046400025FA32462146384604F020FA621E691CDB
:10465000384604F07BFA621E691C304604F076FA94
:1046600007F036FC0028E7D101F052F9BDE8FC81E3
:1046700020140020B0F90630B0F90420B0F902107F
:10468000B0F90000FFF7B6BF7CB514460D460646EC
:1046900000F0AEF90F480068C16C006D0E4405448F
:1046A0000444ADF80060ADF80460ADF80250ADF818
:1046B0000640684607F058FC06E022462946304688
:1046C00004F044FA07F004FC0028F6D101F020F9C8
:1046D0007CBD00002014002010B5002400E001245F
:1046E00000F004F80028FAD1204610BD0B4810B5A0
:1046F0000068002410B1804700B1012406F0B6FC28
:1047000000B101240648006810B1804700B10124BF
:104710000448006800B18047204610BD28140020DE
:10472000601400205C1400202DE9FC411C46154655
:104730000E46074600F05CF910480068C16C006D39
:104740000F4406440D440444ADF80070ADF8045025
:10475000ADF80260ADF80640684607F005FC07E0DA
:1047600023462A463146384604F01AFA07F0B0FBD1
:104770000028F5D101F0CCF8BDE8FC812014002020
:10478000B0F90630B0F90420B0F90210B0F9000019
:10479000FFF7CABF034951F82000C1688A6A08219F
:1047A000104700005414002010B500F021F904F067
:1047B00027FA04F0EFFA044601F0AAF8204610BDEB
:1047C00010B5044600F014F9054800210068C069DE
:1047D000426820469047044601F09AF8204610BDF2
:1047E0002014002070B50C46054600F001F906487B
:1047F00021460068C069426828469047044601F097
:1048000087F8204670BD000020140020002801D049
:1048100006F080BC704710B500F0EAF804F0F8F933
:1048200004F0B8FA044601F073F8204610BD000009
:1048300010B500F0DDF803480068047C01F068F86A
:10484000204610BD2014002010B500F0D1F8044817
:104850000068C069447E01F05BF8204610BD00008E
:104860002014002010B500F0C3F801F07DFD0446CF
:1048700001F04EF8204610BD70B515460E460446B0
:1048800000F0B6F82A463146204604F007FA040044
:1048900002D000203060286001F03AF8204670BD58
:1048A00010B500F0A5F803480068847E01F030F8E8
:1048B000204610BD2014002070B50C46054600F0BF
:1048C00097F82146284601F0ADFDBDE8704001F0A3
:1048D0001FB810B5044601F097FD01462046BDE81B
:1048E000104001F04BBD01F032B8000010B50024BB
:1048F00000F07EF80B48006890F82C1001F00C01D5
:10490000042904D0082906D00C2907D103E0C06986
:10491000047E641E02E0C069007E440800F0F8FFD7
:10492000204610BD20140020017EC07E11FB00F047
:1049300070470000024951F8200000690068704784
:1049400054140020024951F8200000694068704763
:104950005414002070B50C46054600F049F8044890
:1049600000684584848400F0D3FF002070BD0000FF
:104970002014002070B501F0BFF81B4C2E202070D1
:1049800000F0E7FF19480BF0A3FC04F05BFA0546C2
:1049900004F0AEF9C0B1002604F0BEF9B0B10020B9
:1049A000064307D004F0C1F9064604F0AAF93146DF
:1049B00004F03AFC0021084600F014FD06F09CFDCE
:1049C000FFF728F8206B09E00126E5E70120E7E77B
:1049D000006800B18047206B406820630028F7D151
:1049E0000120A070284670BD0C140020F44F002058
:1049F00070B5184CE06820B100F0A7FF61688842EC
:104A000004D000F0B5FF00F0A0FF6060E068401C3B
:104A1000E06001281CD10BF085FA0546206885422C
:104A200016D0002813DBFFF7DDFB01462068C0EB42
:104A30004012206900EB82029167C5EB4511064ADE
:104A400000EB8100011D1160806FFFF7A5FB256061
:104A500070BD0000001600202014002010B5011EBB
:104A600001DD024600E04A42064B012053F8204097
:104A7000944202D8401C0A28F8DB002900DA401CC6
:104A800010BD0000C03201081CB5040004D10E485E
:104A90000068046E002C16D0FFF7AAFF2046FFF72F
:104AA0001FF9009044696846FFF770F94CB1204641
:104AB000FFF716F9019081688968884701A8FFF718
:104AC00065F900F025FF1CBD2014002001490A46AD
:104AD00000F002B801F0FFFF2DE9F04387B0154662
:104AE0000C465FEA000846D0FFF782FF002000F086
:104AF00031FC814621480068066E4046FFF7F0F819
:104B000000900068806900F0EDFB074640F6FF70FA
:104B1000C44204D10098B0F90440B0F9065000989E
:104B2000611E0289ADF804401144ADF808104189B6
:104B3000681E0844ADF80650ADF80A0006F086F885
:104B40006846FFF723F901A807F00EFA06E02A46A7
:104B50002146404600F0D0FA07F0BAF90028F6D115
:104B6000384600F0BFFB304600F090F9484600F0B0
:104B7000F1FB00F0CDFE07B0BDE8F083201400206B
:104B80002DE9FE4F984691468A46834600270C9EA3
:104B9000FFF72EFF184819490068407C51F8204063
:104BA000E1680968042903D02468002CF8D100E0EA
:104BB0001CB9FFF719FB041E1BD0E0680121C26A73
:104BC00020469047050011D02469A0688047401C0A
:104BD00002D10B4C46F001060096CDE90154434644
:104BE0004A465146584600F0E5F9074600F090FE67
:104BF0003846BDE8FE8F0000201400205414002029
:104C00008454010838B504001CD0FFF7F1FE0E48AB
:104C10000068006EA04201D100F056FB2046FFF76D
:104C20005FF80090406908B100F05BFE00980068F2
:104C3000FFF764FA6846FFF7A9F82046FEF798FFE9
:104C400000F066FE38BD0000201400202DE9FF4F63
:104C500083B09A468B460746FFF7CAFEDFF83891C5
:104C6000D9F80000447C4D4800570128204606DD55
:104C700004F044F80546204604F054F805E004F03A
:104C800026F80546204604F028F804461FB302A97A
:104C900001A8FFF711FEB7F90000002800DA002094
:104CA000B7F902608046002E00DA0026019841190B
:104CB000B7F90400491E0CF061F805460298011985
:104CC000B7F90600491E0CF059F8A5EB0802841B41
:104CD000521C641C03E04FF0000846462A46BAF115
:104CE000000F01D1C4F1000A002A51DD002C4FDD74
:104CF00010980090534631464046FFF741FF5FEA67
:104D0000000A10D000F07CF80746A04206D0D9F87F
:104D10000000806C10B1322107F042FC504600F0D8
:104D2000B5F8002523E059460598884700F0F0FDC6
:104D3000012007B0BDE8F08F611BB94202DA50468E
:104D400000F088F83DB172194146504600F0C6F8AF
:104D50005046FFF799FE5946059888471048016864
:104D600009B1002088475046FFF7B0FE3D44A542F8
:104D7000E2DB5046FFF746FF002000F087F8A7422D
:104D800006D0D9F80000806C10B1332107F008FC80
:104D900000F0BEFD0020CCE7201400207814002095
:104DA0002816002038B505004FF0000411D0FFF799
:104DB0001FFE2846FEF794FF009000680069806897
:104DC000804704F00FFD04466846FEF7DFFF00F061
:104DD0009FFD204638BD38B504000ED0FFF708FE11
:104DE0002046FEF77DFF00F1180400906846FEF7AC
:104DF000CDFF00F08DFD204638BD002038BD0000FD
:104E000038B504460025FFF7F3FD1CB908480068D3
:104E1000046E44B12046FEF763FF0090B0F90A50DB
:104E20006846FEF7B3FF00F073FD284638BD00006A
:104E30002014002070B505460024284608F050F8DC
:104E4000641C18B1BDE8704000F07AB8052CF4DBA2
:104E500070BD000038B50C46050004D10A48006852
:104E6000056E002D0FD0FFF7C3FD2846FEF738FF73
:104E70000090B0F90A10A14200DD44816846FEF7B7
:104E800085FF00F045FD38BD20140020F8B505462B
:104E9000FFF7AEFD104E3068046ECDB10CB100F0DE
:104EA00013FA06F00FF82846FEF71AFF0090316853
:104EB0000D660068FFF724F96846FEF767FF04F007
:104EC00015FA04F07BF900BF00F022FD2046F8BD82
:104ED00000F0FAF9F8E70000201400207CB5154630
:104EE0000E46040004D115480068046E002C24D03E
:104EF000FFF77EFD2046FEF7F3FE2DB20090C58041
:104F000034B2848004F05AF90098406980B1FEF709
:104F1000E7FE009A0190B2F908108180B2F90A20E8
:104F2000C28011B10AB10480458001A8FEF72EFFAE
:104F30006846FEF72BFF00F0EBFC7CBD2014002040
:104F400001490A4600F002B801F0FFFF7FB515469F
:104F50000C4606002DD0FFF74BFD3046FEF7C0FE95
:104F600040F6FF710190CC4203D1B0F90440B0F992
:104F700006500289611E1144ADF80840ADF80C10CE
:104F80004189681E0844ADF80E00ADF80A5001A82A
:104F9000FEF7FCFE02A806F0E7FF06E02A462146DF
:104FA000304600F091F806F093FF0028F6D100F0AB
:104FB000AFFC7FBD2DE9FF4FDFF8E8B083B01C46A2
:104FC000DBF80010DDE9106092464FF000084B7CE2
:104FD00042461299FFF756F8050060D028698068AC
:104FE000804704F0FFFB81460AFB09F1C91DCF0889
:104FF000FEF7B2FEF10705D1C11700EB91708010EA
:1050000000EB4000002C09DC1FB11838B0FBF7F0B2
:1050100000E000206442A04200DC0446F00707D113
:105020000090DDE903012346524600F0DFFB804695
:10503000002C03DC2846FFF761F830E004FB07F0A2
:105040001830F10702D0FEF761FD01E0FEF76EFDBA
:1050500006001CD0FEF744FE019005600399818094
:105060000499C180A0F808A04481C0F81480C0E968
:10507000037901A8FEF78AFE1298AE602861DBF87A
:105080000000407CA861304607B0BDE8F08F28469C
:10509000FFF734F8B8F1000001D0FEF769FD0020F9
:1050A000F2E7000020140020054B30B41B68054CCB
:1050B0005B7C54F823301B6930BC0DF0C3B8000092
:1050C0002014002054140020F8B515460E4607465B
:1050D000FEF706FE009000681621C068426A0020B4
:1050E000904704466846FEF751FE002C03D02A463E
:1050F00031463846A047F8BDF8B516460F460500BC
:1051000012D0FEF7EDFD009044696846FEF73EFEC2
:105110002846FFF747FE0346082800DD2CB132463B
:10512000394628460DF058F9F8BD3246394628462A
:105130000DF0F2FAF8BD0000094A126802B1002031
:10514000074A243252F82030002B07DBA2F1180363
:1051500043F820104FF0FF3142F820107047000054
:105160008814002010B5002821D009B30AB3B1F982
:105170000040B2F900309C4200DA23460380B1F9C6
:105180000240B2F902309C4200DA23464380B1F972
:105190000440B2F904309C4200DD23468380B1F91B
:1051A0000610B2F90620914200DC1146C18010BD04
:1051B00011460A6802604968416010BD00280BD0A2
:1051C00003880B44038083881944818041881144FB
:1051D0004180C1881144C1807047000070B500252E
:1051E000FFF706FC094CD4E9002082420AD0D2E93C
:1051F000005610460AF0ECFE20603146284606F0C4
:105200009BFA012500F084FB284670BDF0150020B4
:105210002DE9FC41154DDDE908742D68B5F90860EC
:10522000864200DD3046B5F90C60964200DA32461F
:10523000824219DBB5F90A608E4200DD3146B5F9CC
:105240000E509D4200DA2B468B420DDB00E02C46CF
:10525000E5682D6825B1042D02D02568002DF6D112
:10526000CDE9007403F094FEBDE8FC812014002019
:10527000B0F90220B1F906309A4213DCB1F90220EC
:10528000B0F906309A420DDCB0F90020B1F90430D3
:105290009A4207DCB1F90010B0F90400814201DC48
:1052A00001207047002070470146024874220068C0
:1052B000FBF751B820140020024974220968FBF75B
:1052C0004AB800002014002010B5FFF791FB03F04E
:1052D0002BFF04F00BF805F0B9FCBDE8104000F01E
:1052E00017BB000070B50B4D04462868467CFFF7DD
:1052F0007FFB022C09D22046FEF776FF28B12868F2
:105300004474FFF7E1FF0448046000F001FB3046FD
:1053100070BD0000201400207015002010B5044658
:10532000FFF766FB204603F01FFFBDE8104000F0CA
:10533000EFBA10B50446FFF75BFB204603F04CFFC5
:10534000BDE8104000F0E4BA0149886070470000F1
:105350000C14002010B50446FFF74AFB204603F06A
:1053600069FF044600F0D4FA204610BD70B504462B
:10537000FFF73EFB04480068C56904B1C46100F052
:10538000C7FA284670BD0000201400200249CA69EF
:10539000C861104670470000D813002001494860DA
:1053A000704700000C14002002490A68086010468B
:1053B00070470000D813002002494A684860104630
:1053C00070470000D813002070B50546FFF710FBAA
:1053D00003480068847E857600F09AFA204670BD06
:1053E0002014002070B50C460546FFF701FB094864
:1053F000224605800848048008480068417C084827
:1054000050F82100C1680B6A29469847BDE87040F2
:1054100000F07EBA801400208214002020140020A6
:105420005414002070B50546FFF7E2FA03480068FF
:10543000047E057600F06CFA204670BD2014002032
:1054400070B50446FFF7D4FA04480068B0F92C5050
:10545000848500F05DFA284670BD0000201400200D
:1054600070B50446FFF7C4FA04480068B0F92A5042
:10547000448500F04DFA284670BD0000201400203D
:1054800002480068002800D0004770471C16002022
:1054900002498A6802B98860FFF7F2BFF015002060
:1054A0002DE9FC41984616460D460746FFF7A0FA3F
:1054B0001C20FEF73BFB04002DD01C491A48086055
:1054C0002046FEF70DFC009015B9FFF70CFA0546D3
:1054D00000980760C0E90465A0F80C806846FEF7F4
:1054E00055FC20460BF09EFB114DA86840B90120E9
:1054F000A86005F10C010F480860084601F0E2F8C9
:105500002046FEF7EDFB0190296849B181602C60CF
:1055100001A8FEF73BFC00F0FBF92046BDE8FC814A
:1055200000212C608160F3E76155000828140020F9
:10553000FC1600203110010810B504000ED0FFF752
:1055400057FA20460CF0E4FA20460CF04BFE2046B9
:10555000FEF70EFBBDE8104000F0DAB910BD000008
:105560002DE9F04188B00025FFF742FA184C676832
:1055700025E000BFFFF7B7F906466068FEF7B0FB0D
:1055800001904169891B002915DC6168029604912C
:105590000169039146686660D0F8008001A8FEF7B3
:1055A000F5FB02A84146884766B160680125B8420C
:1055B00005D1002506E001A8FEF7E8FB02E06068DF
:1055C0000028D7D100F0A4F908B02846BDE8F08142
:1055D000FC16002038B50C46050011D0FFF708FA7C
:1055E0002846FEF77DFB00908089204201D00124EF
:1055F00000E000246846FEF7C9FB00F089F900E0EE
:105600000124204638BD38B5040017D0FFF7F0F963
:105610002046FEF765FB0090FFF765F9014600980C
:105620008269114441616846FEF7B0FB20460CF0E8
:10563000D9FD20460BF0F6FA00F06AF938BD38B50E
:105640000C4605000BD0FFF7D3F92846FEF748FBC0
:10565000009084616846FEF799FB00F059F938BD67
:1056600038B50546002028600648046844B1204645
:10567000FEF736FB0090006928606846FEF786FB5F
:10568000204638BDFC16002038B504004FF000005D
:105690000D46086011D02046FEF722FB009084687A
:1056A00044B16846FEF772FB2046FEF719FB0090F6
:1056B000006928606846FEF769FB204638BD000097
:1056C0002DE9F041084E0446056830680168284617
:1056D0008847074630684168284688472844206044
:1056E0003846BDE8F0810000241400202DE9F04187
:1056F0000C4606460025064F05E0386841683046EE
:10570000884706440544641EF7D22846BDE8F08168
:10571000241400202DE9F0411E46069C17468846B9
:1057200005463A46A8687F1C3346D0F804C0414677
:105730002846E047641EF4D1BDE8F08170B5B0F9A9
:105740000040091BB0F904408C422CDD00F1140428
:10575000B0F902500069521B02FB0040CA1800EB6E
:10576000E104521ED010B0EBE10501F007034FF049
:10577000FF0102F0070221FA03F0C2F1070201FA69
:1057800002F1CEB221780FD001436D1E04F8011B47
:10579000002D05DDFF2229462046FAF7FDFD2C44A9
:1057A00020783043207070BD30400143217070BDBF
:1057B00010B5B0F90030B0F90240C91A00F1140375
:1057C0000069121B02FB003000EBE10001F007034F
:1057D00002788021D9400A43027010BDB0F906104A
:1057E000026951431430FAF7DEBD00002DE9F84399
:1057F000804602F10F000011470003FB07F01C4632
:10580000154689461430FEF791F9060018D0FFF7C7
:10581000EFF83046FEF764FA0090A0F80080A0F898
:1058200002908580C48007498160012181810761E0
:105830006846FEF7ABFA00F06BF83046BDE8F88337
:105840000020FBE7105D010870B5B0F90660B0F903
:1058500004400B6800F1140596421BDD0069A34269
:1058600002FB005000EBE30214DA641EE010A0EB30
:10587000E30512F8010B03F00704A040C4B206E0F0
:1058800045B1083312F8014B23F007036D1E002CBD
:10589000F6D004E0002070BD6006040E5B1C2006FC
:1058A000FAD5FF2C07D0184602E06406240E401CEF
:1058B0006606FAD400E0D81DC443640705D006E0AC
:1058C00012F8014BFF2C09D108306D1EF8D5C01A13
:1058D000401C0B6070BD6206140E401C2206FAD4F8
:1058E000F5E738B50546FFF783F82846FEF7F8F9DF
:1058F00000908189491E0CB284816846FEF746FA01
:1059000014B92846FEF734F900F002F838BD00005B
:105910000348C168491EC16001D100F031B8704729
:105920000016002010B505484FF40001FEF718F9E5
:10593000BDE810400248FFF707BD0000000040C06E
:105940003C3A01080120FAF7D9BEFBF7F9BCFAF797
:1059500013BF704710B50020FAF7E2FF034C206038
:105960000020FAF7DDFE606010BD00008C130020FF
:1059700002484FF0FF310068FAF7C0BF8C130020D7
:1059800001480068FAF7DEBF8C1300200EB508B19D
:1059900002AA00E00022002301A9684600F096FC5C
:1059A0000EBD0000074910B50C7818B10120087031
:1059B000801E03E0002008706FF07F4002F022FF9D
:1059C000204610BD0D14002010B5082A0EDC034639
:1059D000012A18D0022A56D0042A76D010F8042BB7
:1059E00003F8012B491EF9D1012010BD102A08DC53
:1059F0004FEA000230F8043B22F8023B491EF9D17D
:105A0000F2E7002010BD10F8042BD207120E491E39
:105A100034D010F8044B491E04F0010442EA841209
:105A20002CD010F8044B491E04F0010442EA441241
:105A300024D010F8044B491E04F0010442EA041279
:105A40001CD010F8044B491E04F0010442EAC402C1
:105A500014D010F8044B491E04F0010442EA8402F9
:105A60000CD010F8044B491E04F0010442EA440231
:105A700004D010F8044B04F00104224303F8012B76
:105A80000029C0D1B0E710F8042B9207120E491E6E
:105A900015D010F8044B491E04F0030442EA041226
:105AA0000DD010F8044B491E04F0030442EA8402AE
:105AB00005D010F8044B04F003042243491E03F8F8
:105AC000012B0029DFD18FE7FFE710F8042B120725
:105AD000120E491E05D010F8044B04F00F042243A7
:105AE000491E03F8012B0029EFD17DE738B50024CA
:105AF000009400F01DF838BD0B4810B5416B00292B
:105B000010D101214163FFF70DFFFDF7B5FF03F051
:105B1000FFFB0549054838310860BDE810400846DC
:105B200000F0D0BD10BD00000C140020450F01088E
:105B30002DE9F0410D460699044601B901461F685A
:105B4000082A09DC0E46012A1AD0022A5BD0042A50
:105B50007DD0082A13D18DE0102A07DCD3F810C0BD
:105B60000E46BCF1000F04D0022389E00020BDE8FE
:105B7000F08101CCB84726F8020B6D1EF9D189E0FF
:105B800001CCB847C0074FEA10686D1E36D001CC73
:105B9000B84748EA801000F0FF086D1E2ED001CCF7
:105BA000B84748EA401000F0FF086D1E26D001CC2F
:105BB000B84748EA001000F0FF086D1E1ED001CC67
:105BC000B84748EAC00000F0FF086D1E16D001CCAF
:105BD000B84748EA800000F0FF086D1E0ED001CCE7
:105BE000B84748EA400000F0FF086D1E06D001CC1F
:105BF000B84740EA080000F0FF086D1E06F8018B68
:105C0000002DBDD146E001CCB84780074FEA1068AF
:105C10006D1E16D001CCB84748EA001000F0FF080E
:105C20006D1E0ED001CCB84748EA800000F0FF0896
:105C30006D1E06D001CCB84740EA080000F0FF080E
:105C40006D1E06F8018B002DDDD123E0FFE701CCAE
:105C5000B84700074FEA10686D1E06D001CCB84760
:105C600040EA080000F0FF086D1E06F8018B002DC9
:105C7000EDD10FE0D3F810C0BCF1000F04D0012328
:105C80002A462046E04705E001CCB84706F8010B5C
:105C90006D1EF9D101206AE77CB5064628480D46FD
:105CA000006868B1002006F05FF906E06A46294600
:105CB000304607F021FB06F00BF90028F6D17CBD39
:105CC000106800901F4C506801902268BDF80000D9
:105CD00032F84C1F0844ADF80000BDF8020091886E
:105CE0000844ADF80200BDF8040011880844ADF87E
:105CF0000400BDF8060091880844ADF80600684627
:105D000006F032F90EE000BF2068BDF800106A46C8
:105D10004184BDF8021081842946304607F0ECFA30
:105D200006F0D6F80028EFD1206830F8221F428D07
:105D3000891A01804188C28D891A41807CBD00008A
:105D40007C140020201400202DE9FF4F85B0002096
:105D50009B4691460D4602900390FEF775FD4FF06D
:105D6000000ADDF814800646544625B128680090E4
:105D70006868019002E06846FEF748FD19F00C0FD4
:105D800002D05D46002713E0BDF902402DE0294610
:105D90007F1C059800F01CFB01466D1A0598FFF763
:105DA000A5FC05990844059005A800F055FB08B925
:105DB000002DECD109F00C00042804D0082802D0F2
:105DC0000C2812D105E0BDF9060007FB1604641C7F
:105DD0000BE0BDF90600BDF90210401A07FB1600E2
:105DE000401C00EBD07001EB60045D46DFF838B179
:105DF0004E4FCDF8148079E02946059800F0E8FA76
:105E00002D1A01460490059800F0B8FA19F0030124
:105E10000ED0012965D002290DD1BDF90420BDF9AC
:105E20000010521A121A02EBD27201EB620101E069
:105E3000BDF900108A463A68401E5044A2F822A0DC
:105E40009484ADF80C00A019401EADF80E00DDE9F9
:105E50000410ADF808A0ADF80A4002AAFFF71CFF35
:105E60009BF8000070B3386890F82A00800729D4A6
:105E7000059941450CD1BDF90A30BDF902108B429C
:105E800006DDBDF90420BDF900005B1EFEF7BCF87D
:105E9000BDF90820BDF90000824206DDBDF90E30D3
:105EA000BDF90A10521EFEF7AFF8BDF90C00BDF99E
:105EB0000420904206DABDF90E30BDF90A10401CEC
:105EC000FEF7A2F8DDE90410FFF710FC059908447D
:105ED0000590FEF7B9FC044405A800F0BDFA28B10E
:105EE00006E0BDF90410091A491CA3E7002D83D16F
:105EF0009BF80000002814D0386890F82A0080072A
:105F00000FD4059941450CD0BDF90E10BDF90630EE
:105F1000994206DABDF90420BDF90000491CFEF7DC
:105F200073F809B0BDE8F08F84140020201400201D
:105F300049B1002802DAA0EB610001E000EB61004A
:105F400090FBF1F070470020704700002DE9FF4FF3
:105F50008DB00020DDF86C90164600901D4604467A
:105F60000246C9F8000008AB03A902A800F0AEF988
:105F700018B1002011B0BDE8F08F0898854200DD0F
:105F80000546604F0B9560493868407C51F82010F9
:105F9000049109690691FEF7FDFB05903868407C85
:105FA000FEF7D0FC59498346884201D0012000E029
:105FB00000200A9001CE1A9988478246000E079069
:105FC00077D0009870BB0D9800EB04084D4800682E
:105FD000B0F90800404503DDA0EB0807804600E06B
:105FE00000270299049801EB840101EB8701CDE9B8
:105FF00000100B990D98421809920E9B40461946C5
:10600000521EFFF705F901200090059818280ADABA
:106010000298DDE9052300EB840000EB8700E91B13
:1060200000F0B2F812E00A9880B1029800EB840008
:1060300000EB87070998A0EB08085946386888479D
:1060400001C7A8F101005FEA0008F6D1304BD8691A
:1060500080B3DDE9020700EB840007EB8402CDE9A1
:1060600002022B4C361F2B46E46930460299A047AA
:10607000FF203168B0EB116F02D10299096804E08A
:10608000029A1268B0EB126F01D1039A1160029963
:1060900006F10406091D02910399091D03916D1E65
:1060A000E7D10397D9F8000040F00100C9F80000DB
:1060B00021E022E0FFE70798FF2812D0C0F1FF029D
:1060C00002981B6850F824102AF07F4098470399E3
:1060D00041F82400D9F8000040F00101C9F800108F
:1060E00005E00298039950F8240041F82400641C4C
:1060F0006D1E7FF45FAF03983CE7039941F824A03D
:10610000E8E700002014002054140020158E000839
:10611000D81300202DE9F04F85B09B46DDE90F87AD
:1061200092460C460546DDF83890FEF761FC1548AE
:106130000068C16C4E190D19016DABF1010001EB46
:106140000A04ADF810502044ADF80C60ADF8120010
:10615000ADF80E4003A805F007FF0BE0CDF8009066
:10616000CDE901875B4622462946304608F058FFB4
:1061700005F0AEFE0028F1D1FFF7CAFB05B0BDE87F
:10618000F08F0000201400202DE9F05F0C1E16DDBA
:106190005E68014600EB8405082A12DC611E012AB4
:1061A00026D0022A47D0042A6AD0082A07D1071924
:1061B00017F8010DB04745F8040D641EF8D1BDE88D
:1061C000F09F102AFBDC5F693FB12246BC46BDE868
:1061D000F04F02235DF804EB604701EB440700BF7A
:1061E00037F8020DB04745F8040D641EF8D1E6E714
:1061F00000EBE10001F0070710F801A981468020BB
:1062000020FA07F8B5F104050AEA0800C7F107010A
:10621000C840B04745F804093FB14FEA48604FEA2B
:1062200010687F1E641EEFD1C9E719F801A907277E
:106230004FF00108F6E700EBA10001F0030710F8AA
:1062400001A981467900C02020FA01F84FF0060B21
:10625000B5F104050AEA0800ABEB4701C840B047B6
:1062600045F804093FB14FEA88604FEA10687F1E85
:10627000641EEFD1A3E7032719F801A9B846F7E791
:1062800000EB6100012710F801A9A7438146B9007E
:10629000F02020FA01F84FF0040B2D1F0AEA080045
:1062A000ABEB8701C840B04745F804093FB14FEA5E
:1062B00008704FEA10687F1E641EEFD17FE719F85F
:1062C00001A901274FF00F08F6E700002DE9F0477C
:1062D000224C06461F46A06990468946002540B9D3
:1062E0000120A06104F128011D480860084600F063
:1062F000E9F9606930B91B480068606110B902F0C3
:10630000E9FC606107B138604EB1A06830B96069DE
:106310008000FDF75FFCA06000B901253060B9F195
:10632000000F0AD0E06830B960698000FDF752FCC8
:10633000E06000B90125C9F80000B8F1000F0AD0EB
:10634000206930B960698000FDF744FC206100B924
:106350000125C8F800002846BDE8F087D8130020C2
:106360001D0F01087014002003480068C069017EF9
:10637000C07E11FB00F070472014002073B5124A54
:1063800001A900981268904700240090C8B10F49F5
:1063900000250968C969496959B10A684AB1019972
:1063A00090477CBD6846FFF78BF90546FEF708FA73
:1063B00004440198401E0190F4D5284600F040F8AE
:1063C000044420467CBD0000EC1500202014002071
:1063D00073B50D460098002490B10A490968C9694F
:1063E000496959B14A684AB1294690477CBD684617
:1063F000FFF766F920B10A2802D0641CAC42F6DB34
:1064000020467CBD2014002031B50024009808B936
:1064100005E0641C6846FFF753F90028F9D12046CF
:1064200038BD0000044AB2F9002002600348B0F908
:1064300000000860704700008014002082140020D3
:1064400038B5002469460094FEF7CCF900998142E2
:1064500000DD0C1A204638BD38B5044600680090AF
:106460006846FFF72DF910B10A2802D003E0012099
:1064700038BD00982060002038BDB0F90030B1F977
:106480000020934200DA0280B0F90230B1F9022014
:10649000934200DA4280B0F90430B1F9042093420B
:1064A00000DD8280B0F90620B1F906108A4200DDD5
:1064B000C180704770B5B1F90040B2F900309C421C
:1064C00000DD23460380B1F90250B2F90240A54233
:1064D00000DD2C464480B1F90460B2F90450AE42AC
:1064E00000DA35468580B1F90610B2F906209142EE
:1064F00000DB1146C1809D4201DBA14201DA002090
:1065000070BD012070BD0000014602480068407C5B
:1065100000F002B8201400202DE9F8430126894636
:10652000044602285DDA304F7A6802B190472E4D5A
:106530005FEA090005F1100532D0012803D0B9F156
:10654000020F4ED118E055F8240088B92046FDF717
:106550004BFE009018B3C0680D21426A6846904710
:1065600002003ED049460098904755F82400002686
:10657000401C45F8240034E02046FDF735FE00902D
:1065800068B1C0680D21426A68469047040028D06F
:10659000386800B1804749460098A047002620E0AF
:1065A00055F82400A846012812D12046FDF71CFE0C
:1065B000009068B1C0680D21426A684690470500A6
:1065C00006D0386800B1804749460098A8470026A1
:1065D00058F8241009B1012200E00022891A48F875
:1065E00024103046BDE8F883CC15002030B581F08A
:1065F0007F43FF2480F07F4094EA116101D120F0B5
:106600007F43010E11FB02F1B1FBF4F100F0FF1525
:10661000C1F1FF0203F0FF14544301FB05444FF0A6
:10662000FF15240A05EA1323C0F30720534340F063
:10663000807001FB003104F0FF1001F0FF210843DE
:1066400080F07F4030BD00002DE9F05F0646DDF8A8
:10665000389015460C4600200D99804688421ED27F
:10666000DFF840B00C9F4FF0FF0A02CE08CCAAEB37
:10667000116202FB09F2B2FBFAF0C2B221F07F40D4
:106680001946DBF80030984720F07F4001C57F1E97
:10669000EBD10A9804EB800408F10100DCE7BDE8C7
:1066A000F09F0000D81300200B88134403808B88D0
:1066B0009B1A83804B8813444380C988891AC18000
:1066C000704700000249CA6A4260C8627047000011
:1066D0000C1400202DE9F84307680646884600257B
:1066E000384600F097F848B3404600F0A3F8441C41
:1066F0003846FDF7E7FA84420DD1FCB13846FDF784
:10670000EFFA104B009022461B68414698476846B6
:10671000FDF73CFB11E02046FDF7F8F904000DD031
:10672000FDF7DEFA41460090F9F748FE6846FDF7AE
:106730002DFB3046FDF740FA346001252846BDE8C0
:10674000F8830000E815002030B50346CCB202E023
:1067500003F8014B521E0AB19907F9D1910818D0DC
:1067600004EB044502F0030205EB052506E020C317
:10677000091F20C343F8085B43F8045C0429F6DAD8
:1067800001E020C3491E0029FBD102E003F8014BC0
:10679000521E002AFAD130BD10B5830702D520F869
:1067A000021B521E530811D001EB0144042B09DBDC
:1067B00010C01B1F10C0042B40F8084B40F8044CBD
:1067C000F6DA01E010C05B1E002BFBD1D20700D02F
:1067D000018010BD024600204FF0804143189342D3
:1067E00001D8D21A581840088908F7D1704700001C
:1067F00000B907A021B906A102E03AB1401C491C2A
:1068000002780B789A42F8D0012070470020704738
:106810000000000038B50D46012448B1FDF760FACC
:1068200029460090FFF7E4FF04466846FDF7AEFAFC
:10683000204638BD4FF0FF3128B100BF10F8012BC2
:10684000491C002AFAD10846704700F5806000F024
:1068500001B8000010B50023C0F30B00B0F5006FC5
:1068600002DD0123A0F50060B0F5806F01DDC0F509
:10687000006081110C4C00F03F00C0F1400234F880
:1068800011005043402A08D0102906DA04EB4101D8
:10689000C2F14002498801FB020020308009002B30
:1068A00000D0404210BD0000184A0108F8B500248D
:1068B000009490F83C20012A19D0012280F83C2055
:1068C0000A680726514D092A1DD90368DF680A3A6C
:1068D00002EB42029640B743DF600A68AA4208D141
:1068E0000268D3680E7A43EA0663D3601BE0022095
:1068F000F8BD0A3A8B6802EB420293400268D66800
:106900003343D3600FE003681F6902EB42029640F5
:10691000B7431F610A788B6802EB4202934002681A
:106920001669334313614A681F26072A13D2036886
:106930005F6B521E02EB82029640B7435F630A8888
:1069400093B20A79521E02EB820293400268566BA0
:106950003343536328E00D2A13D203681F6BD21F01
:1069600002EB82029640B7431F630A8893B20A790A
:10697000D21F02EB820293400268166B334313630B
:1069800012E00368DF6A0D3A02EB82029640B743D9
:10699000DF620A8893B20A790D3A02EB82029340D1
:1069A0000268D66A3343D362194B02689A4208D10F
:1069B0000A68122A05D1D3F8042342F48002C3F8EE
:1069C000042302689A421DD10A68AA4201D0112A02
:1069D00018D1D3F8042342F40002C3F80423096851
:1069E000A9420FD10B490C4A0968B1FBF2F101EB46
:1069F00081014900009102E00099491E009100992F
:106A00000029F9D180F83C400020F8BD12000010A8
:106A1000002001408813002040420F000068C06C35
:106A2000704770B504460026002C03D0206C00256A
:106A300010B107E0012070BD656484F83C50204629
:106A400000F01AF8206CC00610D4206C20F4885096
:106A500040F0020020642046FBF7C2F96564206C18
:106A600020F0020040F00100206400E0012684F8DC
:106A70003C50304670BD000000B587B000680C493E
:106A8000884213D10B48016841F4806101600068BD
:106A900000F4806001904FF4806002900320039026
:106AA00000200490044802A900F094FB07B000BD48
:106AB00000220140443802400014024018B5002270
:106AC000009290F83C10012907D0012180F83C1079
:106AD00001688B68DB0702D014E0022018BD8B68C8
:106AE00043F001038B602749274B0968B1FBF3F1A1
:106AF00001EB4101009102E00099491E00910099CB
:106B00000029F9D101688B68DB0738D0036C40F2AB
:106B10000164A34343F4807303644B685B0505D5AC
:106B2000036C23F4005343F480530364036CDB04CD
:106B300004D5436C23F00603436400E0426480F80C
:106B40003C206FF022020A601049D1F80423D206DB
:106B500007D00068884212D1816811F0405F0AD0E6
:106B60000DE00068816811F0405F08D1816841F054
:106B70008041816003E0816841F0804181600020B4
:106B800018BD00008813002040420F000020014083
:106B900070B50446002C2AD094F83500022828D07D
:106BA0002068016821F0010101602068002505606E
:106BB00020684560206885602068C56020680561A0
:106BC0002120216848612046FBF74CFB34343F21EB
:106BD00094F8282091408160A560E5602561656199
:106BE000A561E561256265702570002070BD0120FA
:106BF00070BD022070BD00002DE9F041044600F098
:106C0000E7FB05465CB1002684F83460022084F876
:106C100035002068016821F0010101600DE00120CC
:106C2000BDE8F08100F0D4FB401B052805D92020E9
:106C30006065032084F83500F2E720680068C0072B
:106C4000F0D121680A6820480240D4E901031843C2
:106C5000D4E903352B43184363691843A3691843E8
:106C6000E3691843236A18431043626A042A03D174
:106C7000D4E90B231A43104308602068406920F0D0
:106C80000700656A29460543012704290DD1A06A3A
:106C90000543E06A48B12046FBF7FAFA28B14020E4
:106CA000606584F835700120BAE7206845612046A8
:106CB000FBF7D8FA94F85C203F219140816066652B
:106CC00084F835700020ABE73F8010E030B5027CDF
:106CD000012A6BD0012202744A680268536B23F0C8
:106CE000010353630268D2F8003423F00103C2F8B1
:106CF00000340268936B23F0030393630268936B81
:106D0000CC68234393630268D36B6FF30D03D363A3
:106D10000268D36B0C692343D3630268136C6FF36F
:106D20000C0313640268136C4C69234313640268F8
:106D3000536C6FF30C0353640268536C8C692343E8
:106D400053640268D36823F00303D3600268D368F6
:106D50000C682343D3600268536923F0070353612F
:106D6000026853694C6A2343D1E907542C432343F7
:106D700053610268136923F00F03136102681369FA
:106D80004C68234313610268D2F8003423F00E03E9
:106D9000C2F800340268D2F800344C6843EA440375
:106DA000C2F800344A68032A02D00BE0022030BD4A
:106DB0000268136923F480731361026813698C6895
:106DC000234313610268936C6FF30B0393640268AF
:106DD000936C8C6A234393640268D36C6FF30B0348
:106DE000D3640268D36CCC6A2343D3640268136D06
:106DF0006FF30E0313650268136D0C6B2343136569
:106E00000268536D6FF3090353650268536D4C6B51
:106E1000234353650268936D6FF30903936502681A
:106E2000936D8C6B234393650268D36D6FF30903F5
:106E3000D3650268D36DCC6B2343D3650268136EB0
:106E40006FF30D0313660268136E0C6C2343136615
:106E50000268936B23F4004393630268936B4C6C5A
:106E6000234393630268936923F47F039361026869
:106E70009369B1F8484043EA044393610268936917
:106E800023F0FF03936102689369CC6C2343936101
:106E90000268936B23F4005393630268936B0C6D49
:106EA000234393630268936B23F4805393630268D4
:106EB000936B4C6D234393630268936B23F40063DD
:106EC00093630268936B8C6D234393630268936BA7
:106ED00023F4806393630268936BCC6D23439363C5
:106EE0000268936B23F4007393630268936B0C6ED8
:106EF000234393630268936B23F480739363026864
:106F0000936B4C6E234393630268936B23F480432B
:106F100093630268936B896E0B4393630021017442
:106F2000002030BD2DE9F04104460D46002C02D072
:106F3000607C18B105E00120BDE8F081204600F03A
:106F4000F0F8032060742068D0F8301441F08071AC
:106F5000C0F8301400F03CFA06464FF47A7706E0A9
:106F600000F036FA801BB84201D90320E4E720681C
:106F7000D0F80C04C004F3D52068D0F830143D4A92
:106F80001140C0F830142068D0F830142A682B89DA
:106F900041EA82016A68D20242EA03421143C0F820
:106FA00030142068D0F8301441F00101C0F83014DA
:106FB00000F00EFA064606E000F00AFA801BB8421E
:106FC00001D90320B8E72068D0F80C04C005F3D538
:106FD000206850F8A01F41F006010160206850F8B9
:106FE000941F21F003010160206850F8941F62682B
:106FF000114341F001010160206850F8A41F21F005
:1070000003010160206850F8A41FE2681143016089
:107010002068816821F0FF01816020688168A26892
:1070200011438160686800B90120134946F2A81233
:107030004843297A884029685143B0FBF1F1206820
:10704000D0F8182422F03F02C0F818242068D0F8A5
:1070500018240A43C0F8182421680020C1F8C4008D
:107060002168C1F8C800A06160610120607400203F
:1070700062E700000386FCFF00093D002DE9FF4F99
:1070800081B005461F46DDE90E860024287C0128D4
:1070900008D00120287400F09BF98246A1464FF4E5
:1070A0007A7B0DE0022005B0BDE8F08F00F090F98A
:1070B000A0EB0A00584503D985F810900320F2E7A9
:1070C0002868406FC007F1D00EE0ECB13019315D97
:1070D000427841EA02218278C078120442EA0060D4
:1070E000014328680167241DBC42EED37F1CDDE903
:1070F0000212C7F3072000902868FBB2FBF704F9DF
:1071000085F810900020CEE73078717848EA0020AA
:1071100040EA0140B17840EA016029680867032429
:10712000E2E770472DE9F84F0446894692469B46B0
:10713000DDF82880207C012808D00120207400F090
:1071400047F9054600264FF47A770AE00220BDE8A9
:10715000F88F00F03DF9401BB84202D92674032095
:10716000F5E72068406FC007F3D0CDF800805B469C
:10717000206852464946FBF7C7F826740020E6E728
:10718000017C012911D00121017401684A6842F093
:1071900001024A600168D1F8042442F00802C1F8F3
:1071A0000424002101740020704702207047000071
:1071B00070B5044600F00CF90546601C02D0044886
:1071C0000078044400F004F9401BA042FAD370BDDB
:1071D0007C1300202DE9F84F0022DFF8A491DFF89E
:1071E000A0814FF0010E09F108094FF00F0C09F1D1
:1071F000040A0EFA02F60B683340B34271D14C68B0
:10720000022C01D0122C11D1D40800EB84073D6A66
:107210005407E40E0CFA04FB25EA0B05D1F810B074
:107220000BFA04FB4BEA050BC7F820B007685400C3
:107230000325A540AF4391F804B00BF0030B0BFA04
:1072400004FB4BEA070BC0F800B04F68012F05D0D4
:10725000022F03D0112F01D0122F11D18768AF4315
:10726000D1F80CB00BFA04FB4BEA070BC0F808B0DE
:107270004768B7430E79C6F3001696403E43466012
:10728000C668AE438D68A5403543C5604C68E400D0
:107290006FD53C4C256845F480452560246804F48E
:1072A00080440094384C22F003052544D5F8087832
:1072B0009407260F0CFA06F4A743344CA04201D1E0
:1072C00000242EE0324CA04201D1012429E0314CAF
:1072D000A04201D1022424E02F4CA04202D1032479
:1072E0001FE046E02D4CA04201D1042419E02C4CB3
:1072F000A04201D1052414E02A4CA04201D1062469
:107300000FE0294CA04201D107240AE0274CA042FB
:1073100001D1082405E0264CA04201D1092400E057
:107320000A24B4403C43C5F80848D8F800409C43C0
:107330004D68ED0300D51C43C8F80040104D2D1DCD
:107340002C689C434E68B60300D51C432C60D9F8CA
:1073500000409C434D68ED0200D51C43C9F8004035
:10736000DAF800409C434D68AD0200D51C43CAF8D2
:107370000040521C102AFFF43CAFBDE8F88F00001B
:10738000003C01404438024000300140000002400F
:107390000004024000080240000C024000100240BD
:1073A0000014024000180240001C0240002002406D
:1073B000002402400069084201D0012070470020EB
:1073C0007047002A01D081617047090481617047CC
:1073D00010B5F9F7B7F9022817D00E480068800BEE
:1073E00070B100BF00BF00BF00BF00BF00BF00BF43
:1073F00000BF00BF00BF00BF00BF401E0028F0D18B
:1074000005490868401C086010BDBDE81040F9F748
:10741000B3B90000881300205013002010B50948AC
:10742000016841F400710160016841F480710160FC
:10743000032000F0A5FB0F2000F006F800F030FB61
:10744000002010BD003C024070B504460D4D4FF4C5
:107450007A712878B1FBF0F00B490968B1FBF0F0C4
:1074600001F094F908B1012070BD102C07D2002260
:107470002146501E00F064FB6C60002070BD0120AE
:1074800070BD00007C13002088130020F0B500249C
:1074900090F8A050012D06D0012780F8A070022599
:1074A00080F8A1501EE00220F0BD03EB830505EB40
:1074B000C30500EB8505AD6C062D1BD00E68F5B23B
:1074C00006F47F4C45EA046545EA0C0506F47F06A0
:1074D0003543091D06684FF0C40C0CEBC31C46F87D
:1074E0000C50641C9442E0D3A0304770002101701E
:1074F0000020F0BD0E6804EB041CF5B245EA0C65F3
:1075000006F47F4C45EA0C0506F47F063543E0E7B8
:1075100030B590F8A030012B18D0012480F8A0409D
:10752000022380F8A1300368902505EBC2129D5814
:1075300005F07F459D500368995001684C6280F8C2
:10754000A140002180F8A010002030BD022030BDF5
:107550002DE9F04104460F46154694F8A000012895
:107560001ED0012684F8A060022084F8A10005EB5B
:107570008500394600EBC500342204EB800038302A
:10758000F8F7E9FE2A463946204602F09FF92068BE
:10759000466284F8A160002084F8A000BDE8F08174
:1075A0000220FBE710B590F8A020012A15D0012396
:1075B00000F8A03F02224270842450F8A02C04EB73
:1075C000C111545824F00204545050F8A01C4B62CE
:1075D000437000210170002010BD022010BD10B5C5
:1075E00090F8A020012A15D0012300F8A03F022224
:1075F0004270842450F8A02C04EBC111545844F07C
:107600001004545050F8A01C4B62437000210170CC
:10761000002010BD022010BD10B590F8A020012A56
:1076200015D0012300F8A03F02224270842450F8B4
:10763000A02C04EBC111545844F00204545050F8EB
:10764000A01C4B62437000210170002010BD02207D
:1076500010BD704770B504462068816B4FF004067A
:107660004FF00005490714D5816B490711D5416BCF
:1076700021F004014163843454F8840CC663206A09
:1076800040F00100206266772577843C2046FFF7B2
:10769000E0FF2068816B890715D5816B890712D5BA
:1076A000416B21F0020141630220843454F8841CB0
:1076B000C863206A40F00200206266772577843C28
:1076C0002046FFF7C6FF2068816B4FF00106C9070F
:1076D0000FD0816BC9070CD0416B21F001014163D0
:1076E0002068C66384F8A16084F8A050204600F0AA
:1076F00097F82068816B090710D5816B09070DD5B4
:10770000416B21F00801416321680820C86384F8B7
:10771000A16084F8A050204600F0DAF870BD0000A7
:1077200070B50446002C04D094F8A100002510B1D7
:1077300006E0012070BD84F8A050204600F0AAF8B1
:10774000022084F8A1002068816921F070418161E4
:10775000D4E901100143D4E9030210430143206836
:10776000826911438161206882682C490A408260E5
:10777000A08A020420688368A669334313438360A8
:107780002068C2680A40C260A08B02042068C368F7
:10779000266A33431343C360206802690A400261CA
:1077A000A08C020420680369A66A33431343036173
:1077B000206842690A404261A08D01042068426944
:1077C000236B1A430A43426194F83500020294F88D
:1077D000360001042068C36A03F07F43C362206857
:1077E000C36A114394F8346033430B43C362206887
:1077F000416B41F0040141632068416B41F002019B
:1078000041632068816941F001018161C4F8A4509D
:10781000012084F8A100002070BD000000F800F0F5
:1078200070B506460024194D55F82400002824DBC5
:107830001649164A0C39083A51F8241052F82420F7
:107840005143124A121F52F824205043104A52F852
:10785000242001FB00212246304600F03AF830682F
:10786000416A41F00101416255F824102046FDF7BC
:1078700063FC4FF0FF3045F82400641C012CD3DB7F
:107880003046BDE87040002100F006B8B813002073
:10789000303201087047000010B590F8A020012A8E
:1078A00011D0012300F8A03F0222427050F8A02C12
:1078B000546B44F001045463044A11604370002186
:1078C0000170002010BD022010BD00004068014082
:1078D000704770B50446084694F8A010012918D0E6
:1078E000012584F8A050022184F8A11002EB820146
:1078F00001EBC20104EB810138314862204601F0FE
:10790000E5FF2068456284F8A150002084F8A000BB
:1079100070BD022070BD70B50446084694F8A010F2
:10792000012918D0012584F8A050022184F8A11063
:1079300002EB820101EBC20104EB810138314861A5
:10794000204601F0C3FF2068456284F8A150002062
:1079500084F8A00070BD022070BD70B504460846D2
:1079600016461A4694F8A01001291FD0012584F864
:10797000A050022184F8A11002EB820101EBC201A8
:1079800004EB8101383108608B6A184448608E60CE
:10799000C86A3044C860204601F098FF20684562FC
:1079A00084F8A150002084F8A00070BD022070BDB2
:1079B0002DE9F0410446084617461A4694F8A010EF
:1079C00001291FD0012584F8A050022184F8A110BC
:1079D00002EB820101EBC20104EB81013831002688
:1079E0000E6048608E60CF608862CF62204601F0F2
:1079F0006DFF2068456284F8A15084F8A0600020E3
:107A0000BDE8F0810220FBE7144A41781160111DA6
:107A100003780A1D002B1CD043680B60017BC37ADE
:107A2000090741EA0361837A41EAC341437B41EAA2
:107A30008341837B41EA4341C37B41EA0341437A6B
:107A400041EA0321037A007841EA430101431160CE
:107A500070470020086010607047000098ED00E05B
:107A6000BFF35F8F0448016821F48031016002494F
:107A7000002070310860704724ED00E0074940F0B5
:107A80000100086005487038016841F480310160E8
:107A9000BFF34F8FBFF36F8F7047000094ED00E08E
:107AA00008B51F48016841F080510160006800F08E
:107AB000805000901A48001D016841F48041016027
:107AC000006800F480400090032000F059F8002284
:107AD0006FF00B00114600F033F800226FF00A003F
:107AE000114600F02DF800226FF00900114600F059
:107AF00027F80022501F114600F022F80022101F24
:107B0000114600F01DF80022901E114600F018F8F2
:107B10000022BDE80840501E114600F011B80000D8
:107B200040380240002809DB012100F01F0291408B
:107B30004009800000F1E020C0F80011704700000B
:107B4000F0B40D460D4B1B68C3F30223C3F10704C9
:107B5000042C00D90424191D072901D2002300E0B8
:107B6000DB1E012606FA04F1491E294099409E4079
:107B7000761E16403143F0BC0BF016B80CED00E059
:107B800000F00701054A10684FF6FF03184040EA6D
:107B90000120034908431060704700000CED00E02D
:107BA0000000FA05F8B51948016841F080510160FC
:107BB000006800F080500090154C206840F4803040
:107BC0002060FFF705FC05464FF47A7606E0FFF7E4
:107BD000FFFB401BB04201D90320F8BD6068C00321
:107BE000F5D5206840F400302060FFF7F1FB054632
:107BF00006E0FFF7EDFB401BB04201D90320F8BDC2
:107C000060688003F5D50020F8BD000040380240D0
:107C1000007000402DE9F84F044600250026DFF8EB
:107C200008A42078C0070ED0DAF8000020F4000085
:107C3000CAF80000DAF80000616B0843CAF80000D7
:107C4000606B00B901252068F84F00030CD5386837
:107C5000E16B20F4401008433860E06BB0F5801F02
:107C600000D1012500B901262068C0020CD5386872
:107C7000216C20F4400008433860206CB0F5800F80
:107C800000D1012500B901262068C10100D50125D8
:107C900080066BD5E4483830016841F080510160BE
:107CA000006800F080500090DFF88493D9F800005D
:107CB00040F48070C9F80000FFF78AFB804608E0B6
:107CC000FFF786FBA0EB0800642802D90320BDE87B
:107CD000F88FD9F80000C005F2D5DFF85083A8F17D
:107CE0001C08D8F8000000F4407060B3218E01F445
:107CF0004071814227D0D8F8000020F44070D8F8B5
:107D0000001041F48031C8F80010D8F8001021F4B8
:107D10008031C8F80010C8F80000D8F80000C0078B
:107D200011D0FFF755FB814641F2883B07E0FFF792
:107D30004FFBA0EB0900584501D90320C7E7D8F84D
:107D400000008007F3D5206BC0F3012103297DD00B
:107D5000DAF8000020F4F810CAF80000D8F80000A3
:107D6000218EC1F30B010843C8F800002078C0063B
:107D700007D5386820F0807038603868A16B0843F8
:107D8000386020884104AB4805D50168626E21F453
:107D90004031114301602188090405D50168A26EB4
:107DA00021F44021114301602168C90305D5016810
:107DB000E26E21F44011114301602168890305D569
:107DC0000168226F21F440011143016021784906C6
:107DD00005D50168626C21F003011143016021782F
:107DE000090605D50168A26C21F00C011143016060
:107DF0002188C90505D50168E26C21F030011143E5
:107E000001602188890505D50168226D21F0C00136
:107E1000114301602188490505D50168626D21F48F
:107E20004071114301602188090505D50168A26DE3
:107E300021F44061114301602188C90405D501681E
:107E4000E26D21F440511143016000E05FE02188C0
:107E5000890405D50168226E21F440411143016077
:107E60002168490205D50168A26F21F080611143A4
:107E7000016021684FF00069890209D50168E26F4D
:107E800021F0006111430160E16F494500D10126F5
:107E900021680A0700D50126490305D50168626FEC
:107EA00021F04071114301602168090206D5016883
:107EB000D4F8802021F080511143016021684901EC
:107EC00006D50168D4F8842021F0005111430160E7
:107ED0002068000106D53868D4F8881020F00070BA
:107EE000084338602068C00006D53868D4F88C1084
:107EF00020F0806008433860DFF82C81012DA8F164
:107F000008080ED02068B0F1007F0AD09CE0DAF8B3
:107F10000010494A21F4F81110400143CAF800103A
:107F20001CE7D8F8000020F08060C8F80000FFF7D8
:107F30004FFA054606E0FFF74BFA401B642801D9CB
:107F40000320C4E6D8F800000001F4D420783B49AF
:107F5000C00711D0606B78B90868C0F301400A68A7
:107F6000C2F3036263689B0143EA004040EA026097
:107F7000227A40EA027008602068020303D5E26BAF
:107F8000B2F5801F05D0C0021AD5206CB0F5800F65
:107F900016D10868C0F301400A68C2F30272636830
:107FA0009B0143EA0040237B40EA036040EA027001
:107FB00008603868626A20F01F00521E1043386063
:107FC0002068C0010FD50868C0F303600A68C2F3D7
:107FD00002726368258A9B0143EA054343EA006015
:107FE00040EA02700860206880010BD56068228A30
:107FF000800140EA0240227B40EA0260227A40EAA5
:1080000002700860D8F8000040F08060C8F80000F6
:10801000FFF7DEF9054613E0FFF7DAF9401B6428A5
:108020000ED9032053E60000083802408C38024085
:108030000070004090380240FFFCFF0F843802407F
:10804000D8F800000001E7D5012E7DD1D8F8000056
:1080500020F08050C8F80000FFF7BAF9054606E0A6
:10806000FFF7B6F9401B642801D903202FE6D8F8A2
:108070000000C0438000F3D520683449020301D5D5
:10808000E26B1AB1C00219D5206CB8B90868C0F308
:1080900001400A68C2F3027263699B0143EA00402F
:1080A000237E40EA036040EA02700860386820F4EA
:1080B000F852A06A401E42EA002038602068800220
:1080C00012D5E06F48450FD10868C0F303600A6815
:1080D000C2F302726369258C9B0143EA054343EABC
:1080E000006040EA027008602078000715D5086833
:1080F000C0F303600A68C2F3014263699B0143EA6B
:10810000024242EA0060227F40EA0270086038685A
:10811000E16A20F4403008433860D8F8000040F0AD
:108120008050C8F80000FFF753F9044607E00BE061
:10813000FFF74EF9001B642801D90320C7E5D8F8E2
:108140000000C0438000F3D40020C0E5883802401E
:108150002DE9F04704460D46002C17D0DFF830819A
:10816000D8F8000000F00F00A84211D2D8F80000A3
:1081700020F00F002843C8F80000D8F8000000F0F5
:108180000F00A84204D00120BDE8F0870120FBE7E2
:108190002068404E810712D5400703D5306840F46F
:1081A000E05030602078000703D5306840F460402C
:1081B00030603068A16820F0F0000843306020781B
:1081C000C0072ED0334960680839012806D002283C
:1081D00009D0096889070BD40120D5E7096889030C
:1081E00006D40120D0E70968890101D40120CBE73A
:1081F000316821F0030101433160FFF7E9F80746D8
:1082000041F2883906E0FFF7E3F8C01B484501D981
:108210000320B9E73068616800F00C00B0EB810F13
:10822000F1D1D8F8000000F00F00A8420ED9D8F81C
:10823000000020F00F002843C8F80000D8F8000024
:1082400000F00F00A84201D001209DE720784007F0
:1082500005D53068E16820F4E050084330602078AC
:10826000000706D53068216920F4604040EAC1006B
:10827000306000F015F83168074AC1F30311515C12
:10828000C840064908600F20FFF7DEF800207BE7B2
:10829000003C0240083802402032010888130020C8
:1082A00010B51748006810F00C01164816D0164B90
:1082B000042912D0082911D1114C241F216801F082
:1082C0003F02216849020AD52068C0F38810A0FB4C
:1082D00003010023F8F70EF809E0184610BD2168E5
:1082E0000023C1F38811A1FB0001F8F703F821680E
:1082F000C1F30141491C4900B0FBF1F010BD000081
:10830000083802400024F40040787D012DE9F84F40
:1083100004464FF00008002C15D02078DFF8C093F9
:10832000A9F10407C007A7F1040560D0D9F800003F
:10833000C0F3810001280CD0D9F80000C0F38100FF
:10834000022803D00CE00120BDE8F88F3868400215
:1083500006D5286880034AD5606870BB0120F3E722
:108360006068B0F5803F11D0A8B1B0F5A02F1BD048
:10837000286820F480302860286820F48020286055
:10838000606830B3FFF724F806461EE0286840F422
:1083900080302860F4E7286820F48030286028685E
:1083A00020F480202860EBE7286840F480202860D3
:1083B000286840F480302860E2E718E0FFF708F80A
:1083C000801B642801D90320BEE728688003F5D507
:1083D0000DE0FEF7FDFF064606E0FEF7F9FF801B05
:1083E000642801D90320AFE728688003F5D42078FA
:1083F00080074BD5D9F8000010F00C0F08D0D9F841
:108400000000C0F38100022812D1386840020FD466
:108410002868800704D5E068012801D0012093E78F
:108420002868216920F0F80040EAC10028602DE0AA
:10843000E068C8B1286840F001002860FEF7C8FF76
:10844000064606E0FEF7C4FF801B022801D9032080
:108450007AE728688007F5D52868216920F0F800B8
:1084600040EAC100286011E0286820F0010028607F
:10847000FEF7AEFF064606E0FEF7AAFF801B0228C5
:1084800001D9032060E728688007F5D42078000729
:1084900030D5DFF84CA260690AF16C0AA8B1DAF8AD
:1084A000000040F00100CAF80000FEF791FF064608
:1084B00006E0FEF78DFF801B022801D9032043E769
:1084C000DAF800008007F4D514E0DAF8000020F0B4
:1084D0000100CAF80000FEF77BFF064606E0FEF743
:1084E00077FF801B022801D903202DE7DAF800006E
:1084F0008007F4D42078400775D5DFF8E4A10AF1AD
:10850000380ADAF80000C0000CD4DAF8000040F0B5
:108510008050CAF80000DAF8000000F080500090A7
:108520004FF00108DFF8BCB1DBF80000C00514D43F
:10853000DBF8000040F48070CBF80000FEF748FF45
:10854000064606E0FEF744FF801B642801D903209D
:10855000FAE6DBF80000C005F4D5DFF884B1A068C6
:108560000BF1680B012814D0D0B1052825D0DBF819
:10857000000020F00100CBF80000DBF8000020F044
:108580000400CBF80000A06870B3FEF721FF064698
:108590002BE0DBF8000040F00100CBF80000F2E730
:1085A000DBF8000020F00100CBF80000DBF8000051
:1085B00020F00400CBF80000E5E7DBF8000040F015
:1085C0000400CBF80000DBF8000040F00100CBF81D
:1085D0000000D8E7FEF7FCFE811B41F288308142A3
:1085E00003D90320B0E61FE004E0DBF800008007B9
:1085F000F0D510E0FEF7ECFE064608E0FEF7E8FED8
:10860000811B41F28830814201D903209CE6DBF8CE
:1086100000008007F2D4B8F1010F05D1DAF80000AC
:1086200020F08050CAF80000A069E8B3D9F8001023
:10863000C1F38101022951D0022807D0286820F017
:1086400080702860FEF7C4FE044642E0286820F0EF
:1086500080702860FEF7BCFE064606E0FEF7B8FE16
:10866000801B022801D903206EE628688001F5D41A
:1086700054F81C0F4FF0FF336168E2680843A168AB
:1086800003EB5202890141EA02410843217C40EA9E
:108690000160217D40EA01703860286840F08070F8
:1086A0002860FEF795FE00E016E0044606E0FEF7BF
:1086B0008FFE001B022801D9032045E628688001AF
:1086C000F5D509E0FEF784FE001B022801D903203E
:1086D0003AE628688001F5D4002035E6012033E62B
:1086E000083802400070004070B504460D46002C6A
:1086F00003D094F82C0010B107E0012070BD0020D9
:1087000084F82D00204600F011F8022084F82C0097
:108710002068211DF9F71BFED4E900022946F9F76C
:1087200055FE012084F82C00002070BD704710B564
:10873000044694F82C0002280AD0022084F82C0069
:108740002068F9F72DFE012084F82C00002010BDD0
:10875000022010BD70B504460D4694F82C00022886
:108760000ED0022084F82C0020682946F9F71EFE5E
:108770002868022806D0012084F82C00002070BD53
:10878000022070BD052084F82C00F7E710B5401ECC
:10879000B0F1807F01D3012010BD4FF0E024606173
:1087A0000F2160170AF000FA0020A0610720206165
:1087B000002010BD70B5FF23104CB3EB116F05D135
:1087C0002346050E1B680AD0FF2D14D00C4B02EB7C
:1087D0000212D2B21B6898472168084070BD51420E
:1087E00001EB01114FF07F4220F07F4002EB01616D
:1087F0000843184070BD01EA030070BD1017002047
:10880000D813002002490A6808601046704700002B
:10881000101700200449054A0968497C52F82110C4
:10882000096909680847000020140020541400203A
:10883000C1B2C0F30722C0F30740914207D1824280
:1088400005D111200831B1FBF0F07830704701EB11
:108850008103FF2100EB800002EB82027F307F3337
:108860007F32B0FBF1F0B3FBF1F3B2FBF1F202EBBC
:10887000420103EB410100EBC00001EB80006C28DA
:10888000E4D32830704700002DE9F04F05468DB045
:108890007B48DDF860901A9C00681E4617464FF032
:1088A000000A78B11B9B199ACDF808900593CDE981
:1088B0000324DDE91623CDE90023046833463A4654
:1088C000284680E0DDE9160201EB060805EB070CFF
:1088D0001043A8F10108ACF1010C012806D0C9F140
:1088E00008000590002002910990C6E065480268E2
:1088F000B2F90A30581A002806DD361A002E63DD58
:108900001946199B00FB0344B2F90E00A8EB0000C6
:10891000002802DD361A002E56DDB2F90C00ACEB51
:108920000000002800DD3F1AB2F908300020AB42F9
:1089300035DD581B3F1A4B46B9F1080F26D006DC2F
:10894000012B0BD0022B11D0042B28D116E0102BB9
:108950001ED0182B1FD0202B21D11CE020F00703A4
:1089600004EBE0041D4400F0070018E020F00303CE
:1089700004EBA0041D4400F0030010E020F001030C
:1089800004EB60041D4400F0010008E0044404E02E
:1089900004EB400401E004EB800405440020002FB8
:1089A00012DD1B9BDDF864C0CDE90403CDE900694D
:1089B000CDE902C4527C34483B4650F82200C268DC
:1089C00054680A462946A0470DB0BDE8F08F1799B4
:1089D000029808440C902B49401E00900A68B2F996
:1089E0000A30834241DCB2F90E10029881423CDB2E
:1089F0004FF0000BD84603950A9434E0BBF1000F0A
:108A000005D10A984FF0080B10F801AB0A900599B0
:108A1000ABEB090B3AFA01F00AFA09F101F0FF0A8F
:108A200004D118490968097C890716D415490968D1
:108A3000C96B0A680B921B9A0AB152F820000860B1
:108A400016990398009B4218521E029900F0A8F84C
:108A50000C490B980968C96B08600399169808F1CE
:108A6000010808440390B845C8DB0998401C0990E8
:108A70000C980290199804440998B042A7DBA3E728
:108A80007C1400202014002054140020F0B40C4664
:108A900012490968B1F90A30A3421CDCB1F90E3061
:108AA000A34218DBB1F90830834200DD1846B1F962
:108AB0000C30934200DA1A4682420CDB4B7C0849A8
:108AC00051F8235013462246E9688E68014628462D
:108AD000B446F0BC6047F0BC704700002014002092
:108AE000541400200A46174930B40968B1F90A3015
:108AF000934225DCB1F90E30934221DBB1F9083005
:108B000083421DDCB1F90C30834219DB0B7C0E4C27
:108B1000DB0709D0497C54F82130D968CC6901467B
:108B2000A44630BC18466047CB6B497C1B6854F8A0
:108B30002140E1688D6901462046AC4630BC604763
:108B400030BC70472014002054140020124B30B465
:108B50001B68B3F9084084421CDCB3F90C40844222
:108B600018DBB3F90A408C4200DD2146B3F90E4010
:108B7000944200DA22468A420CDB5C7C074B53F8B5
:108B80002440E368DD6813460A4601462046AC46A9
:108B900030BC604730BC70472014002054140020C3
:108BA00038B5134C2468B4F90850854200DD2846D6
:108BB000B4F90C50954200DA2A46824217DBB4F928
:108BC0000A508D4200DD2946B4F90E509D4200DA6C
:108BD0002B468B420BDB0093647C064B53F82440FE
:108BE000E3681D6913460A4601462046A84738BD7A
:108BF0002014002054140020082107F00DB80000B4
:108C000002480068806B0068704700002014002054
:108C100002480068C06B0068704700002014002004
:108C2000044B03EB800253F82000C068436A1046EF
:108C300018470000541400200C2106F0EDBF0D2150
:108C400006F0EABF024809210068407C06F0E4BF54
:108C500020140020092106F0DFBF70B500252C4646
:108C60002046FBF7C1FA00B16D1C641C022CF7DB37
:108C7000284670BD02480068407C00F003B8000040
:108C80002014002010B5FBF7AFFA002805D0C1680A
:108C9000CA6ABDE810400221104710BDF8B515465C
:108CA0000E460124FBF7A0FA009058B1C0680421D9
:108CB000426A68469047030004D02A46314600982D
:108CC000984700242046F8BD0E2106F0A5BF0321D9
:108CD00006F0A2BF032007F044B8042106F09CBFB1
:108CE000024801210068407C06F096BF2014002055
:108CF0000148006870470000DC140020012106F0E4
:108D00008BBF012007F02DB8024802210068407C8B
:108D100006F082BF20140020014840687047000020
:108D2000DC140020022106F077BF022007F019B8FA
:108D300000F002B8AFF300802DE9F041060008D042
:108D4000B76837B11248816819B13468B4F5807FCB
:108D500002DD0020BDE8F08101688C4200DD0C4698
:108D60000025804609E000BF57F82500FFF752FDB7
:108D7000D8F8081041F825006D1CA542F4DBD8F89E
:108D80000410444609B130468847A068E2E7000075
:108D9000C81400200449054A0968497C52F821108A
:108DA0000969496808470000201400205414002075
:108DB00010B5A0F17801102906D201EB011000EBEB
:108DC000012000EB003010BD6C2804D3942801D2A0
:108DD000002010BD28380621B0FBF1F3B0FBF1F202
:108DE000B3FBF1F401FB120201FB14312423B0FBAD
:108DF000F3F002EB021201EB011102EB420201EB74
:108E0000410100EB001000EB400002EB012101EBFF
:108E1000004010BD7047000010B500F01F01074A68
:108E2000074BC0F34514C0F3C4201B5D105C515CBC
:108E300000EB032000EB014010BD0000B846010824
:108E4000D8460108F8B500F0B9F900F049F8040077
:108E500040D100252846FBF7C7F9009048B1C0680B
:108E60000C21426A68469047010007D00098884765
:108E700004436D1C022DEDDB14B12BE00120F8BD85
:108E800000F048F8144815490068884222D00125AE
:108E900043F6FF762846FBF7A7F90090C0B12846B5
:108EA000FCF720FA042000F0C5F9002132463346D1
:108EB0000846FFF775FE002000F0BCF900980E216F
:108EC000C068426A68469047010001D00098884710
:108ED0006D1EDFD52046F8BD1C140020785634FFE7
:108EE00010B50A4CA06860B920688000FAF772FEDD
:108EF000A06040B104F10C01054808600846FDF788
:108F0000E1FB002010BD012010BD0000C8140020AE
:108F10007D0F01082DE9F047FFF79FFE074600246B
:108F2000DFF860802AE02046FBF75EF928B3D8F826
:108F3000000090F8119044742046FFF75DFE082869
:108F400017DC1148114950F824000069884210D0FC
:108F50002046FFF77FFE0646002508E0E8B2FFF74F
:108F600019FF0246E9B2204600F06AF96D1CB542CD
:108F7000F4DBD8F8001081F81190641CBC42D2DBFD
:108F8000BDE8F08720140020541400206C4A01082A
:108F90002DE9FF4F83B01646DDE910408B46C068CF
:108FA0004769426A7AB1012111A8904705000AD0A9
:108FB0000698CDE9000433465A4603991198A8470C
:108FC00007B0BDE8F08F57480068407CFBF7E2FB34
:108FD0008246082801DC012005E0BAF1100F01DC0F
:108FE000022000E004208046002596E04046B8F1CB
:108FF000010F05D0022871D0B8F1040F25D17CE013
:10900000BAF1090F21D2DFE80AF08605213F3F5966
:1090100059595900039815E001465A461198B84726
:10902000C5F1070188404FF67F722178EA40114070
:1090300001436D1C217004EBE50425F00700054198
:1090400009F101008146B042E6DD64E0039817E0D3
:1090500001465A461198B8470621A1EB45018840C0
:109060006B004FF63F722178DA40114001436D1CCE
:10907000217004EBA50425F00300054109F101006E
:109080008146B042E4DD46E0039813E001465A46CB
:109090001198B8470421A1EB850188402178AB00E5
:1090A0000F229A401140014321702C4485F00105A4
:1090B00009F101008146B042E8DD2CE0DDF80C90BA
:1090C00007E001465A461198B847207009F1010996
:1090D00044444846B145F4DD1DE0FFE7DDF80C905F
:1090E00007E001465A461198B847208009F1010966
:1090F00044444846B145F4DD0DE0DDF80C9007E04E
:1091000001465A461198B847206009F101094444C4
:109110004846B145F4DD0BF1010B06998B457FF70D
:1091200065AF4DE72014002010B50D4C0D492068A7
:10913000407C51F8200048B1C16811B10968042988
:1091400001D00068F7E708B1FBF730F8206800218C
:10915000016600F108014161BDE8104000F02EB841
:109160002014002054140020014909684968084768
:10917000C4140020044909680A7C520701D5C96B50
:1091800000E0896B08607047201400207CB5094C12
:1091900005462068417C084850F82100C1680A6BE8
:1091A0006946904720686A4629460830FDF782F9EB
:1091B0007CBD0000201400205414002004480168E5
:1091C00004484A7C083150F82200C268126B1047EC
:1091D0002014002054140020014909680968084738
:1091E000C4140020044909680A7C520701D5896B20
:1091F00000E0C96B0860704720140020F8B51546E0
:109200000E460124FAF7F0FF009058B1C06816210D
:10921000426A68469047030004D02A4631460098C7
:10922000984700242046F8BD014AC2E90001704772
:10923000DC1400200149096889680847C41400202B
:10924000F8B515460E460124FAF7CEFF009058B146
:10925000C0681021426A68469047030004D02A463D
:1092600031460098984700242046F8BDF8B51546C9
:109270000E460124FAF7B8FF009058B1C0680B21E0
:10928000426A68469047030004D02A463146009857
:10929000984700242046F8BD38B50D460124FAF75A
:1092A000A3FF009050B1C0680921426A6846904708
:1092B000020003D02946009890470024204638BD7C
:1092C000F8B515460E460124FAF78EFF009058B106
:1092D000C0680A21426A68469047030004D02A46C3
:1092E00031460098984700242046F8BD10B5074C39
:1092F0002068006BFFF78EFAFFF774FF2068406B61
:10930000FFF788FABDE81040FFF734BF20140020B3
:1093100070B500233D493E481A46FAF7DBFE0020AF
:10932000FFF7D2FC4FF448744FF4F07550B10020B1
:1093300022462946FFF79AFF002022462946FFF7DA
:10934000BFFF09E000202A462146FFF78FFF0020DB
:109350002A462146FFF7B4FF00242E4D2E4E20460C
:1093600055F82410FFF798FF2046FFF745FCC01082
:1093700046F82400641C012CF1DB0024254E361D28
:1093800056F8240000BB254A21212046FFF736FF6E
:10939000234A23212046FFF731FF204606F034FD03
:1093A0000546042D09D81F4A19212046FFF726FF3C
:1093B0001D4A25212046FFF721FF022D04D11B4A1B
:1093C00024212046FFF71AFF641C012CD8DB184922
:1093D0001848FAF7A3F918491848FAF7A5F91849EF
:1093E0001848FAF7ADF918491848FAF7A3F91848D8
:1093F000FBF7CCFF1748FBF7D1FF1748FBF7D4FF6B
:10940000BDE870401548FBF7D7BF0000F0320108F7
:109410001433010830320108B41300203505010867
:109420008105010819070108B1060108490601086C
:109430002D01010839CB000895010108A5CB0008D2
:10944000AD010108BDCB0008A1010108B1CB0008A6
:1094500031D00008B107010805D20008C50A01088B
:109460002DE9FC4105460F46144600263648374A8A
:109470000068904201D007F0B9FA0F2F5ED2DFE802
:1094800007F05D085D0C161C1F2C27224E5D5358FB
:109490001100284607F0B8F952E006CC284607F03C
:1094A0008FFB4DE02A49206841F8250048E02279E9
:1094B0002846216807F058FB42E007F0ADF83FE08E
:1094C00007F092F83CE02168284607F093FB37E06C
:1094D00006CC284607F068FB32E001A96A46284618
:1094E000FBF7CAF92846FFF7EFFB02001848A0F186
:1094F0000C0000F1040106D0626840F825202068C5
:1095000041F8250005E0226840F82520606841F810
:109510002500DDE90021284607F04CFB10E021681A
:10952000284607F039FB0BE02168284607F010FBBE
:1095300006E006CC284607F0FBFA01E04FF0FF36C4
:109540003046BDE8FC810000A04D002000680140CD
:10955000B81300207047704730B5ABB01B480168A6
:1095600041F400710160006800F4007001904FF454
:10957000004402940120039004900320059002A966
:10958000134D2846FDF726FE002221462846FDF70A
:1095900018FF1420FDF70CFE012221462846FDF796
:1095A00010FF0A20FDF704FE082007904FF4C0705A
:1095B0000C9004200E900020129007A8FEF72AFBC2
:1095C00007A8FEF727FB2BB030BD00003038024063
:1095D000002402402DE9FF4F8DB01746674ADDF8A1
:1095E00070901E9E209812681D4600248AB11D9B13
:1095F0001F98CDE90293CDE90460DDE91A03CDE9B6
:10960000000314682B463A460D98A04711B0BDE8F8
:10961000F08F0D9A01EB050802EB070CDDE91A2328
:109620001A43A8F10108ACF1010C012A06D0C9F1D6
:1096300008004FF0000B029105909CE0504A126820
:10964000B2F90A40631A002B06DDED1A002DDDDDAC
:1096500021461D9C03FB0466B2F90E30A8EB030300
:10966000002B02DDED1A002DD0DDB2F90C30ACEB91
:109670000303002B00DDFF1A0D9B1C1AB2F9083002
:10968000A3420DDDA3EB040C0CEB0003181A20F031
:1096900007000444A7EB0C0706EBE30603F0070002
:1096A000002FB3DDDDF874C01F9BCDE902C6CDE904
:1096B0000403CDE90059527C32483B4650F8220061
:1096C000C26855680A462146A8479FE71B99029839
:1096D00008440C902A49401E00900A68B2F90A30EA
:1096E000834242DCB2F90E10029881423DDB4FF01A
:1096F000000A0D980A96D046039034E0BAF1000FA4
:1097000005D10A984FF0080A10F8014B0A90059904
:10971000AAEB090A34FA01F004FA09F4E4B204D11C
:1097200017490968097C890717D415490968C96B65
:109730000A680B921F9A0AB152F820000860039938
:109740001A98009B0A18DDE90210521EFFF728FA4A
:109750000B490B980968C96B086003991A9808F1BE
:10976000010808440390B845C8DB0C9802901D9886
:109770000BF1010B0644AB45A8DB47E77C14002046
:109780002014002054140020002818D0410817D0BD
:10979000810817D0C10817D0010917D0410917D087
:1097A000010A17D0410A17D0010B15D0C10B13D0F5
:1097B000010C11D0810C11D0000E11D02020704767
:1097C0000120704702207047032070470420704733
:1097D00005207047082070471020704712207047FE
:1097E0001820704700B50022FFF7CEFF012804D0F3
:1097F000811E062903D808220BE0012209E0A0F10E
:109800000901072901D8102203E011380F2800D8D8
:109810002022104600BD0220704700002DE9F041D3
:1098200086B01148016841F400710160006800F4DD
:109830000070009000240D4D00264FF00208012713
:1098400005EBC400808801900297CDF80C80049647
:1098500001A955F83400FDF7BDFC641C022CEFD3C0
:1098600006B00020BDE8F08130380240A431010884
:1098700010B50024022809D2064A02EBC00152F8B2
:10988000300000228988FDF79CFD01E04FF0FF3495
:10989000204610BDA431010810B50024022809D2C9
:1098A000064A02EBC00152F8300001228988FDF718
:1098B00088FD01E04FF0FF34204610BDA4310108BF
:1098C0000148FDF7C7BE0000A04D0020F0B50368B9
:1098D0008C88DD68C5F30B452C442504882404EBF3
:1098E000C2141E5906F470461E5103680F68DE68E4
:1098F000C6F30B46761C3E442E431E5103688C89EA
:10990000DD68C5F30A052C4425048C2404EBC2143D
:109910001E5906F470461E5103688F68DE68C6F350
:109920000A06761C3E442E431E510468942303EB22
:10993000C213E55825F00705E55005680C69EC50A1
:1099400091F831304FEA032C91F832301E040B7E2F
:109950001F0604689C2303EBC213E5580025E5505D
:1099600091F830403E4344EA0C0434430668F45016
:109970000468982303EBC213E65826F0FF06E6506E
:1099800006684C69F4500468A02303EBC213E65840
:1099900040F20777BE43E650D1E9074634430668F4
:1099A000F4500468AC2303EBC213E658E550056895
:1099B0004C6AEC500B69002B31D0012B31D0042BB9
:1099C00031D0022B2FD0032B2DD0072B2BD00123EE
:1099D0000568B02404EBC2142E5906F0E0262E517F
:1099E000D1E90065AD1B0E8D5D43ED1C5E4345EA7C
:1099F000064305682B510468B42303EBC213E558F2
:109A00006FF30A05E5500468C96AE15000688421D3
:109A100001EBC211425842F001024250F0BD042352
:109A2000D6E70323D4E70223D2E71FB5FEF718F8E1
:109A300001218DF800104FF04040019017208DF863
:109A4000080003208DF80B0000208DF80F008DF822
:109A50000E008DF80D008DF801008DF80A108DF8BC
:109A600009008DF80C106846FDF7CEFF0420FEF7C4
:109A700005F81FBD7FB51448124901604FF48031CD
:109A800041600024846004610125856104624562AF
:109A9000C4620E498162C460C56104634561FCF71C
:109AA000C0FF08B1F8F752FC08200090019502941D
:109AB00069460548FCF7FAFE002801D0F8F746FC95
:109AC0007FBD000000220140341800200100000F7B
:109AD00008B50948016841F080010160016801F0A2
:109AE00080010091016841F020010160006800F0F0
:109AF0002000009008BD000030380240FDF758BB40
:109B000070B504460D46FE490020F8F707FCFC49F5
:109B100003206F31F8F702FCF9490020891CF8F79F
:109B2000FDFBF74902206631F8F7F8FBF449002005
:109B3000891CF8F7F3FBF2490020091DF8F7EEFB4A
:109B40000A20FFF7DBFFEE490020891DF8F7E6FB4E
:109B5000EB4900200831F8F7E1FB0A20FFF7CEFFC0
:109B6000E74900200A31F8F7D9FBE54900200C311C
:109B7000F8F7D4FBE24900200E31F8F7CFFBE049BB
:109B800000201031F8F7CAFBDD4900201231F8F748
:109B9000C5FBDB4900201431F8F7C0FBD849002091
:109BA000F8F7BCFBD64900201631F8F7B7FBD449CB
:109BB00000201831F8F7B2FBD14900201A31F8F72C
:109BC000ADFBCF4900201C31F8F7A8FBCC490020A1
:109BD0001E31F8F7A3FBCA4900202031F8F79EFB9D
:109BE000C74900202231F8F799FBC54900202431EC
:109BF000F8F794FBC24900201031F8F78FFBC049F9
:109C00000020F8F78BFBBE4902206931F8F786FB8C
:109C1000BB4900202631F8F781FBB94900202831E3
:109C2000F8F77CFBB64900202A31F8F777FBB449F6
:109C300000202C31F8F772FBB14900202E31F8F7E3
:109C40006DFBAF4900203031F8F768FBAC490020CC
:109C50001831F8F763FBAA4900203231F8F75EFBB0
:109C6000A74900201C31F8F759FBA54900203431E1
:109C7000F8F754FBA24900203631F8F74FFBA04912
:109C800002206C31F8F74AFB9D490020891CF8F747
:109C900045FB9B4906208131F8F740FB984900209D
:109CA0003831F8F73BFB96490E20AA31F8F736FB1E
:109CB000934900203A31F8F731FB91490E20B93130
:109CC000F8F72CFB8E4900203C31F8F727FB8C4934
:109CD0000A20C831F8F722FB894900203E31F8F705
:109CE0001DFB874900205A31F8F718FB84490020F2
:109CF000891CF8F713FB82490A20D331F8F70EFBD1
:109D00007F4900204031F8F709FB7D490F20DE3103
:109D1000F8F704FB7A4900203831F8F7FFFA784960
:109D20000F20EE31F8F7FAFA754900203A31F8F7CA
:109D3000F5FA73490A20FE31F8F7F0FA704900206D
:109D40003C31F8F7EBFA6F490F20F8F7E7FA6C4966
:109D500000203E31F8F7E2FA6A490F201031F8F797
:109D6000DDFA674900204231F8F7D8FA65490A2040
:109D70002031F8F7D3FA624900204431F8F7CEFADF
:109D800060490A202B31F8F7C9FA5D490020891C87
:109D9000F8F7C4FA5B490A203631F8F7BFFA584998
:109DA00000204031F8F7BAFA56490F204131F8F750
:109DB000B5FA534900203831F8F7B0FA51490F206D
:109DC0005131F8F7ABFA4E4900203A31F8F7A6FACC
:109DD0004C490A206131F8F7A1FA494900203C3189
:109DE000F8F79CFA47490F206C31F8F797FA444985
:109DF00000203E31F8F792FA42490F207C31F8F703
:109E00008DFA3F4900201831F8F788FA3C490020C4
:109E10005C31F8F783FA3A4900205E31F8F77EFAB0
:109E2000374900206031F8F779FA3549002062316E
:109E3000F8F774FA324900206431F8F76FFA3049C4
:109E40000020F8F76BFA2E4903207331F8F766FA11
:109E50002B490020F8F762FA29490020F8F75EFA4A
:109E6000284910208139F8F759FA25490020F8F7D8
:109E700055FA244910207039F8F750FA204900208B
:109E80004631F8F74BFA7820FFF738FE3CB1022C48
:109E90000AD11B4900204831F8F740FA04E018497C
:109EA00000204A31F8F73AFA012D0ED1144900206A
:109EB0004C31F8F733FA124904207731F8F72EFACB
:109EC0000F4904207C31F8F729FA0D4900204E3162
:109ED000F8F724FA0A4900205031F8F71FFA084928
:109EE00000205231F8F71AFA054900205431F8F7EA
:109EF00015FA034900205631F8F710FA004903E03B
:109F00000C300108153101080020F8F707FA034961
:109F10000020F8F703FA002070BD0000643001084B
:109F200038B5446805460146204600F030FD00285B
:109F300011D028680B280FD00F2817D12046F9F729
:109F4000CFFE0090406E05686846F9F71FFF002DB0
:109F500001D02046A84738BD2046F9F7C1FE009041
:109F60003830F9F729FE6846F9F710FF2846BDE8B2
:109F7000384000F0B7BFF0B585B00DF1280C9CE873
:109F8000F0004FF0000C8DE8F01000F003F805B081
:109F9000F0BD00002DE9FF5F9846DDE90E569146C1
:109FA0008A468346109F129CFAF722FD25484034CA
:109FB000CDE90204CDE9005643464A46514658468B
:109FC00000F0D8FE050037D00520F9F7AFFD0400FA
:109FD00032D02846F9F784FE00220090119900F053
:109FE0000BFE1949284600F080FD184E00981822F3
:109FF00031684166311D4C30F6F7ADF90098022109
:10A00000A0F84010642181640021416480F86870E8
:10A0100084632046F9F764FE01460190002200980F
:10A0200008F0A4F801A8F9F7B1FE6846F9F7AEFE0A
:10A030003068416828468847FBF76AFC04B0284628
:10A04000BDE8F09F219F00086854010844150020D6
:10A0500070B50446006A6268052A22D01C490B2AA2
:10A0600002D0122A31D121E00868006AFBF761F9B9
:10A07000D4E90410A269FAF747FAD4E90620216965
:10A08000FAF742FAD4E90401E269491C521EFAF7D0
:10A09000FBFAD4E90510E269491C521EFAF7F4FAFA
:10A0A00013E00168204603F06FF90EE0026862B920
:10A0B00085680868406AFBF73CF90220FBF7D0F995
:10A0C000D4E904122846FAF725F9002070BD0000F3
:10A0D00064540108F0B587B00C4607007ED0FAF74B
:10A0E00087FC3846F9F7FCFD0090416CA14200DD89
:10A0F0000C46816CA14200DA0C46416BA1426ED045
:10A1000090F8681040F6FF76C907416B4FF00005E4
:10A1100019D0A14207DD214600F0C3F8ADF80E00CA
:10A120000098416B05E000F0BCF8ADF80E00214648
:10A13000009800F0B6F8ADF80A00ADF80850ADF898
:10A140000C6000985FE0A14207DD214600F0A9F80D
:10A15000ADF808000098416B05E000F0A2F8ADF8FA
:10A1600008002146009800F09CF8ADF80C0000981B
:10A17000ADF80A50ADF80E6090F86810890742D427
:10A1800004950595806BF9F79DFD05280EDA00987A
:10A19000856B6846F9F7FAFD05212846F9F7AEFD0B
:10A1A00005463846F9F79CFD00908563009800F05D
:10A1B00036F8019030B30098C06CFBF7D7F805462D
:10A1C000DDE9000204A900F02DF802A904AA08465E
:10A1D000FAF7C8FFDDE90001224601E01DE017E0C3
:10A1E00007F0C4FFDDE9000204A900F01BF802A992
:10A1F00004AA0846FAF7B6FF2846FBF7B7F801A805
:10A20000F9F7C4FD00E0446302A9384601F0E2F921
:10A210006846F9F7BBFDFBF77BFB07B0F0BD806B31
:10A22000F9F75EBD2DE9F04105460C46B0F9040092
:10A23000B5F90010471AB5F90600B5F902107F1CF0
:10A24000401A00F101081046FAF743FB0646FAF7F8
:10A2500009FBE96A95F84020096802F00302012A27
:10A2600006D0022A07D1B91B01EBD171491002E0D7
:10A27000BA1B511A491E2180A8EB000101EBD171D4
:10A28000491061802288AB8F761E1A442280EB8FA2
:10A29000324419446180401EA2800844E080BDE839
:10A2A000F08170B590F8682012F00104C26A13685A
:10A2B00004D0B0F90620B0F9025003E0B0F9042050
:10A2C000B0F90050551BD0E911206D1C914200DA05
:10A2D0001146814200DD01465E4205EB46050CB1A8
:10A2E000411A00E0891A4D43801A95FBF0F018449A
:10A2F00070BDF8B50D4604000FD0FAF779FB204683
:10A30000F9F7EEFC0090066D6846F9F73FFD71190C
:10A31000204600F031FAFBF7FBFAF8BD7CB5456842
:10A3200004460146284600F032FB002826D020686B
:10A3300023287BD006DC0B280FD00E2824D00F2832
:10A340000ED10EE024284BD0A0F5807013386AD0CF
:10A35000A0F580702D387FD111E0284600F036FA44
:10A360007AE02846F9F7BCFC0090002806D0406C43
:10A3700004686846F9F70AFD2846A0477CBD2146D7
:10A38000284607F031F867E02E462846F9F7A8FC82
:10A390000190456D01A8F9F7F9FCE068D0E90010DB
:10A3A000002859DD132913D006DC102914D01129F7
:10A3B00012D0122950D10BE0212902D022294BD1F1
:10A3C00001E0294600E069423046FFF792FF43E092
:10A3D000304600F0CEF93FE0304600F0E9F83BE0CF
:10A3E0002E463046E568F9F77BFC01902968C26C7F
:10A3F000914207D1426DAB689A4203D1026D6B68FE
:10A400009A4211D0C164A968416569680165304606
:10A4100001F020F901A8F9F7B9FC0521304601F057
:10A4200083F919E002E014E001A80FE02846F9F7EB
:10A4300057FC009080B1E168C06C08600098E26849
:10A44000416D9160E168006D48606846F9F79EFCD7
:10A4500002E0284606F05CFF204600F043FD7CBD8C
:10A460001FB50A0703D5FE2340F28A5202E0FF23FC
:10A4700040F28A32CDE90213CDE9000200231A46E8
:10A480001946184600F007F80446062101F04CF979
:10A4900004B0204610BDF0B585B00DF1280C9CE845
:10A4A000F0004FF0000C8DE8F01000F003F805B05C
:10A4B000F0BD00002DE9F04F87B01F46DDE9126ABC
:10A4C000144688468146DDF840B0FAF791FA364DD9
:10A4D00054EA070022D105A9584600F0B7FE30071C
:10A4E0000ED5B5F90040BDF91800BDF91680BDF9CB
:10A4F0001A10001BA1EB080700F101097F1C0DE0F9
:10A50000B5F90070BDF91A00BDF91490BDF9181025
:10A51000C01BA1EB090400F10108641C14981199F7
:10A52000224B3C30CDE90230CDE900B13B4622461A
:10A530004146484600F01EFC04002FD0F9F7D0FB3E
:10A5400000220490310700D50822F10601D542F01F
:10A5500010025146BAF1FF0F04D0BAF1FE0F01D03C
:10A5600042F0100200F048FB05F1080304984ECBBE
:10A5700000F1340787E84E006421C1640A21416577
:10A58000002101656968416404A8F9F7FFFB686868
:10A59000416820468847204600F018F9FBF7B8F9D3
:10A5A00007B02046BDE8F08FD01600201DA300089C
:10A5B0004FF0FF31FFF79DBEF0B504468DB0006847
:10A5C000F9F78EFB0646079007A8F9F7DFFB208A0C
:10A5D000256AADF82C00A08AADF82E00208BADF8CE
:10A5E0003000A08BADF83200DDE90B01CDE90901A7
:10A5F000286848B10BAA1146304600F005FB4C4ACA
:10A60000DFF830C14C4F03E04C4ADFF834C14D4F06
:10A61000606810283AD006DC082815D0092861D0D7
:10A620000C287FD132E0112830D013283DD01928D2
:10A6300078D1286810B12169A06901E06169E069F9
:10A64000401A401C0DB0F0BD686802281BD03E4C7B
:10A650000BA82146904708AB02AA09A8296805F073
:10A66000E5F9606AFAF765FE4FF0FF300090BDF93A
:10A670002A00BDF92610401A401C4210BDF92400E2
:10A68000089901444AE0304C2C3CE1E72E48BDF9E2
:10A690003230BDF93020016AC069CDE90001BDF951
:10A6A0002E10BDF92C00E0473CE0686803280AD072
:10A6B000254C0BA821469047286838B1BDF93200D7
:10A6C000BDF92E1006E0204C2C3CF2E7BDF930001D
:10A6D000BDF92C10401A401C0F2823DB21460BA883
:10A6E000B8471FE0686801281ED0174C0BA8214608
:10A6F000904708AB02AA09A8296805F097F9606A93
:10A70000FAF717FE01200090BDF92A00BDF92610C6
:10A71000401A4210BDF928000899411A3046029BA0
:10A7200000F004FA00208DE7074C2C3CDEE7000027
:10A73000E9D40008C54300081DEE00088DD40008C8
:10A740003D440008C1ED00086017002038B5050041
:10A750004FF000040BD0FAF74BF92846F9F7C0FA8E
:10A760000090046D6846F9F711FBFBF7D1F820461D
:10A7700038BD0121FFF7BDBD38B50C46050024D01A
:10A78000FAF736F92846F9F7ABFA0090426DC16C3A
:10A79000891A00D50021002C00DA00248C4200DD4B
:10A7A0000C46016DA1420BD00465284600F052FF13
:10A7B0006846F9F7EBFA0521284600F0B5FF02E0FC
:10A7C0006846F9F7E3FAFBF7A3F838BD10B504467D
:10A7D00000F0C1FD00F03EFF204600F0AFFDBDE8F7
:10A7E0001040252101F08DB810B590F832201207E5
:10A7F0000FD5828800880B88101A8A88401C4C88E4
:10A80000C31A0C80CC885B1E8C80801ACB80401EC3
:10A81000488010BD30B593B0012001900004029033
:10A8200000250495022407948001089019200990BE
:10A830004FF4D8700A900B9409200C9001A8FDF7F2
:10A8400065FD08B1F7F782FDFDF7ACF908B1F7F740
:10A850007DFD0F200E900F9410954FF4A050119095
:10A860004FF48050129007210EA8FDF771FC0028CC
:10A8700001D0F7F76BFD13B030BD000070B51D4E71
:10A88000306800F00C001C4B1C4900280ED01C4DF9
:10A8900004280DD008280DD00B603068194AC0F389
:10A8A0000310105C0A68C2400A6070BD0B60F4E7D8
:10A8B0000D60F2E70F4A121F1068C0F38054106851
:10A8C00000F03F0034B1B5FBF0F01368C3F3881318
:10A8D000584305E0B3FBF0F01368C3F38813584303
:10A8E0001268C2F30142521C5200B0FBF2F0086041
:10A8F000D3E70000083802400024F4008813002049
:10A9000040787D01203201081048016841F470014F
:10A9100001600F48016841F0010101600C4A00210B
:10A920000832116002680B4B1A400260031D0A4A8C
:10A930001A60026822F48022026005480C3001602F
:10A9400058060249803908607047000088ED00E031
:10A9500000380240FFFFF6FE1030002438B50D46E7
:10A96000040013D0FAF744F82046F9F7B9F900903B
:10A97000428E1146AA43914203D04286204600F0FF
:10A9800069FE6846F9F702FAFAF7C2FF38BDFEB56C
:10A990000C4606004FF001055DD0F9F7A1F90190D2
:10A9A0002168162959D008DC0D2943D0112932D04D
:10A9B00014297DD0152949D12AE000271E294FD01E
:10A9C0001F2970D0312903D0B1F5407F3ED101E07D
:10A9D000E7603AE0C16AE2680968C26210680C1A6E
:10A9E00001A8F9F7D3F9FAF703F83046F9F778F93F
:10A9F0006242234611460094029001F0F3FD02A842
:10AA0000F9F7C4F9FAF784FF304600F023FE1CE0A2
:10AA1000B0F9300045E090F83200C00616D5E06885
:10AA2000A0B1007A90B101A8F9F7B0F9304601F071
:10AA300005F80BE0E068C06840B1007A30B101A8C9
:10AA4000F9F7A4F9304600F04DF90025019810B14E
:10AA500001A8F9F79BF92846FEBDA1890186F4E714
:10AA6000E168408E012906D020F00101304600F057
:10AA700047F8092507E0C1060FD540F0010130462F
:10AA800000F03EF8082501A8F9F780F9294630467C
:10AA900000F04AFE9CE70BE005E001A8F9F776F923
:10AAA0000120E060D1E790F83200C0F30010F8E731
:10AAB000E16800F093F8C8E738B50C46050013D0FC
:10AAC000F9F796FF2846F9F70BF90090418E34EA22
:10AAD000010204D021434186284600F0BBFD6846B0
:10AAE000F9F754F9FAF714FF38BD1FB500220292A6
:10AAF0004FF4407203910092694600F0F3FE1FBDCF
:10AB000038B50C460546F9F773FF2846F9F7E8F81B
:10AB10000090418EA14203D04486284600F09AFD61
:10AB20006846F9F733F9FAF7F3FE38BD2DE9F0413D
:10AB300090F83200069F1C4616460D46000707D4C3
:10AB400011E03219311B2846F9F7DEFC3D44641E42
:10AB5000002CF6DABDE8F0813219311B2846F9F7EE
:10AB600093FD3D44641E002CF6DAF3E77CB50C003F
:10AB7000054603D1684600F0CDFA6C4695F83200E0
:10AB8000000705D522466946284600F03DF86C4688
:10AB90002146284604F0A6FB002803D0E86A016994
:10ABA000204688477CBD1CB590F832000C46000753
:10ABB0000FD5684600F0AEFABDF802002080BDF85F
:10ABC0000600A080BDF800006080BDF80400E080B1
:10ABD0001CBDBDE81C40084600F09CBA70B50C4690
:10ABE000054601F03FF9E86A21460268BDE8704079
:10ABF0000846FBF759BD0000024B1B68C362428642
:10AC000001867047EC16002030B5858800881488CE
:10AC1000281AD5889388451B0D805288801A888011
:10AC20004C80CB8030BD70B50C4616460546FE21E3
:10AC300000F0A0FA214600F0D1FFFF21284600F0E5
:10AC400099FA3146BDE8704000F0C8BF02490120C2
:10AC5000096881F854007047201400202DE9F04164
:10AC60008AB00446F9F7C4FEBCB32046F9F738F8B9
:10AC70000190D0E90012CDE90412876A056A01A8A3
:10AC8000F9F784F8204601F043F9060025D0204664
:10AC900000F054FB8046B80704D52A46414604A874
:10ACA00001F0AAFA2046F9F71BF801904046F9F79F
:10ACB00017F806903046F9F713F8039005620698E6
:10ACC000019AC1691162C46101A8F9F75FF806A889
:10ACD000F9F75CF803A8F9F759F8FAF719FE0AB082
:10ACE000BDE8F08110B50446F9F782FE204601F078
:10ACF000A9FDBDE81040FAF70BBE82680168891A09
:10AD000000D500214268002A01DA002242608A420E
:10AD100000DD4160704700002DE9F8431646884683
:10AD20000746F9F765FE0C20F8F700FF04001AD07B
:10AD3000F9F7D9FD8119012322460D48FAF7B0FB36
:10AD4000050020460CD0F8F7CBFF009080E8A0016A
:10AD50006846F9F71BF831462846FAF770FC02E01E
:10AD6000F8F706FF0024FAF7D3FD2046BDE8F88384
:10AD7000052D01082DE9FC5F9846DDE90C5491464C
:10AD80000E460746DDF83CB0F9F732FEDFF828A1A1
:10AD9000DAF81C0004434DB9BAF8020048B347483A
:10ADA0000AF148010068407C51F82050681C0ED020
:10ADB000FDB12846F8F794FF0190B0F90010B0F902
:10ADC00002200F441644B9F1000F02D006E000251E
:10ADD0000FE0B0F90430591A01F10109B8F1000F80
:10ADE00004D1B0F90600801A00F1010801A8F8F7B3
:10ADF000CDFF0BF12C00F8F799FE5FEA000B56D05F
:10AE0000BAF80200401CAAF802005846F8F768FF9A
:10AE10000090078007EB09014680491E818006EB00
:10AE20000801491EC1800E990161254A816A2240AC
:10AE3000114381626846F8F7A9FFDAF814005E460C
:10AE400050B1F8F7BBFF07463046F8F7B7FF0146A9
:10AE5000786948617E6101E0CAF814B02946584615
:10AE600001F0FAF8A00602D5584600F019FDE007F7
:10AE700004D0DAF82810491CCAF82810600602D558
:10AE80005846FFF7EBFEA0070DD55846F8F728FF08
:10AE90000090816A41F0020181626846F8F776FF0E
:10AEA000584600F0D7FB0121584601F08CFBFAF719
:10AEB0002FFD5846BDE8FC9F60150020201400209F
:10AEC0009F3F3F00064910B50968002081F85400F3
:10AED000F9F78EFDFEF772F9BDE81040FAF718BDDC
:10AEE0002014002010B50446C168D4E90020172AB8
:10AEF0000DD004DC0E2A0CD0142A07D104E0222A3B
:10AF00000CD0282A02D10BE000F09CFF0020E0606A
:10AF100010BD2146BDE8104000F000BD0248F6E734
:10AF2000BDE8104000F096BB785634FF38B50400F9
:10AF300010D0F9F75DFD2046F8F7D2FE00900068CA
:10AF4000FAF7FAFA6846F8F721FF2046F8F710FEFC
:10AF5000FAF7DEFC38BD0000F8B5050070D0F9F74F
:10AF600047FD284601F074F9002867D0284600F014
:10AF7000E1FF07460B21284601F025FB284600F09B
:10AF800000FF2846F8F7ACFE0090406A08B1F9F7D8
:10AF900039FE2C4C002104F16002A163206952F8B3
:10AFA0002030AB4201D142F82010264A583252F8E4
:10AFB0002030AB4201D142F82010A06904E0436880
:10AFC000AB4200D1416000680028F8D10721284633
:10AFD00000F0AAFB009802F067F9284600F008FF8D
:10AFE00060690CE0F8F7EAFE064640692946A84287
:10AFF00005D10846F8F7E2FE4069706101E00028DB
:10B00000F0D10098806AC10702D0A16A491EA162EE
:10B01000800602D5A088401EA0806846F8F7B6FEDC
:10B020006088401E60802846F8F7A2FD002F05DBEF
:10B030000448483050F8270000F032FCFAF768FC6A
:10B04000F8BD00006015002010B504000DD0F9F720
:10B05000CFFC2046F8F7B2FE816A42F20402914327
:10B060008162BDE81040FAF753BC10BD70B50025F1
:10B07000F9F7BEFC1A4C606B10B1804700E0012567
:10B0800004F0C6F90028FAD11648006890F8540078
:10B0900038B1A08828B1606A012620B100688047D5
:10B0A00004E0002602E00120FBF72EFAFAF730FC5C
:10B0B00000E0012504F092F90028FAD1F9F798FC94
:10B0C0004EB1606A20B1406880470020E06002E035
:10B0D0000020FBF719FAFAF71BFC284670BD0000A8
:10B0E000601500202014002070B514460D46064659
:10B0F000F9F77EFC22462946304600F08DFEBDE879
:10B100007040FAF705BC000001480068806C704789
:10B110002014002010B50446F9F76AFC06480068C0
:10B1200010B906480068806C214600F009F8BDE8B7
:10B130001040FAF7EDBB00008C1500202014002011
:10B1400070B50C460546F9F753FC2146284600F039
:10B1500079FEBDE87040FAF7DBBB00000348044904
:10B160000068407C51F82000704700002014002047
:10B17000A8150020F8B50E4607004FF000041FD0B8
:10B18000F9F736FC38460025F8F7AAFD0090C469A7
:10B190006846F8F7FBFD0EE0204600F041F8B042AB
:10B1A0000CD03146204604F076FD050005D120463E
:10B1B000F8F704FE046A002CEED12C46FAF7A8FB3F
:10B1C0002046F8BD10B5040007D0F9F711FC204661
:10B1D000F8F7F4FDC469FAF79BFB204610BD70B583
:10B1E00005004FF0000408D0F9F702FC2846F8F7F4
:10B1F000E5FD008D84B2FAF78BFB204670BD70B57B
:10B2000005460024F9F7F4FB35B12846F8F7D6FDDA
:10B2100090F8280000F00104FAF77AFB204670BD90
:10B220001FB50021019102910391152100916946FA
:10B2300000F058FB039804B010BD0000014602481E
:10B240000068806C00F002B8201400201FB5039144
:10B2500014210091694600F045FB1FBDF0B587B091
:10B260000C4607004AD0002C48D0FF21FFF782FF90
:10B270000546FE213846FFF77DFF064602A93846FF
:10B2800000F0BEF804A93846FFF7E0FFC6B16946F2
:10B29000304600F0B5F8BDF90A004242BDF9080099
:10B2A00041426846F9F78AFF3046FFF798FF0106EA
:10B2B00006D5800704D5BDF80000401EADF8140087
:10B2C000C5B16946284600F09BF8BDF90A00424224
:10B2D000BDF9080041426846F9F770FF2846FFF7BC
:10B2E0007EFFC10506D5800704D5BDF80200401ECB
:10B2F000ADF81600049820600598606007B0F0BDB6
:10B3000010B50446F9F774FB1CB12046F8F756FD5A
:10B31000046AFAF7FDFA204610BD000002480068F2
:10B32000806C00F04DB80000201400200248006836
:10B33000806C00F055B800002014002010B5040007
:10B3400007D0F9F755FB2046F8F738FD8469FAF77E
:10B35000DFFA204610BD70B50546FFF761FF0446D1
:10B36000FF2802D0FE2C02D002E0FE2400E0FF24E1
:10B370002846FFF7E3FF2146BDE87040FFF7FABE1D
:10B3800070B505004FF0000408D0F9F731FBFF213C
:10B39000284604F080FC0446FAF7BAFA204670BD4D
:10B3A00070B505004FF0000408D0F9F721FBFE212D
:10B3B000284604F070FC0446FAF7AAFA204670BD4D
:10B3C00070B505004FF0000408D0F9F711FB2846CE
:10B3D000F8F7F4FCB0F90040FAF79AFA204670BD8D
:10B3E00070B505004FF0000408D0F9F701FB2846BE
:10B3F000F8F7E4FCB0F90240FAF78AFA204670BD8B
:10B4000070B50C4605000ED0002C0CD0F9F7F0FA00
:10B410002846F8F7D3FC0168216040686060BDE809
:10B420007040FAF775BA70BD38B50446F9F7E0FA1E
:10B43000204604F049FBF8F753FC0090B0F90410E3
:10B44000B0F900000C1A6846641CF8F79FFCFAF784
:10B450005FFA204638BD38B50446F9F7C9FA2046E8
:10B4600004F032FBF8F73CFC0090B0F90610B0F99C
:10B4700002000C1A6846641CF8F788FCFAF748FAD0
:10B48000204638BD064A0549126851F8221081420B
:10B4900001D101207047002070470000B81500203E
:10B4A00070150020064A0549126851F822108142A1
:10B4B00001D101207047002070470000C015002016
:10B4C0007015002038B5040014D0F9F791FA204621
:10B4D000F8F706FC0090816A8A0706D521F0020180
:10B4E0008162026A816900F087FE6846F8F74EFCC7
:10B4F000FAF70EFA38BD00002DE9FF5F2D4D687890
:10B50000002855D12C496861A8630968DFF8ACA010
:10B5100004464864A88068804FF0040902274FF071
:10B52000FF3B43F6FF7805F148062046F8F75CFE3E
:10B53000A0B1CDF800B0CDF80C90CDE9017A002192
:10B54000424643460846FFF715FC1A4A46F82400CF
:10B5500050321B4942F8241000F07CF8641C022C85
:10B56000E3DB184FDFF86080DFF86090002400BF55
:10B5700007EBC40000F0CEFB08EBC40000F0CAFBF0
:10B5800009EBC40000F0C6FB641C022CF0DB306841
:10B5900000F086F9FFF75AFB012006496870403138
:10B5A0000B48086004B00846BDE8F05FFBF78AB8B6
:10B5B000BDE8FF9F60150020201400206D2C0108BD
:10B5C000785634FFF0500020005100201051002028
:10B5D000950F010870B586B00D46060031D0F9F719
:10B5E00007FA3046F8F77CFB0090846AA10723D560
:10B5F000D0E90010CDE90110E00302D5304600F09B
:10B6000081FD5DB1286803906868049003A90098E3
:10B6100000F088FB03A901A8FAF72FFF314601A823
:10B6200000F088FB40B140F601000440012C0AD034
:10B6300001A9304600F062FD6846F8F7A7FBFAF76B
:10B6400067F906B070BD0098026A816901A800F030
:10B65000D3FDF1E70021FFF7BDBFFEB515460E464D
:10B6600004001CD0F8F73CFB0246009090F828003C
:10B67000800711D5314601A8FAF71CFF60B1684672
:10B68000F8F784FB2A4601A9204604F0BDFE2046B7
:10B69000FFF798FD04460CE06846F8F777FBFEBD1F
:10B6A0002A4601A92046FFF7D8FF2046F8F786FB77
:10B6B000046A002CF4D1FEBD7FB506004FF00005F2
:10B6C00014D0F9F795F93046F8F778FB846AFAF761
:10B6D0001FF9A0070AD5E00608D4002003901F2018
:10B6E00000906946304600F0FDF8039D04B02846FE
:10B6F00070BD10B50446F9F77BF9204600F0A8FDAF
:10B700000446FAF705F9204610BD70B514460D46FB
:10B710000646F9F76DF922462946304600F0A8FDA5
:10B72000BDE87040FAF7F4B81FB5262203910092E5
:10B73000694600F0F3F81FBD70B586B00D460646A9
:10B740000024F9F755F90B490948096850F8210018
:10B7500048B10E210595009104A9CDE9031669466B
:10B7600000F000FF0124FAF7D3F806B0204670BDC0
:10B77000C01500207015002070B5154606468AB029
:10B780000C4651EA05006FD0002E6DD0F9F730F964
:10B790003046F8F7A5FA0590D0E90012CDE902127B
:10B7A000CDE906127CB1816A0A0607D5890505D460
:10B7B000BDF81810091BADF8181004E0BDF81C10F6
:10B7C0002144ADF81C107DB1816ACA0507D5490531
:10B7D00005D4BDF81A10491BADF81A1004E0BDF8E5
:10B7E0001E102944ADF81E10806AC00302D53046F1
:10B7F00000F088FC05AB93E80700C0E9001290F860
:10B80000280080070AD506AA02A908A8F9F7AAFC09
:10B810000598026A816908A800F0EEFCBDF91E00D7
:10B82000BDF90E10401A0090BDF91C00BDF90C10B6
:10B83000431ABDF91A00BDF90A10421ABDF91800E1
:10B84000BDF90810411A059800F0CCFE059901F1E8
:10B850000800FAF712FE0521304600F0B4FE05A8F4
:10B86000F8F794FAFAF754F80AB070BD38B50C46F8
:10B87000050013D0F9F7BCF82846F8F731FA009024
:10B880001CB100682146F9F7DAFE00980068F9F764
:10B89000BAFE6846F8F77AFAFAF73AF838BD0000C7
:10B8A00070B50446F9F7A4F80C4D2868866C0CB9FD
:10B8B0000B494C698464204600F04AFEFDF77EFC8B
:10B8C0002046F8F77BFA2968B0F90020CA64B0F97D
:10B8D00002000865FAF71CF8304670BD20140020FD
:10B8E0006015002070B50D46040009D0F9F780F806
:10B8F0002946204600F036FEBDE87040FAF708B849
:10B9000070BD70B50C460546F9F772F82146284619
:10B9100000F046FEBDE87040F9F7FABF70B50C00C4
:10B9200005460DD0F9F764F82846FFF707FD18B172
:10B930002146A56000F016FEBDE87040F9F7E8BFAB
:10B9400070BD00002DE9F0410D460446F9F750F8AE
:10B95000094F084E386856F82000A04201D000F088
:10B96000B7FD386846F8204004480570BDE8F0414E
:10B97000F9F7CEBFB815002070150020C8150020BB
:10B980002DE9FF471D4616460C468146FFF77AFD16
:10B99000DFF8908090B3B8F900102068471AB8F922
:10B9A00002106068441A56EA050033D069464846DA
:10B9B000FFF726FD2DB1BDF802006D1E2844ADF83D
:10B9C00006004846FFF7BAFC02A9FFF719FD224618
:10B9D00039466846F9F7F2FB02A932460846FAF7FB
:10B9E00063FE02A96846F9F743FC002804D022460A
:10B9F00039464846FFF789FEBDE8FF87FFE701218A
:10BA00004846FFF79FFF2088A8F80000A088A8F804
:10BA10000200F1E704B0224639464846BDE8F04747
:10BA2000FFF773BEF416002010B5F7F797FC024934
:10BA300000200968486410BD20140020F0B587B0CC
:10BA4000002604460296039604960596F8F7D0FF62
:10BA50008CB3234D214F286857F82000A04236D0E0
:10BA60000596CDE900041E21029110B102A900F053
:10BA700079FD0120059002A9204600F073FD05998B
:10BA800020266846002902D1296847F82140059FF1
:10BA90001ED105462046FFF751FC040005D002A93F
:10BAA0000296059500F05EFDF4E7009C2046FFF746
:10BAB00020FE30B90CE00AE002A90296059500F0DC
:10BAC00051FD2046FFF73AFC0400F5D100E00127C4
:10BAD000F9F71EFF07B03846F0BD0000C015002082
:10BAE0007015002070B505004FF0000427D0F8F75E
:10BAF0007FFF2E46284600F0CBF90146304604F081
:10BB00004DF905462C4606E02146304604F046F93C
:10BB10000446A84202D0FFF7CFFD90B164B10A4DB0
:10BB200020462E6800F006FA411C06D02860204608
:10BB3000FFF784FF2E6000B10024F9F7E9FE2046EC
:10BB400070BD002CE0D1F7E77015002070B505003E
:10BB50004FF000041BD0F8F74BFF284600F098F98F
:10BB600004F094F905462C4605E0204604F08EF9D1
:10BB70000446A84204D0FFF79FFD08B9002CF4D179
:10BB80002046FFF75BFF00B10024F9F7C1FE204615
:10BB900070BD000038B50446F8F72AFFCCB1204646
:10BBA000F8F79EF8009090F82800C0070ED12046C4
:10BBB00000F070F80098816A41F001018162064846
:10BBC0000168491C01602046FFF744FD6846F8F70C
:10BBD000DDF8F9F79DFE38BD881500201FB5002857
:10BBE00007D0002905D02422039100926946FFF76F
:10BBF00079FE1FBD70B50C460546F8F7F9FE2146E3
:10BC0000284600F0E7FC0446F9F782FE204670BDA6
:10BC100070B50C460546F8F7EBFE2146284600F0C5
:10BC2000DDFC0446F9F774FE204670BDF8B51646F3
:10BC30000C4605001DD0F8F7DBFE2846F8F750F853
:10BC40000090B0F90410B0F90020891A641AB0F914
:10BC50000610B0F90200641E081A361A6846761EED
:10BC6000F8F794F8324621462846FFF785FDF9F7A4
:10BC70004FFEF8BD70B50546F8F7BAFE04480068F7
:10BC8000446C456400F022F8F9F742FE204670BD8E
:10BC90002014002038B50446F8F7AAFE84B12046E7
:10BCA000F8F71EF80090816A8A0606D521F0200177
:10BCB000816205490888401E08806846F8F766F8E2
:10BCC000F9F726FE38BD0000641500200EB50E48B9
:10BCD000006890F8541009B10C4811E0806CF7F737
:10BCE000FFFF0090D0E90010CDE901106846F8F799
:10BCF0004DF80748C16A11B101A800F01BF801A86E
:10BD000005F0DEFF0EBD0000201400207050002062
:10BD10006015002002490A68026008607047000050
:10BD2000781500200B46B0F90220B0F90010184633
:10BD3000F9F744BA38B50C4605462046F7F7D0FF68
:10BD40000146009090F82800800703D46846F8F771
:10BD50001DF812E02846FAF790FB0098806920B1A0
:10BD600004466846F8F712F8E7E76846F8F70EF871
:10BD7000204601F0B1FA002801DA002038BD012088
:10BD800038BDF8B50546F8F733FE6846F9F768FCA4
:10BD90001AE001212046F9F71DFC009981B178B124
:10BDA0000846F8F70BF84068A84209D169462046D2
:10BDB000009EF9F769FC04463046FFF7B7F804E047
:10BDC00069462046F9F760FC0446002CE1D1F9F7FA
:10BDD0009FFDF8BD10B5F7F7F1FF816A41F400410E
:10BDE000816202490120C86310BD00006015002077
:10BDF00038B50446F7F774FF0090816941B1026AD3
:10BE000000F0FAF9204600F079FB009900208861E3
:10BE10006846F7F7BBFF38BD70B516460D46F7F715
:10BE2000CDFFC4690BE031462046A847324629467B
:10BE30002046FFF7F1FF2046F7F7C0FF046A002C09
:10BE4000F1D170BD38B50C4600280AD0002C08D0BE
:10BE5000F7F746FF2146009000F004F86846F7F730
:10BE600095FF38BD00224A800A8082880388D21A52
:10BE70008A80C2884088101AC880704710B5FFF7C2
:10BE80005DFA002802D0F7F799FFC06910BD0000E5
:10BE900070B5084E0146064D3068002455F8200064
:10BEA00000F0C5F910B1306855F82040204670BD4B
:10BEB000C01500207015002010B5040006D000BF8A
:10BEC000F7F77CFF006A08B10446F9E7204610BD89
:10BED0000D4810B5006890F85400002806D00B4CAF
:10BEE0006069012803DD401E6061002010BD2069EB
:10BEF000401C206103F02AFC18B1FFF7E7FE012087
:10BF000010BD6069EFE70000201400206850002099
:10BF100070B50546FFF7B2FF08E0AC4201D100243E
:10BF200006E0F7F74BFF006AA84201D00400F4D105
:10BF3000204670BD10B50446F7F740FF8069002821
:10BF4000F9D12046BDE8104001F0C6B9B0F904109F
:10BF5000B0F90000081A401C7047B0F90610B0F99B
:10BF60000200081A401C7047F0B5384E074687B0EB
:10BF7000306890F8541041B1354C6169491C6161D9
:10BF8000012905DD012007B0F0BDFFF79FFEF9E7AD
:10BF9000806CF7F7A5FE2F4D4FF0FF310090216127
:10BFA000297821B181680291C068039007E090F878
:10BFB000281089073CD5D0E90010CDE902101FB147
:10BFC000394602A8FAF759FA3068406C78B30098FD
:10BFD00004903068406C0168059140680690E86AFA
:10BFE00030B104A8F7F7D2FEE86AF7F779FE0490BB
:10BFF00005A90498FFF796FE05A902A8FAF73DFAED
:10C000000DF11000F7F7C2FEE96A19B102A8FFF7B7
:10C0100091FEB0B13068816C02A8FFF78BFE80B151
:10C02000DDE90201C4E90001FFF752FFABE706E0DA
:10C030006069401E60616846F7F7A8FE04E0684644
:10C04000E0E76069401E606100209CE7201400204A
:10C050006850002060150020FEB50D00044647D052
:10C06000F7F73EFE00900021856101622846F7F750
:10C0700037FE00990290C56991F8281001F0080672
:10C080002DB12846F7F72CFE019036B115E0C461BA
:10C090006846F7F77BFE02A828E090F82800000722
:10C0A0000BD5009805620298C4616846F7F76EFEEA
:10C0B00002A8F7F76BFE01A818E002A8F7F766FEE2
:10C0C00001A8F7F763FE2846F7F778FE11E004624F
:10C0D0000BE02846F7F772FE5EB990F828100907C2
:10C0E00007D501980462009805626846F7F74EFE8E
:10C0F000FEBD0190056A002DEBD1E8E7202204F097
:10C1000083B9000038B5040022D0F7F7E9FD0090AC
:10C1100090F82810890718D5406A40B10D49096B7D
:10C12000A14204D0F8F76EFD009900204862204635
:10C13000FFF748F8044606E02046FFF7E3FF2046F5
:10C14000F7F73CFE046A002CF6D16846F7F71EFEAE
:10C1500038BD00006015002070B5064615460C4637
:10C160000846F7F72BFE806AC00302D54FF48043E0
:10C1700000E020232A4621463046BDE87040AFF358
:10C1800000802DE9FF419846164607460D0031D044
:10C190000846F7F7A5FD0090846A0246A00726D559
:10C1A000394601A8FAF786F908B340F601000440C1
:10C1B000012C07D0424601A9284604F025F9009831
:10C1C000C46912E000984346026A816901A8FFF73A
:10C1D000D8FFF4E7B4420AD0424601A92046FFF74F
:10C1E0003CFA2046F7F7EAFD046A002CF2D16846D3
:10C1F000F7F7CCFDBDE8FF812023FFF7C2BF0000A9
:10C2000070B50C46002550B14CB100BFF7F7D6FD14
:10C210008069A04201D1012501E00028F6D128461D
:10C2200070BD884201D101207047FFF7E9BF38B5E2
:10C230000D46002450B1F7F753FD009018B1806906
:10C24000A84200D101246846F7F7A0FD204638BD7A
:10C2500010B5044605484069002802D0A04201D12B
:10C26000012010BDF7F7AAFDF5E7000060150020DA
:10C27000F0B58BB006004FF0000015460C46049058
:10C280000590069007903ED054EA05003BD030461A
:10C29000F7F726FD0090D0E90012CDE902122A46F8
:10C2A0002146F8F78BFF00982A4621460830F8F718
:10C2B00085FF0098C7696846F7F768FD2A4621465A
:10C2C000384604F05FFD3046F7F70AFD009090F81D
:10C2D000281089070AD5816941B1026AFFF73CFF3E
:10C2E0000098026A816902A8FFF736FF6846F7F7EF
:10C2F0004DFD0320049007AA08A882E8310004A994
:10C30000304600F02FF90BB0F0BD00002DE9F141EF
:10C3100087B000250798F7F7E3FC0190D0E90212F7
:10C32000CDE9031207698669846A01A8F7F72EFD33
:10C3300044F2200814EA080F30D0DFB103A80799AF
:10C34000FFF7F8FCB0B10798FFF7AAFA60070DD520
:10C3500056B144F30000401C0090002307AA114985
:10C3600003A8F8F773FC05E00120F5E7079800F053
:10C3700063F801250798F7F7B3FC0190816A21EA79
:10C38000080181628A0402D541F00401816201A89A
:10C39000F7F7FCFC04498888401E888008B02846CE
:10C3A000BDE8F081C12C010860150020F0B589B00E
:10C3B0000546F7F795FC0290866A0469D0E90210F9
:10C3C000CDE9001002A8F7F7E1FC002C30D0B0074F
:10C3D0002ED52E212846FFF794FA164C6F4620786A
:10C3E000401C2070F0044FF00F0609D5CDE904651C
:10C3F0000797FFF719FB04A9284600F0B3F810E0EF
:10C400003846FFF7B1FD0AE0CDE904650797FFF76D
:10C410000BFB04A9284600F0A5F8FFF759FD0028FA
:10C42000F2D120782F21401E20702846FFF769FAAC
:10C4300009B0F0BD6015002038B50446F7F750FC90
:10C440000090806A40F601010840012805D0684646
:10C45000F7F79CFC204605F04FFA1448806A002844
:10C4600023D0204605F0A0FA2046F7F7A7FC8569FF
:10C47000046A18E02046F7F7A1FC90F82800C043B2
:10C48000800702D1204605F049FA204605F08CFAD3
:10C490002046F7F793FC046A002CEBD12846F7F707
:10C4A0008DFC8569046A002DF6D138BD6015002029
:10C4B000B0F90010B0F90420914205DCB0F9021087
:10C4C000B0F90600814201DD00207047012070476D
:10C4D0007FB5094D074C286854F82000002808D083
:10C4E00018210091694600F03DF82968002044F8C1
:10C4F00021007FBDB81500207015002070B50646DC
:10C50000F7F75CFC05468069002809D0F7F756FC70
:10C510000446C069B0420ED1F7F750FC006AE061F2
:10C5200070BD00BFF7F74AFC0146006AB04202D175
:10C53000286A086270BD0028F4D170BD0B46B0F9BE
:10C540000210B0F900004A4241421846F8F736BEE0
:10C5500010B5FFF7EFFC002803DBBDE81040F8F74B
:10C56000C1BE10BD70B50D4C06460D46206814289E
:10C570000DDA3046F7F722FC01696E6041B12068A0
:10C58000401C2060284688472068401E206070BDFF
:10C590002846BDE87040FEF7A5BC0000F01600205C
:10C5A0007FB50546002000900190029003900C4654
:10C5B0002846F7F703FC0269002A03D06846CDE954
:10C5C000004590477FBD1FB5CDE900106946FFF7D4
:10C5D000C9FF1FBD0023FF2205F049BD0823FE222D
:10C5E00005F045BD2DE9FF4F81B09B46C66962E06D
:10C5F0003046F7F775FB01460090D1E90004896ADF
:10C60000254601F420730246802B09D0B3F5207F24
:10C61000029B134406D063F30F02029B234405E000
:10C6200002EB0B0363F30F0204EB0B0301F4A061B5
:10C6300063F30F04B1F5807F0BD0B1F5A06F0399C0
:10C640004FEA224307D0194461F31F422314039990
:10C6500006E00E991314194461F31F420E99231436
:10C6600019440FFA82FA61F31F440FFA80F9171484
:10C670004FEA2048AAEB0901A7EB080251EA0200A1
:10C6800002D03046FFF741F82AB221B2A2EB0900EE
:10C69000A1EB0A01091AC7EB2440C8EB2542821A14
:10C6A00051EA020002D03046FFF766F80098066AA9
:10C6B0006846F7F76BFB002E9AD105B0BDE8F08F06
:10C6C00030B50C4B1A680C2A12DA00210A4C002AE9
:10C6D0000ADD114604EB410535F9025C854203DBB6
:10C6E00024F81150491EF5D124F81100521C1A608B
:10C6F00030BD0000F8160020205100202DE9F04147
:10C70000214D0C460646E968A86B0844A119401E55
:10C71000814206D80846096819B941680E4405F0F7
:10C72000DDF9A86BA0420AD254F8040C271A386825
:10C7300028B978680644384605F0D0F93C463046BA
:10C7400003F01EFB10281CD205EBC0073246002167
:10C7500020467B6C05F06EFD57F8440F083400B19D
:10C7600044602060002060603C602868304428609D
:10C7700095F8291029B9E968081AA968814200D2F8
:10C78000A8603046BDE8F081284F00202DE9F04137
:10C79000054603F0E1FD2A48046CAC4202D8ED1CCA
:10C7A00025F00304804600680C34A04202D2002029
:10C7B000BDE8F08105F046F9071EF9D0204603F0E8
:10C7C000DFFA414630E000BF01EBC002526C52B3C9
:10C7D000956845B36B68A34206D2AA681AB39568F8
:10C7E0000DB36B68A342F8D3D8F84000191B0C3086
:10C7F0001E46814200D23446284605F06FF90421D6
:10C80000D8F8340001EBC7010023455022463946D1
:10C81000284605F00FFDA64203DD2919301BFFF75E
:10C820006DFF3846C4E7401C1028CDD3204605F0E4
:10C830009DF90028C2D0384605F024F9B7E700007A
:10C84000284F00207CB5040016D0F7F749FA009075
:10C85000016A91B190F82800000713D40846F7F751
:10C860003FFA019090F82800000708D56846F7F7CE
:10C870008DFA01A8F7F78AFA7CBD6846FAE701A8A5
:10C88000F7F784FA009885696846F7F77FFA20463B
:10C89000FFF734FE29462046FFF7DEFB2046FEF771
:10C8A000D9FE002202492046FEF71EFC7CBD000096
:10C8B000BD2C01082DE9F04391B00D460746F7F76E
:10C8C0000FFA0290D0E90012CDE9031290F832106D
:10C8D000BDF90C40BDF90E60090702D5BDF9121073
:10C8E00001E0BDF91010A96190F83210C1F3C00148
:10C8F0000E91016C19200994CDE90570BDF90E0067
:10C900000A90BDF910000B90BDF912000C900EA812
:10C910000D9005A8884780460298018EFF2911D105
:10C920008069FEF73DFD68B16946FEF769FDBDF916
:10C930001000BDF90410884204D1BDF80000401E6B
:10C94000ADF810000298018EFE2911D18069FEF722
:10C9500017FD68B16946FEF753FDBDF91200BDF938
:10C960000610884204D1BDF80200401EADF8120046
:10C970007242614203A8F8F721FC03A90298FDF76F
:10C9800033FFBDF91010BDF90C2002988F1AC8F1C1
:10C9900000017F1CD0F84C9007EB4106406D4946E2
:10C9A0007043F9F7C5FA04461648B0F90010881C20
:10C9B000844200DA8C1CB44200DD3446BDF90C0020
:10C9C0002860A8F101006860781E6861A7EB080084
:10C9D00028610298361B426D006DA9EB020170437D
:10C9E000F9F7A6FA6968401C0844611EA86008446B
:10C9F000E860C5E9076402A8F7F7C8F911B0BDE817
:10CA0000F0830000E816002001207047F0B40F4CBE
:10CA1000246814B1A446F0BC60470D4DDFF834C063
:10CA200010C855FA84F63778C4F30726C4F30744D0
:10CA30001CF806602C5D521E04EB461404EBC72460
:10CA40000C801944ECD1F0BC70470000B4140020F5
:10CA5000184801081849010810B510C80C6019449D
:10CA6000521EFAD110BD00002DE9F047DFF83490D6
:10CA7000DFF834A09846174605460C4640CDD9F855
:10CA8000001026F07F4088470AEB16617F1E097868
:10CA9000C1F10F0140EA011020704444EED1BDE81D
:10CAA000F087000090460108184701082DE9F0477B
:10CAB000DFF82C909846164605460C464FF47F4A00
:10CAC00080CDD9F8001027F07F40884701462AEA38
:10CAD0001740084320804444761EF1D1BDE8F0871A
:10CAE000503201082DE9F041114C24681CB1A446D4
:10CAF000BDE8F04160470F4D4FF0010E10C855FAE8
:10CB000084F696F800C0C4F30726521EAF5DC4F346
:10CB100007468EEAD474AE5D06EB471606EB8C260C
:10CB200006EBC4340C801944E8D1BDE8F081000064
:10CB3000C01300201848010838B50324009400F001
:10CB4000AFFA38BD2DE9F041154C24681CB1A4465C
:10CB5000BDE8F04160474FF0FF0E112440C8F7B226
:10CB6000C6F3072CC6F30745AEEB16660836083742
:10CB7000B6FBF4F6B7FBF4F70CF1080C0835BCFB78
:10CB8000F4FCB5FBF4F5360306EB072606EB0C16B2
:10CB900035440D801944521EE0D1BDE8F0810000FB
:10CBA000C813002038B50424009400F079FA38BD89
:10CBB00038B50024009400F073FA38BD38B500246D
:10CBC000009400F06DFA38BD2DE9F0478146FCF77E
:10CBD00039F84FF0000807466FF07F444546FCF7F0
:10CBE00049F8060018D000BF56F82510494502D173
:10CBF0002846BDE8F0876D1CBD42F5DB5FF00005FF
:10CC0000484656F82510F7F7D3F9A04201D204465A
:10CC1000A8466D1CBD42F3DB4046EAE7F0B5C4B25E
:10CC2000C0F30725611CC0F30740552901D301213A
:10CC300000E000216A1C552A01D3012200E00022F5
:10CC4000431C552B01D3012300E000234FF0FF3C90
:10CC50000CEB02272F400CEB03250CEB01260540C3
:10CC600026408818C418480000EB8200114300EBEE
:10CC7000C30019430AD0F1192944C4EB84121144AA
:10CC8000C4EBC412B1FBF2F100EB5100F0BD0000A7
:10CC900010B50749044620F07F40096888470549D8
:10CCA00001EB14610978C1F10F0140EA011010BDD8
:10CCB000904601081847010810B50649044620F0BF
:10CCC0007F40096888474FF47F4121EA14410843B7
:10CCD00010BD0000503201087047000010B50A492D
:10CCE00051FA80F21378C0F30722C0F307448A5C3C
:10CCF000095D012401EB421184EAD07001EB83212C
:10CD000001EBC03010BD00001848010810B5C3B2D7
:10CD1000C0F30721C0F30742FF24A4EB10641120E5
:10CD2000083308310832B3FBF0F3B1FBF0F1B2FB8A
:10CD3000F0F20834B4FBF0F0000300EB032000EB4A
:10CD40000110104410BD000010B5084A52FA80F1DD
:10CD5000074BC0F30724C0F307401B5D105C097844
:10CD600000EB431000EBC12010BD00001848010883
:10CD7000184901082DE9F05F9A46DDE90A879146D6
:10CD80000C4605468B46164635F8020B4146884749
:10CD9000B84701C4761EF7D15046BAF1200F06D22B
:10CDA000024649465846BDE8F05FF8F70DBEBDE8BB
:10CDB000F09F2DE9F05F9A46DDE90A8791460C461F
:10CDC00005468B46164615F8010B41468847B8477D
:10CDD00001C4761EF7D15046BAF1200F06D20246A2
:10CDE00049465846BDE8F05FF8F7EEBDBDE8F09F54
:10CDF0002DE9F04116460F46804603F0F3FAD8F8C5
:10CE00000840002C25D0B74223D0D8F80C000821C8
:10CE1000826A40469047D4E9052151434143A068C6
:10CE2000CA0820B150F8271050F8265004E0606876
:10CE300002FB070102FB0605A36B2BB13246394604
:10CE4000D8F81800984703E0034B28461B6898471A
:10CE50002560BDE8F0810000E815002030B58BB0FA
:10CE60000446F6F73DFF0090C06D85686846F6F70A
:10CE70008DFF0020CDE90140696801A888470BB00B
:10CE800030BD30B58BB00446F6F72AFF0090406EF7
:10CE900085686846F6F77AFF0020CDE901402968E9
:10CEA00001A888470BB030BD30B58DB00446F6F709
:10CEB00017FF009090F83210056CC1F3C0010B9180
:10CEC000064981646846F6F761FF0020CDE902401B
:10CED0000BA80A9002A8A8470DB030BDB5C800083D
:10CEE0002DE9F04786B08246F6F7FAFE0390D0E9C6
:10CEF0000075D0F8249003A8F6F748FF29B20FFA7E
:10CF000087F83E14A1EB0804C6EB2545641C6D1C94
:10CF1000002C01DD002D03DC002006B0BDE8F08709
:10CF2000B9F1000014D0F6F7DBFE0490B0F904402C
:10CF3000B0F9065004A8F6F729FF38B2A04201D193
:10CF4000AE425BD0324641464846F7F7C7FF55E050
:10CF5000FEF704F9824513D1FBF7C2FE0746FBF743
:10CF6000D3FEBC4201DC85420ADDBC4200DD3C460A
:10CF7000854200DD05462A4621465046FEF756FE0C
:10CF8000254A264901208DE80700314640462B46B8
:10CF90002246F8F70FF806465046F6F7A1FE039032
:10CFA000466286B3816A41F48031816203A8F6F754
:10CFB000EDFE3046F7F76AFF07460120F8F7F2FC6E
:10CFC0003046F7F708FF174B15496C431B68A20062
:10CFD00009789847144E154C5046C6F800A02568AD
:10CFE000FEF7EEF920605046FFF7E0F900202560DB
:10CFF0003060F8F7D7FC3846F7F748FF5046F6F7A9
:10D00000DDFE406A89E7FFE703A8F6F7BFFE50465A
:10D01000FFF7CCF980E7000084540108DC5C0108CC
:10D020002C160020E4150020901500207414002018
:10D030002DE9F0410F4615461E460B4C32466168FD
:10D0400003F05EFAA1683246384603F059FAA16847
:10D050003346D4E9002000F009F82068324629461A
:10D06000BDE8F04103F04CBA9413002030B40B4CEF
:10D07000094D2560E0606161E26300202061A061EC
:10D080002064E06160626063012000EB0340606443
:10D0900030BC00F067B800000002020000B002409F
:10D0A000F8B50E461446069F2246064D296803F041
:10D0B0002EFA0094002228683B46314600F004F81E
:10D0C000F8BD000094130020F0B4049D4FF48136A5
:10D0D000074C2660E060E163002020612064E2618B
:10D0E0006363012000EB05406064F0BC00F03AB8D7
:10D0F00000B002402DE9F0470D4616461F46DDF808
:10D100002080DDE9099A02F07FFE094C4FF400719E
:10D110002160E560E663C4F81090C4F840A0E061C7
:10D1200067F31F48C4F84480BDE8F04700F01AB820
:10D1300000B00240F0B404ADE0CD094C4FF4813CA6
:10D14000C4F800C0E060E163226123640520E0616F
:10D15000656347EA06406064F0BC00F003B8000075
:10D1600000B002400548016841F00101016000E0A3
:10D1700030BF0168C907FBD17047000000B0024012
:10D180002DE9F047884617461D46DDE9089602F06E
:10D190003BFE094C07492160A663C4F83C80C4F8F3
:10D1A0004090606367F31F456564BDE8F047FFF793
:10D1B000D9BF00000002030000B00240F8B51446D9
:10D1C0000E46069A0023064D00942968FFF77CFF5F
:10D1D000286822463146BDE8F84003F098B90000BF
:10D1E00094130020064AD062491EC8B2012101EB07
:10D1F0000020D061D06940F02000D061704700006D
:10D2000000B0024030B5164C80F07F406368186073
:10D2100081F07F40A16808601348124D0560C3602B
:10D2200041612168C1634FF4803141EA0261C1610B
:10D23000C2F1FF0109064162002141634FF0011173
:10D240004164016841F00101016000E030BF016804
:10D25000C907FBD12068006880F07F4030BD000026
:10D26000941300200002020000B00240F0B4049DBC
:10D270000C4C0B4E2660E0606161E2634FF480303D
:10D2800040EA0360E061C3F1FF0000066062002035
:10D290006063012000EB05406064F0BCFFF762BFF3
:10D2A0000002020000B0024010B50446E069FDF73C
:10D2B00053FEE0690028F9D110BD08B5F6F710FD5E
:10D2C0000090406EFDF732FE009900204866C86568
:10D2D0006846F6F75BFD08BD0146064A002000BF20
:10D2E00052F820308B4204D0401C0228F8DB4FF06B
:10D2F000FF307047A8150020F7B515461E4A01A952
:10D300000098126890471D4C00902068406920B139
:10D310002946F7F7ADFF00282DD00120F9F7F4F8E2
:10D320002068174DC1694969F1B1164D2A684AB1A3
:10D33000B0F922408A68DDE900019047296820465B
:10D34000884715E08A68DDE90001904710E06846EB
:10D35000F8F7B6F906462068C06901683046884784
:10D36000296809B1304688470198401E0190EED5E2
:10D370000020F9F7C9F8FEBDEC15002020140020AC
:10D38000681400206C1400202DE9FC47D0F8209090
:10D3900005468269C369D5E90407D9F804C03A4C47
:10D3A00099B3111A491C4E102168BCF1000F26D008
:10D3B000D1E9002C00214FF0010800BFCDE9002C7D
:10D3C0008219A3EB08033944401CF6F7FBFFD9F898
:10D3D00004000028206819D0D0E902230021012090
:10D3E000CDE90023EA69761C131AD5E90502014448
:10D3F0002869521E3044F6F7E5FFBDE8FC87D1E905
:10D40000042C01214FF00008D8E704E0D0E90623FE
:10D4100001210020E4E7D91B491C4E102168BCF112
:10D42000000F25D0D1E904384FF0000C5FF0010166
:10D43000CDE90038521ABB19791C6044F6F7FEFF9B
:10D44000D9F804000028206818D0D0E9061300207D
:10D450005FF00102CDE90013D5E906138A1A696964
:10D460002C69761C314420445B1EF6F7E7FFC4E7C5
:10D47000D1E900384FF0010C0021D9E7D0E90213BF
:10D4800001200022E6E70000645401087CB50D4647
:10D49000044601F06CFAD5E90301CDE90001B4F9C5
:10D4A0000210B4F90600B4F9042008444310B4F99A
:10D4B0000000891C801C921EF6F7C0FFD5E905010B
:10D4C000CDE90001B4F90200B4F906300121184495
:10D4D00001EB6001B4F90420B4F90000921E801C35
:10D4E0009B1EF6F7ABFF7CBD7CB50D46044601F0F4
:10D4F0003EFAD5E90301CDE90001B4F90000B4F921
:10D500000410B4F9063001444A10B4F90210801C2A
:10D51000891C9B1EF6F756FFD5E90501CDE90001F0
:10D52000B4F90000B4F904200121104401EB6000BB
:10D53000B4F90630B4F90210921E891C9B1EF6F74E
:10D5400041FF7CBD2DE9F05FD0F808A0DDF8288010
:10D550009946DAF82040414402FB04163549DDE9DA
:10D560000B7399F80020DFF8C8B00968D3E900C34D
:10D570001BF80240097CC8F1080524FA08F411F0F0
:10D58000030118D0012903D0022935D0032931D154
:10D590000069806880475B46E10706D0DAF8002022
:10D5A00032F81610414022F8161064086D1E06F17C
:10D5B000010635D038E0BD4201D2284600E03846A9
:10D5C0000146E20701D01A4600E06246DAF8008020
:10D5D0006408401E28F8162006F10106F1D16D1AE4
:10D5E000A7EB010704D119F8011F08251BF801401A
:10D5F000002FE0D1BDE8F09F99B25846E20703D072
:10D60000DAF8002022F8161064086D1E06F10106F3
:10D6100003D119F8012F0825845C7F1EEED1E9E7BC
:10D6200019F8011F08255C5C7F1EB5D1E2E70000F8
:10D63000844A0108201400202DE9FF5F9046DDE9AF
:10D640000E924D4B99F80050C2F108048A465D5D78
:10D65000DDE91071D540494A139E1268127C12F020
:10D66000030226D0012A03D0022A37D0032A72D11E
:10D670000069806880471FFA80FBBC4200D93C46A5
:10D680003F1BBAF1000F68D0E8070AD0DAF80800AB
:10D690004146039A036850469847318881EA0B0156
:10D6A00031806D0808F10108641E06F10206EBD115
:10D6B0005EE0314ABC4200D93C463F1B05F0010008
:10D6C0006D0831F8200026F8020B641EF6D1002FF9
:10D6D00050D019F8010F0824155CEBE788881FFA71
:10D6E00080FBBC4200D93C463F1BBAF1000F17D06B
:10D6F00095B1E80708D0DAF808004146039A0368B4
:10D7000050469847A6F800B008F10108641E06F1DB
:10D71000020612D06D08EBE706EB4406A0440CE0CD
:10D720004DB1E80701D0A6F800B0641E06F102066C
:10D7300003D06D08F4E706EB4406002F1AD019F861
:10D74000011F0D480824455CCBE719F8011F0A4862
:10D750000824455C91E70DE0FFE7E80703D0308837
:10D7600080EA0B0030806D08641E06F10206F4D1D9
:10D77000002FEAD1BDE8FF9F844A01082014002051
:10D780002DE9FF4F81B08A46DDF8388011ACDFF813
:10D7900004B198F800509146DDE90F1794E8450070
:10D7A0001BF80550C1F10804CD403B495B460968B0
:10D7B000097C11F003011FD0012903D0022930D0C8
:10D7C000032964D110680069806880475946BC42CB
:10D7D00000D93C463F1BEA0702D032684240326023
:10D7E0006D08641E06F10406F5D1002F4FD018F81D
:10D7F000012F08248D5CEAE71946BC4200D93C465B
:10D80000B7EB040705F001026D0850F82220641EF2
:10D8100004C6F7D1002F3AD018F8012F08248D5CE8
:10D82000EBE740680090BC4200D93C463F1BBAF190
:10D83000000F17D095B1E80708D0DAF8080049467C
:10D84000049A0368504698470098306009F101092E
:10D85000641E06F1040612D06D08EBE706EB8406A1
:10D86000A1440CE04DB1E80701D000983060641E7F
:10D8700006F1040603D06D08F4E706EB8406002FDA
:10D8800005D018F8011F08241BF80150CBE705B09C
:10D89000BDE8F08F844A0108201400202DE9FF5FC5
:10D8A000424893460EAA006892E89002007C0D1947
:10D8B0001E7810F0030198464FF0C0001CD00229DA
:10D8C00037D15FEA090155D04FEA000AC4F10300DD
:10D8D0004100C1F106022AFA02F03040C84006D0E9
:10D8E00059F820305A462946009804F0F4FA641C8E
:10D8F0006D1C042C38D03AE05FEA09011BD0824647
:10D90000C4F103004100C1F106022AFA02F03040DE
:10D91000C840294659F820306D1C5A46009804F03A
:10D92000DAFA641C042C02D118F8016F00247F1E5F
:10D93000E6D1BDE8FF9F8146C4F103004000C0F17D
:10D94000060129FA01F33340C34029466D1C5A46AB
:10D95000009804F0C0FA641C042C02D118F8016F7E
:10D9600000247F1EE8D1E4E718F8016F00247F1E31
:10D97000ACD1DEE74FEA0009C4F103004000C0F17A
:10D98000060129FA01F33340C34004D05A46294620
:10D99000009804F0A0FA641C6D1C042C02D118F845
:10D9A000016F00247F1EE7D1C3E700002014002090
:10D9B0002DE9FF5F8B460FA9DDF8388091E821043F
:10D9C000C0F10401CCB298F80010400081402F480B
:10D9D000129F91460068CEB2007C10F0030004D084
:10D9E00001283AD002284FD114E0AC4200DDECB25D
:10D9F0002D1BB1093AF8210027F8020BB006060EDC
:10DA0000641E14F0FF04F4D1002D3DD0042418F856
:10DA1000016FEAE7AC4200DDECB22D1BB0090DD07E
:10DA2000B109BBF1000F3AF82100388006D0DBF8CD
:10DA300008004946039A036858469847B006060E00
:10DA4000641EBF1C09F1010914F0FF04E6D1002D8A
:10DA50001AD0042418F8016FDCE7AC4200DDECB208
:10DA60002D1BB00903D0388880F0FF003880B00645
:10DA7000060E641EBF1C14F0FF04F2D1002D03D06B
:10DA8000042418F8016FE8E7BDE8FF9F2014002088
:10DA90002DE9FF5F8B460FA9DDF8388091E821045E
:10DAA000C0F10401CCB298F80010400081402F482A
:10DAB000129F91460068CEB2007C10F0030004D0A3
:10DAC000012839D002284ED113E0AC4200DDECB27F
:10DAD0002D1BB1095AF8210001C7B006060E641EBD
:10DAE00014F0FF04F5D1002D3DD0042418F8016F87
:10DAF000EBE7AC4200DDECB22D1BB0090DD0B10953
:10DB0000BBF1000F5AF82100386006D0DBF808009E
:10DB10004946039A036858469847B006060E641EA5
:10DB20003F1D09F1010914F0FF04E6D1002D1AD0C0
:10DB3000042418F8016FDCE7AC4200DDECB22D1BC9
:10DB4000B00903D0386880F0FF003860B006060ED8
:10DB5000641E3F1D14F0FF04F2D1002D03D00424F5
:10DB600018F8016FE8E7BDE8FF9F000020140020CF
:10DB70002DE9F0479946DDE908540A9F92465FEA8D
:10DB80000108064608D0D8F8080023464A46D0F8CF
:10DB900004C051464046E0473069DFF88090C168D4
:10DBA00039B1A20029463846D9F80030BDE8F0471F
:10DBB00018474168002088474FEA106828462146E8
:10DBC0004246002608C81B0E934201D106F1010609
:10DBD000A1F1010101D10029F4D166B1D9F80030D9
:10DBE0004FEA860229463846984707EB860705EB39
:10DBF0008605A41B0DE02868010EFF2906D2084BFC
:10DC0000C1F1FF0239681B6898473860641E2D1DFA
:10DC10003F1D002CD2D1BDE8F0870000E8150020A0
:10DC2000D81300202DE9FF5F424893460EAA0068F2
:10DC300092E89002007C0D191E7810F003019846BE
:10DC40004FF0F0001CD0022937D15FEA090155D00E
:10DC50004FEA000AC4F101008100C1F104022AFA6E
:10DC600002F03040C84006D059F820305A462946C4
:10DC7000009804F030F9641C6D1C022C38D03AE096
:10DC80005FEA09011BD08246C4F101008100C1F1A5
:10DC900004022AFA02F03040C840294659F82030E0
:10DCA0006D1C5A46009804F016F9641C022C02D12F
:10DCB00018F8016F00247F1EE6D1BDE8FF9F814662
:10DCC000C4F101008000C0F1040129FA01F33340DE
:10DCD000C34029466D1C5A46009804F0FCF8641CA9
:10DCE000022C02D118F8016F00247F1EE8D1E4E76E
:10DCF00018F8016F00247F1EACD1DEE74FEA00095F
:10DD0000C4F101008000C0F1040129FA01F333409D
:10DD1000C34004D05A462946009804F0DCF8641C3D
:10DD20006D1C022C02D118F8016F00247F1EE7D170
:10DD3000C3E70000201400202DE9F05F92460BAAF3
:10DD4000894692E842010A9F9B468B003A78C1F1CE
:10DD500002009A40D5B24F4A0E9CC0B21268127CA3
:10DD600012F003021BD0012A7CD0022A3AD1D9B387
:10DD700028090DD02909B9F1000F38F821002080B9
:10DD800006D0D9F808005A465146036848469847D5
:10DD9000A41C0AF1010A17F8015F761E4CE039B1A4
:10DDA0002909761E38F8210024F8020B17F8015FC4
:10DDB000022E11DB701006F001062A09401E38F809
:10DDC000221005F00F0224F8021B38F8221024F864
:10DDD000021B17F8015FF0D1002E03D0290938F893
:10DDE00021002080BDE8F09F26E028090DD02909F8
:10DDF000B9F1000F38F82100208006D0D9F80800CA
:10DE00005A46514603684846984715F00F000DD012
:10DE100038F820006080B9F1000F07D0D9F8080069
:10DE20005A460AF1010103684846984717F8015F0E
:10DE3000241D0AF1020AB61E022ED6DA002ED1D017
:10DE40002809CFD038F820002080B9F1000FC9D0C0
:10DE5000D9F808005A46514603684846BDE8F05FC5
:10DE60001847FFE7B04200DDF0B2361AA90903D027
:10DE7000218881F0FF01218029070D0E401EA41C7E
:10DE800010F0FF00F2D1002EACD0022017F8015F95
:10DE9000E8E70000201400202DE9F05F92460BAA6D
:10DEA000894692E842010A9F9B468B003A78C1F16D
:10DEB00002009A40D5B24D4A0E9CC0B21268127C44
:10DEC00012F003021BD0012A79D0022A37D1C1B344
:10DED00028090DD02909B9F1000F58F82100206058
:10DEE00006D0D9F808005A46514603684846984774
:10DEF000241D0AF1010A17F8015F761E49E031B1CD
:10DF00002909761E58F8210001C417F8015F022E76
:10DF10000FDB701006F001062A09401E58F8221087
:10DF200005F00F0202C458F8221002C417F8015F6E
:10DF3000F2D1002E03D0290958F821002060BDE855
:10DF4000F09F26E028090DD02909B9F1000F58F8F3
:10DF50002100206006D0D9F808005A4651460368CF
:10DF60004846984715F00F000DD058F82000606023
:10DF7000B9F1000F07D0D9F808005A460AF101019B
:10DF800003684846984717F8015F08340AF1020A07
:10DF9000B61E022ED6DA002ED1D02809CFD058F8DE
:10DFA00020002060B9F1000FC9D0D9F808005A4606
:10DFB000514603684846BDE8F05F1847FFE7B042A6
:10DFC00000DDF0B2361AA90903D0216881F0FF0103
:10DFD000216029070D0E401E241D10F0FF00F2D114
:10DFE000002EACD0022017F8015FE8E720140020D3
:10DFF00070B5DDE90454002C69D08068066A0068B9
:10E0000002FB061100EB410037490968097C11F059
:10E01000030134D002295AD162E000BF13F8011B7A
:10E02000083D34F8211020F8021B13F8011B34F8C6
:10E03000211020F8021B13F8021B34F8211020F8DD
:10E04000041B13F8011C34F8211020F8021C13F8EB
:10E05000041B34F8211020F8081B13F8031C34F8B3
:10E06000211020F8061C13F8021C34F8211020F8A7
:10E07000041C13F8011C34F8211020F8021C082D90
:10E08000CCDA18E013F8011B2D1F34F8211020F80A
:10E09000021B13F8011B34F8211020F8021B13F89F
:10E0A000021B34F8211020F8041B13F8011C34F86B
:10E0B000211020F8021C042DE4DA06E013F8011BFD
:10E0C0006D1E34F8211020F8021B002DF6D170BD12
:10E0D000197811B134F821100180801C5B1C6D1E71
:10E0E000002DF5DC70BD0000201400202DE9FF4F4D
:10E0F00085B08346816891465D48DDE91262DDE9BD
:10E100001474DDF85C8000681D46042A51D005DCDB
:10E11000012A11D0022A25D1002046E0082A5CD02D
:10E12000102A1FD1D1F84CC0BCF1000F02D0007CE6
:10E13000C0077CD0002097E0D1F83CC0BCF1000FB4
:10E1400002D0007CC00701D000201CE0CDE903789C
:10E15000CDE901361698009023464A46DBF81800B0
:10E160000699E04709B0BDE8F08F00BF16980AEBAA
:10E1700009028DE82101234658460699FFF7E2F986
:10E180003C440AF101008246B042EFDBEAE700BFFF
:10E1900016990AEB09028DE8220123465846069992
:10E1A000FFF77CFB3C440AF101008246B042EFDB02
:10E1B000D8E700200DE000BF16980AEB09028DE8B1
:10E1C0002101234658460699FFF72CFD3C440AF1ED
:10E1D00001008246B042EFDBC4E7D1F840C0BCF199
:10E1E000000F10D0007C80070DD45FEA08000AD031
:10E1F000CDE90036CDE9027823464A46DBF818001F
:10E200000699E047AEE700200CE000BFCDE90058DA
:10E210000AEB0902234658460699FFF7E9FE3C44FB
:10E220000AF101008246B042F0DB9BE7FFE78DE890
:10E23000C80023464A46DBF818000699E04791E7F4
:10E24000DBF80800069A08EB0903D0F820C0006844
:10E2500003FB0C22074B00EB420021461B686A00BF
:10E2600098473C4408F101008046B042E8DB79E77A
:10E2700020140020E81500202DE9FF4F8FB0A94899
:10E28000DDE91F860068DDE91C970C46006EF5F796
:10E2900027FD0790406908B1F5F722FD0A9007981D
:10E2A000C0680C9007A8F5F771FDA01910900A98A6
:10E2B00058B19C490968097C890706D110ACCDF892
:10E2C000009094E80E00F7F725FADDE9100104F05C
:10E2D000C5FB0446102F03D0182F5EDB002058E04A
:10E2E00000251FE0DDE910B02844DDF828A00190EA
:10E2F000129E5FEA080120460FD070B18A4B72006F
:10E300001B689847BAF1000F07D0DAF808003346C7
:10E31000594647685046019AB8471E990C98884458
:10E3200004446D1C4D45DDDBF2E00A980390DDE905
:10E3300010B00699DDF848A0084401905FEA08058E
:10E34000264620D0FEB1039830B180685346594626
:10E350004768019A0398B8470F99286809690968BE
:10E3600088473080039828B180685946019A03682D
:10E37000039898472D1DAAF10100B61C0BF1010B63
:10E380005FEA000AE8D10C981E9904440698884474
:10E39000401C06904845C8DBBAE0082F02D02198FF
:10E3A000C8B36DE0002065E02198DDF840A00028AA
:10E3B0000A98029030D01198129F584400902198EA
:10E3C00004905848454626460068007C10F003003B
:10E3D00002D0022848D109E015F8011B04987F1EDD
:10E3E00030F8210026F8020BF6D13DE0287858B12C
:10E3F000049931F820003080029828B18068514695
:10E40000009A0368029898476D1CB61C0AF1010A2D
:10E410007F1EEBD128E031E01199129F0BEB010038
:10E4200000904048464625460068007C10F00300F6
:10E4300002D0022818D106E03B4B3A4641461B6801
:10E440002046984710E0307840B12880029828B1E3
:10E4500080685146009A036802989847AD1C761C64
:10E460000AF1010A7F1EEED10C981E9904448844DB
:10E470000BF101008346484596DB49E02B4821908B
:10E48000002543E03846012F04D002281CD0042F79
:10E4900037D128E023480068006EF5F721FCCDF85D
:10E4A00000800790129A21990594CDE90310CDE9D7
:10E4B000016211980A992B18DDE90F02FFF7BCF8E9
:10E4C00007A8F5F763FC1CE021981299CDE902102A
:10E4D000CDE90086119804942B18DDE90F020A9902
:10E4E000FFF766FA0DE021981299CDE90210CDE907
:10E4F0000086119804942B18DDE90F020A99FFF7A2
:10E500001BFC1E990C98884404446D1C4D45B9DBD6
:10E510000A98002802D00AA8F5F738FC13B0BDE825
:10E52000F08F000020140020E8150020F0530108AF
:10E530002DE9FF4F0C46A5498DB00868DDE91A9614
:10E54000DDE91D87006E00287ED0F5F7C9FB069037
:10E55000406908B1F5F7C4FB0A900698C0680890B6
:10E5600006A8F5F713FCE0190E900A9858B19749E0
:10E570000968097C890706D40EACCDF8009094E8B0
:10E580000E00F7F7C7F8DDE90E0104F085FA04463E
:10E59000182E15DB002510E01098CDF80080CDE98D
:10E5A00001040F980A992B18DDE90D02FFF7E0FA34
:10E5B0001C986D1C8044089804444D45ECDBFBE03E
:10E5C000102E05D0082E42D01F98002877D0ACE03E
:10E5D000002036E00E98029009990F98DDF828A0E7
:10E5E00008440190DDF840B0464625465FEA0A003F
:10E5F00007D0DAF80800DDE9012147685B4650469C
:10E60000B8470D9930880969496888472860BAF188
:10E61000000F06D0DAF80800DDE901210368504652
:10E62000984702982D1D401C0290ABF10100B61CCA
:10E630005FEA000BE5D108981C99044409988844C6
:10E64000401C0990484500E0BCE0C3DBB4E000207A
:10E6500065E01F9800280A9832D00090DDE90EA1ED
:10E660000BEB010001901F9803905848109F4546FE
:10E6700000682646007C10F0030002D0022848D132
:10E6800008E015F8011B03987F1E50F8210001C611
:10E69000F7D13EE0287858B1039951F82000306056
:10E6A000009828B1806851460368DDE90002984768
:10E6B0006D1C361D0AF1010A7F1EEBD129E032E004
:10E6C0000490DDE90EA058440B904048109F454649
:10E6D00000682646007C10F0030002D0022818D102
:10E6E00006E03B4B3A4641461B682046984710E0FF
:10E6F000287840B13060049828B1806851460B9A60
:10E700000368049898476D1C361D0AF1010A7F1EA4
:10E71000EED108981C99044488440BF1010083460B
:10E72000484596DB48E02B481F90002542E0012E2B
:10E7300004D0022E1CD0042E37D128E023480068D4
:10E74000006EF5F7CDFA0690CDF800801F9A10996B
:10E750000594CDE90320CDE901710F980A992B1892
:10E76000DDE90D02FFF70CF806A8F5F70FFB1CE03A
:10E7700010991F98CDE90087CDE902100F980494F5
:10E780002B18DDE90D020A99FFF782F90DE01099C7
:10E790001F98CDE90087CDE902100F9804942B183B
:10E7A000DDE90D020A99FFF777FB1C990898884468
:10E7B00004446D1C4D45BADB0A98002802D00AA813
:10E7C000F5F7E4FA11B0BDE8F08F00002014002046
:10E7D000E81500209C5C01082DE9FF4F85B01D461F
:10E7E000DDE9120614462A4302430B4632437DD02C
:10E7F00005986946C06A07681846FCF72FFDFCF7C4
:10E800008DFD0390FCF792FD0290BDF90000BDF96B
:10E81000041000EB040BBDF9020000EB050A12988E
:10E82000A1EB0009BDF90600A0EB06080598806B76
:10E83000F6F774FD0598C06BF6F77BFDCCB1149824
:10E84000E219521EB0F900100398081A904210DC29
:10E85000BDF90630BDF900009B1BE9195B1CF5F7FB
:10E86000D3FB08F10102AAF10101ABF10100F5F7B8
:10E870000BFFC5B11498EB195B1EB0F9021002989A
:10E88000081A98420FDCBDF90000BDF90210BDF96D
:10E890000420F5F7B9FB09F10102ABF10101AAF17E
:10E8A0000100F5F731FE1298C8B11499BDF90420A2
:10E8B000B1F904300399101A591A401C81420EDB39
:10E8C000BDF90630E9199B1B5B1CF5F79DFB08F1B0
:10E8D0000102AAF1010109F10100F5F7D5FE002EB0
:10E8E0001AD0BDF906301498991B00E014E0B0F975
:10E8F00006200298491C101A88420DDBBDF9000061
:10E90000BDF90420F5F780FB09F10102ABF101012B
:10E9100008F10100F5F7F8FD09B0BDE8F08F704788
:10E920001CB56846FCF7F6FB684600F003F81CBD12
:10E930007047000010B59EB004466846F6F7BCFC70
:10E9400009480068FAF748FCB4F90630B4F9042025
:10E95000B4F90210B4F90000F5F74CFE6846F6F77A
:10E96000A3FC1EB010BD00008C170020704770B5CE
:10E9700004460D460868F6F7DCFCB4F90420B4F947
:10E980000010B4F90200491C521EF5F7BDFDB4F9A0
:10E990000420B4F90010B4F90600491C521EF5F722
:10E9A000B3FDB4F90620B4F90210B4F90000491C13
:10E9B000521EF5F769FEB4F90620B4F90210B4F955
:10E9C0000400491C521EF5F75FFE6868F6F7B1FCBB
:10E9D000B4F90420B4F90010B4F90200491C401C39
:10E9E000521EF5F791FDB4F90420B4F90010B4F902
:10E9F0000600491C401E521EF5F786FDB4F906209C
:10EA0000B4F90210B4F90000891C401C921EF5F7FD
:10EA10003BFEB4F90620B4F90210B4F90400891CD5
:10EA2000401E921EF5F730FEA868F6F782FCB4F996
:10EA30000210B4F90000F5F7B7FDB4F90610B4F907
:10EA40000000F5F7B1FDB4F90210B4F90400F5F7D0
:10EA5000ABFDB4F90610B4F90400BDE87040F5F759
:10EA6000A3BD2DE9FF4F87B09846DDE91457F5F7B0
:10EA7000D2FE0190BD420ED12846FAF7ADFB1798A1
:10EA800020B107AC434694E8070080E0DDE90710B9
:10EA90004246099B7BE0089A0126B8EB020470D03D
:10EAA000E9B2FAB2521A059204FB01F204EBD471F6
:10EAB00002EB610BC5F30722C7F307239B1A6243DE
:10EAC00002EB610A0493C5F30742C7F307439B1A9D
:10EAD000624302EB61092A0E0393C2EB17636243A0
:10EAE00002EB61070293089D3CE09BFBF4FE059A54
:10EAF00099FBF4FC93449AFBF4F2049B02999A4428
:10EB0000039B994497FBF4F30F444EEA022141EA38
:10EB10000C4141EA0361009108998D4220DD009982
:10EB2000814201D1761C1BE0FAF756FB1798012EA3
:10EB30000CDD20B1A91B6B1E099A079803E0A81BE6
:10EB40006A1E099B0799FAF72BF808E0099A10B199
:10EB5000691E079801E00799681E169B98470126D1
:10EB600000986D1C4545C0DDFAF736FB1799404605
:10EB7000012E0FDD31B1811B4346491C099A0798CC
:10EB800005E015E0841B4246601C099B0799FAF7D3
:10EB900007F807E0099A11B14146079800E0079984
:10EBA000169B984701980BB0BDE8F04FFAF714BBDD
:10EBB0000BB0BDE8F08F00002DE9FF4F8FB09046FD
:10EBC000DDE91D93DDF870A05FEA0A025AD05FEA22
:10EBD000090257D0002955DD1AF1010215D0BAF10A
:10EBE000010F4A4618D0012A1CD00525734A4FF060
:10EBF000FF3E12685269002A16D000BFB2F90240E7
:10EC00000894B2F90640049412E0B9F1010F01D062
:10EC10000225EBE70125E9E7012A01D00325E5E715
:10EC20000025E3E70425E1E7CDF810E0CDF820E08A
:10EC30004FF00004A3460E46069414D0B2F90070BB
:10EC4000A7F1010CC44504DDA7EB0804641E00D540
:10EC5000002408EB0107B2F904207F1E974202DD71
:10EC6000A2EB0806761C2BB100EB4107BF1ECDF8C6
:10EC700030E003E0012100EB44070C9101200A90F1
:10EC8000B44270DB13B0BDE8F08F00BF0C99B7F948
:10EC9000000007EB4107A0F5FE41FF390AD00A99B1
:10ECA00089B300210A91062D2AD2DFE805F0291246
:10ECB00015181D220A990698084305D104EB08008F
:10ECC0005946401EF9F70EFF01200A9000200690D9
:10ECD0006EE01299081A6AE01299091A01E0129975
:10ECE0000144B1FBF9F062E01299084400FB0AF01C
:10ECF0005DE01299084400FB0AF0B0FBF9F056E021
:10ED00001299084453E0FFE7062D3ED2DFE805F0F4
:10ED10003D03062C31361299081A02E01299091A9D
:10ED200024E0089901908B4502DA019888423ADB89
:10ED300004998B4502DD0198884234DC01980199E1
:10ED4000584400EBD070401003908B4504EB080052
:10ED50001EDC07905946401E039AF9F7F7FE019A08
:10ED6000039907981DE024E012990144B1FBF9F0E2
:10ED7000D7E71299084400FB0AF0D2E71299084439
:10ED800000FB0AF0B0FBF9F0CBE712990844C8E7A2
:10ED900005905A46401E0399F9F7D8FE039A019947
:10EDA0000598F9F7D3FE0698401C06900198834613
:10EDB000641CB442FFF66AAF64E700002014002030
:10EDC00070B5B0F90420B0F900301A445410B0F90D
:10EDD0000620B0F90230D01AC01C80101E18151A77
:10EDE000886AF6F7A6FA2A4631462046F5F74CFC23
:10EDF0002A463146A01CF5F747FC2A463146201D1D
:10EE0000F5F742FC2A463146A01EF5F73DFC2A469E
:10EE10003146201FBDE87040F5F736BC70B5B0F93B
:10EE20000620B0F902301A445410B0F90420B0F9A9
:10EE30000030D01AC01C80101E18151A886AF6F708
:10EE400078FA2A4631462046F5F75EFB2A463146D7
:10EE5000A01CF5F759FB2A463146201DF5F754FB57
:10EE60002A463146A01EF5F74FFB2A463146201FA1
:10EE7000BDE87040F5F748BB2DE9FF4F904685B0DF
:10EE80000A46044669461046DDF84CB0FCF7E6F940
:10EE9000E06ABDF9001000680390BDF90400D4E9F0
:10EEA0001176411A1298A1EB0801081A00F1010924
:10EEB000BDF90600BDF90210411A0898091AA1EB24
:10EEC0000B0000F1010A206CF6F733FAF5F7E8FCC5
:10EED000029067B394F87800E16CC00701D000207D
:10EEE00001E0D4F88C0038440D1800E0ED1BBD4261
:10EEF000FCDA94F87A00F6F767FA16E0039805EB67
:10EF000008010844BDF902200899BDF906301144F2
:10EF1000A3EB0B0294F87A3023B113460246F5F7BF
:10EF20001FFB01E0F5F7B0FB3D444D45E6DB4EB37A
:10EF3000206DD4F880103044451A00E0AD1BB54276
:10EF4000FCDA94F87B00F6F73FFA19E0BDF90610F9
:10EF5000BDF90020A1EB0B0002EB0807BDF904206E
:10EF60001299401B521A94F87B1029B10346194696
:10EF70003846F5F7F5FA02E03946F5F7C5FA3544B3
:10EF80005545E3DB0298F6F71FFA09B0BDE8F08FAC
:10EF900008B5009200F078FA08BD08B5009200F0BC
:10EFA00087FA08BD08B5009200F0D8FA08BD000045
:10EFB000034A1268527E002A01D1F4F773B87047F1
:10EFC000201400202DE9F041134E9EB00125B46BB2
:10EFD00004B974696846F6F76FF910480068D0E91B
:10EFE0000C875CB12046FDF791F900B16D1E2046FB
:10EFF000F4F7E4FE44690CB1002DF3D14046B4634C
:10F00000F6F797F93846F6F789F96846F6F74CF9B6
:10F010001EB0BDE8F0810000601500202014002023
:10F020002DE9F04F8DB0824616981C1E17460D46EE
:10F0300076DDF6F77EF9661E07EB04082F1B0DF14F
:10F0400014090AEB04051EE0A8EB0600039009ABC7
:10F050000AAA3146CDF80090204600F081FF0A98B8
:10F0600009992B1A07EB000B78186A1A00F1010AAC
:10F070001846521E0399F9F709FD5A46504603995E
:10F08000F9F704FD761E002EDEDC012C48DD179812
:10F09000F6F74FF9A61E1EE0A8EB0600039009AB99
:10F0A0000AAA3146CDF80090204600F059FF059895
:10F0B00009992A1A6B1A384407EB010B00F1010A6F
:10F0C0001846521E0399F9F7E1FC5A465046039937
:10F0D000F9F7DCFC761E002EDEDC022C20DD189811
:10F0E000F6F727F9E61E1BD005A80090A8EB060A44
:10F0F00009AB0AAA3146204600F032FF05986A1E85
:10F100002B1A07EB000B07F1010951461846F9F7D6
:10F11000BDFC5A4651464846F9F7B8FC761EE3D185
:10F120000DB0BDE8F08F70471CB56846FBF7F2FFE5
:10F13000684600F003F81CBD7047000010B59EB093
:10F1400004466846F6F7B8F809480068FAF744F844
:10F15000B4F90630B4F90420B4F90210B4F900008F
:10F16000F5F748FA6846F6F79FF81EB010BD0000A4
:10F170008C17002008B500930B4600F085F908BDF8
:10F180002DE9FC47DFF8AC8081461E46D8F8000028
:10F1900015468A46006EF4F7A3FD0190406908B158
:10F1A000F4F79EFD00902946504603F057FC0446B4
:10F1B0000198C768D8F80000017CC90715D0D9F8B4
:10F1C00010008068804787B2009820B181682A4685
:10F1D0000B685146984720886D1C78402080019824
:10F1E000B542C0680444EFDD19E0C06B01680098C7
:10F1F00070B11FFA81F800982A4681680B68514661
:10F200009847A4F800806D1C3C44B542F3DD06E04D
:10F21000701B89B2401C21803C44401EFBD101A8D8
:10F22000F4F7B4FD0098002802D06846F4F7AEFD6C
:10F23000BDE8FC87201400202DE9FC47284F1E461E
:10F24000154638688946006EF4F74AFD019040691A
:10F2500008B1F4F745FD00902946484603F01CFC30
:10F26000396804460198CA6B097CD0F80C8017688D
:10F27000C90715D000680069806880470746009874
:10F2800020B181682A460B684946984720686D1C62
:10F29000784020600198B542C0680444EFDD13E077
:10F2A000009858B100982A4681680B6849469847EB
:10F2B00027606D1C4444B542F4DD05E0701B401C22
:10F2C00027604444401EFBD101A8F4F75FFD00987D
:10F2D000002802D06846F4F759FDBDE8FC8700001D
:10F2E000201400207CB50D46C16A0C68D0E90212DA
:10F2F000CDE900126946FDF721F9B5F90000BDF925
:10F3000000102044884214DCB5F90400BDF9041053
:10F31000001B88420DDBB5F90200BDF90210204444
:10F32000884206DCB5F90600BDF90610001B8842CC
:10F3300001DA01207CBD00207CBD017001207047F6
:10F340002DE9F047234C0427E06AE0B1206907EB80
:10F35000D0014518E800FDF719FA060038D0616BB6
:10F3600007EBC600B9460F5820691B4BC20008378F
:10F370001B683846D4F82C8098476763E6624A4693
:10F38000691E20690EE01348C030D0E90110083032
:10F39000B1FBF0F5AD1CDDE7666B431C02EBC0076B
:10F3A000401CF3518842F7D3636B09EBC000002186
:10F3B0001950206960626168281A084425616060FC
:10F3C000B8F1000001D0F4F7D3FB0020BDE8F087CE
:10F3D0000120FBE7284F0020E81500200A4810B55F
:10F3E000006890F8540068B1084CA08850B1F5F757
:10F3F000FFFAFFF7E7FDF6F78BFAA088002800D0A8
:10F40000012010BD002010BD201400206015002038
:10F41000F8B51A4DE86BE8B1F5F7EAFA6C6913E054
:10F420002046F4F75DFC0090018D090408D52646BE
:10F4300044696846F4F7AAFC3046FBF78DFD03E00B
:10F4400044696846F4F7A2FC002CE9D10020E86387
:10F45000F6F75EFA286A00B180470948006808B1EB
:10F46000804738B90748006890F8540020B1F5F794
:10F47000B5FE08B10120F8BD0020F8BD60150020E0
:10F4800064140020201400207CB58468069D646B01
:10F4900044B1064E3668F66B3668CDE90056806991
:10F4A000A0477CBD009500F0ABF87CBD2014002087
:10F4B0002DE9FF4FDFF8A0A00C4685B0DAF8000078
:10F4C000DDF848801F46C16B154609680391006E40
:10F4D000F4F706FC01902946204603F0BFFA0646E1
:10F4E0000198391B01F1010BD0F80C90406950B321
:10F4F000F4F7F6FBA8EB0501491C00915B462A4690
:10F5000002902146F6F706F902A8F4F73FFC1AE04C
:10F51000DAF80000007CC0070DD005985F4634463D
:10F5200000698068804780B22188414024F8021B2E
:10F530007F1EF9D105E003985A4681B23046F7F7AD
:10F540002BF94E446D1C4545E2DD01A8F4F71EFC85
:10F5500009B0BDE8F08F0000201400202DE9FE4F17
:10F56000264E1F46144630680D46DDF83090006E7A
:10F57000F4F7B6FB01902146284603F08DFA791B7B
:10F5800001F1010A316880460198C96BD0F80CB0CE
:10F590000E68406958B3F4F7A3FBA9EB0401491CBA
:10F5A00000915346224602902946F6F7B3F802A886
:10F5B000F4F7ECFB1BE011480068007CC0070CD09E
:10F5C0000198574645460068006980688047296869
:10F5D000414002C57F1EFAD107E0BAF1000004DD08
:10F5E00001464046491E40C0FCD1D844641C4C45ED
:10F5F000E1DD01A8F4F7CAFBBDE8FE8F201400206E
:10F60000F0B584684F48059E5B1A0768F86B3F7C2D
:10F610000568206A24684FEA600C0CFB02FCB21AF1
:10F620000CEB510C4610521C00205B1C04EB8C04AC
:10F63000FF074FEAC17130D061B11100204607D0F9
:10F64000414F05687D40056000EB8600491EF8D1FA
:10F650005B1E241D022B12DB11000CD0481E7043D0
:10F660001D4604EB8000AD1E0768FF4380C0022DDD
:10F67000F9DA491EF2D1044623F001001B1A002BCF
:10F680000ADD002A08D04FF6FF712068484020604C
:10F6900004EB8604521EF8D1F0BD69B1110020467A
:10F6A00008D00788491EBFB247EA0547076000EB4C
:10F6B0008600F6D15B1E241D05EB0541102B1FDBD8
:10F6C000103B170017D0781E70439C4604EB800057
:10F6D000BCF1100C02C002C040F8081B40F8041C2A
:10F6E00040F8101B40F80C1C40F8081C40F8041CA3
:10F6F000EED57F1EE7D1103323F00F070446DB1B46
:10F70000022B12DB17000CD0781E70439C4604EBD2
:10F710008000ACF1020C02C0BCF1020FF9DA7F1ECE
:10F72000F2D1044623F001001B1A002BB4DD002A9D
:10F73000B2D020686FF30F002843206004EB8604EA
:10F74000521EF4E7201400200000FFFFFEB54F4CCE
:10F75000D4E90201CDE90001206970B3A089401C01
:10F7600000B2ADF800006189ADF80210B4F90410E0
:10F77000884207DD2088ADF80000E08910F1010023
:10F78000ADF80200BDF90200B4F90610884274DC3D
:10F790003F4D2868806CF4F7A3FA0290BDF9000091
:10F7A000B4F90010884220D1E088ADF80600A088A6
:10F7B000ADF804002868806C0FE0FFE72088ADF802
:10F7C00000006088DCE700BFF4F7F8FA0646006A3C
:10F7D0000022694600F0D5F8B0690028F4D10298FB
:10F7E00000226946C06900F0CCF8BDF80000ADF811
:10F7F00004002868806C0AE0F4F7E0FA0646006A24
:10F800000022694600F046F80028EED1B0690028D1
:10F81000F2D1029800226946C06900F03BF8002846
:10F82000E3D1B4F90400BDF90010ADF8040088423A
:10F8300007DADDE90001C4E9020102A8F4F7A6FA3B
:10F8400098E72868806C08E0F4F7B8FA0546006A83
:10F850000022694600F05CF8A8690028F4D10298FB
:10F8600000226946C06900F053F802A8F4F78EFA46
:10F87000206944F62061884201DD0020FEBDDDE9FB
:10F880000001C4E902010120FEBD00006850002013
:10F8900020140020FEB517460E460546002433E02E
:10F8A0002846F4F71DFA0090856A0146A80726D578
:10F8B00027B13A4601A8F6F7FDFD03E0D1E90001C2
:10F8C000CDE9010101A93046F5F7D2FCB8B1E8074E
:10F8D00002D00098C56910E0BDF80800401C3080D7
:10F8E00001240CE001AA31462846FFF7D3FF00B1FE
:10F8F00001242846F4F762FA056A002DF2D1009837
:10F90000056A6846F4F742FA002DC9D12046FEBDCB
:10F91000FEB516460D46044630E02046F4F7E0F901
:10F920000090846A0146A00723D526B1324601A87B
:10F93000F6F7C0FD03E0D1E90001CDE9010101A91D
:10F940002846F5F795FCA0B1E00702D00098C469FD
:10F950000DE0BDF80400401EA8800AE001AA294677
:10F960002046FFF7D5FF2046F4F728FA046A002C5A
:10F97000F4D10098046A6846F4F708FA002CCCD158
:10F98000FEBDFEB516460D4604464AE02046F4F795
:10F99000A7F90090846A0146A0073DD526B13246FA
:10F9A00001A8F6F787FD03E0D1E90001CDE90101E7
:10F9B00001A92846F5F75CFC10B3E00702D00098D7
:10F9C000C46927E000983EB1B0F90210B6F9020010
:10F9D000814203DD084601E0B0F90200B5F90210EA
:10F9E000814207DABDF90600B5F90610401E05E0B0
:10F9F000E88011E0BDF90A00B5F906108842F7DB8E
:10FA00000AE001AA29462046FFF7BBFF2046F4F78B
:10FA1000D5F9046A002CF4D10098046A6846F4F71A
:10FA2000B5F9002CB2D1FEBDF4F7A2B810B521B1E2
:10FA3000B0F90410B0F9000003E0B0F90610B0F915
:10FA400002000324081A401C011F91FBF4F111600D
:10FA5000411AA0EB6100401E186010BD70B58AB05D
:10FA60000C460546F4F73CF90990066D09A8F4F731
:10FA70008DF9009534B1012C06D0022C0AD0032C4C
:10FA800004D109E0182000E0162001906846B04734
:10FA90000AB070BD1520F8E71720F6E7074A0749B6
:10FAA000121D51F8201052F820205143034A083209
:10FAB00052F820004143084670470000AC13002074
:10FAC0000078704701207047002801D1FBF71CBB6C
:10FAD000704700008068012905D0032901D000206B
:10FAE00070470068704701487047000030540108B3
:10FAF000012901D0002070470048704730540108A8
:10FB0000012901D00020704700487047DC5C0108E3
:10FB10002A294AD2DFE801F04947211D1F4923491C
:10FB20004915191B254927294949492B2D2F3549A5
:10FB300049374949494949493B313343493F494993
:10FB400049171B4870471B4870471B4870471B48A4
:10FB500070471B4870471B4870471B4870471B483D
:10FB600070471B4870471B4870471B4870471B482D
:10FB700070471B4870471B4870471B4870471B481D
:10FB800070471B48704700688068406B704700688A
:10FB90008068C06B704700688068006C70470068C0
:10FBA0008068406C70471348704700207047000021
:10FBB000012101082921010841210108BB20010878
:10FBC000791F010871FE0008471C010899210108EE
:10FBD000B9020108FD0D0108F30D01086D1C0108B3
:10FBE000AF1C01089D1C0108F1CD0008BF210108D0
:10FBF0002D1D0108AD1A0108162901D000207047FB
:10FC000000487047F9500008162901D000207047BD
:10FC100000487047A950000870B500240D4602281E
:10FC200007DAF4F7E1FA20B1C1688A6A29469047F9
:10FC30000446204670BD80680F2917D2DFE801F026
:10FC400016080A0C0E1616161014121214141400AC
:10FC5000006970474069704780697047C0697047A4
:10FC60001020704701207047002070474FF0FF3090
:10FC70007047082904D0006820B1C268926A104712
:10FC8000102070474FF0FF307047082901D0002046
:10FC90007047202070472DE9F0410E4607460025A9
:10FCA000F4F78CF8C46908E02046FBF7B9FAB042D3
:10FCB000204616D0F4F782F8046A002CF4D13846B6
:10FCC000F4F77CF8C46909E031462046FFF7E3FF0A
:10FCD000050005D12046F4F771F8046A002CF3D131
:10FCE0002846BDE8F08110B5F8F7ACFFB0F5807F8D
:10FCF00003D0802803D307211AE0082118E0402808
:10FD000001D3062114E0202801D3052110E010289A
:10FD100001D304210CE0082801D3032108E00428C2
:10FD200001D3022104E0022801D3012100E00021D7
:10FD300001208840401E10BD0F207047FF207047F3
:10FD4000FF2070474FF6FF7070474FF0FF3070474D
:10FD50004FF6FF7070474FF6FF7070474FF6FF7019
:10FD6000704770B500240646012531462846FFF746
:10FD700053FF844200DA04466D1EF6D5204670BD5E
:10FD80000146054A0F2000BF02EBC0031B6C8B42EB
:10FD900001D9401EF8D57047284F002070B50546A0
:10FDA0000C0004D00846F4F709F8006A18B9284690
:10FDB000F4F704F8C069A04200D1002070BD70B50E
:10FDC000DDE90445466D0E60816D1160C16D1960FD
:10FDD000016E2160C06A0068286070BD8068036A97
:10FDE000006802FB031130F81100704710B5084697
:10FDF000114602F033FE008810BD10B508461146CA
:10FE000002F04AFE006810BD012801DB00207047A7
:10FE1000104951F820001049884201D10220704752
:10FE20000E49884201D1032070470D49884201D113
:10FE3000042070470B49884201D1052070470A49C8
:10FE4000884201D1062070470849884201D1072025
:10FE50007047FEE7A0130020F0320108803201084D
:10FE6000983201085032010838320108683201081E
:10FE700070B514460D46064600F0B4FAB068002886
:10FE800003D0416A2960806A206070BD10B504000B
:10FE900002D0FCF73DF810B92046FCF70DF8A0425F
:10FEA00000D1002010BD806800220A804A80028BA9
:10FEB000521E8A80808B401EC880704738B50C4621
:10FEC0008068F3F70DFF0090808820800098C0883C
:10FED00060800098818802891144491EA180C188F0
:10FEE00040890844401EE0806846F3F74FFF38BD64
:10FEF00038B50C468068F3F7F3FE009080882080C8
:10FF00000098C08860800098818802891144491E49
:10FF1000A180C18840890844401EE0806846F3F70C
:10FF200035FF38BD70B500240C4D0CE0F5F70DFD24
:10FF30002A69C4EB441152F82110814201D12046B4
:10FF400070BD29B1641CA8688442EFDB002070BD3D
:10FF5000C4EB441142F82100F1E700000016002034
:10FF60002DE9F0470D460446461E01FB05F76043A8
:10FF700099469246C01BDDF82080F6F72BFCCAF8A4
:10FF800000004FF0000AB54210DA7643F01BF6F796
:10FF900021FCA41EC9F80000A54204DA401EC8F8DE
:10FFA0000000BDE8F087C8F800A0FAE75046C9F89D
:10FFB00000A0F4E7054A904201D1503A01E000F177
:10FFC000080209B18A4200D010467047D050002084
:10FFD0000021FFF7EFBF0000F0B4124C646814B1C9
:10FFE000A446F0BC6047541E04FB030401EB8200EE
:10FFF0000D4DDFF838C0001F2188E41A01F01F06FC
:020000040801F1
:10000000521EAF5DC1F3451605EBD1211CF8066009
:10001000097801EB062101EB074140F80419EBD107
:10002000F0BC7047B4140020B8460108D846010857
:1000300010B50468184410C1521EFAD110BD00005A
:100040002DE9F0471446521E984602FB080601EBC4
:100050008405DFF83090DFF830A02D1F3778D9F80D
:100060000410384688470AEB1711A6EB08060978F2
:10007000641EC1F1FF0140EA016045F80409EDD1B9
:10008000BDE8F08790460108A84601082DE9F04731
:100090001446521E984602FB080601EB8405DFF861
:1000A0002C904FF07F4A2D1F3788D9F80410F8B2F2
:1000B000884707F47F428AEA0241014345F8041960
:1000C000A6EB0806641EEFD1BDE8F08750320108A8
:1000D000F0B4144C646814B1A446F0BC6047541EDC
:1000E00004FB030401EB82000F4D001F2188E41A7A
:1000F00001F01F06521E15F806C0C1F34416AF5D8D
:10010000C1F3842641F3C031AE5DC1F1FF0106EBBE
:10011000072606EB0C4606EB016140F80419E5D111
:10012000F0BC7047C0130020B846010838B503245E
:100130000094FDF743F838BDF0B4144C646814B172
:10014000A446F0BC6047541E04FB030501EB82008B
:100150000F49001F2C88ED1AC4F3032611F806C0BE
:10016000C4F303168F5D04F00F0601EB14348E5DAB
:100170002478E443240604EB064404EB0724644497
:1001800040F80449521EE5D1F0BC7047C813002066
:10019000A846010838B504240094FDF70FF838BDCF
:1001A00038B500240094FDF709F838BD38B50024AF
:1001B0000094FDF703F838BD70B50446F8F742FD2A
:1001C0000546F8F757FDAC4201D3002070BD00286A
:1001D000FCD050F8240070BD70B5C0F38001C0F3AE
:1001E000C00201EA000602EA0003C0F3400404EA88
:1001F000000560193144C5EBC010C6EBC1111A44AB
:10020000C3EBC21240EA012040EA024070BD000088
:1002100010B507490446C0B249688847054901EB53
:1002200014110978C1F1FF0140EA016010BD00001E
:1002300090460108A846010810B506490446C0B218
:100240004968884704F47F414FF07F4282EA0141C8
:10025000084310BD5032010810B50A4900F01F02D2
:10026000C0F384248B5CC0F3441240F3C0308A5C3A
:10027000095DC0F1FF0001EB022101EB034101EB3D
:10028000006010BDB846010810B50A49C0F303224A
:1002900000F00F048B5CC0F30312C0F303300C5D5D
:1002A000085C8A5CC043000600EB044000EB0220BF
:1002B000184410BDA846010870B5054600F092F834
:1002C000044600220121A869F9F7CAF8204370BD4D
:1002D00070B504461C4D17A020676869011DC0E970
:1002E0000E010064091D6161417C05F1480050F870
:1002F0002100C1680A6B04F1080190471348606649
:10030000A868E06168690830606101202076E076C5
:10031000FAF724FFA064032084F868000C482063E7
:1003200060632869F8F720FFE868F8F755FF094887
:10033000A86170BD53454747455220656D57696EAA
:1003400020563534363035000C140020E8320108D0
:10035000785634FF5C4A01082DE9F0411F4C94F8AF
:100360002800002838D101251D4884F82850102283
:1003700004F1C00102600B4688685B6808B9980800
:1003800088605A202062002002FA00F604EBC007C1
:10039000401C3E641028F7D309680222C81814389C
:1003A000C4E90D01C4E903320020042105E0636BB8
:1003B000421C01EBC006401C9A512269521E824227
:1003C000F5D865622069401E6060A16BE068FCF7AB
:1003D00095F9FEF7B5FF2563BDE8F081284F0020B1
:1003E0000814002010B50446806848B95020F3F77F
:1003F000F1FB50220021A060F6F7A6F9A06808B131
:10040000002010BD012010BDFEB514460E46054665
:10041000F3F7D4FC0090836A980739D53046FCF78F
:1004200047F8002834D040F601000340012B2FD0BC
:100430002846F3F755FC02460090314601A8F6F72E
:1004400039F801A8FCF734F8F8B1009944F2200219
:10045000886A104205D0083101AA0846F4F782FEE6
:1004600013E0DDE9012320430A4C8862C1E902233D
:10047000A088401CA0802846FBF75CFD012181403C
:10048000E0680143E160F4F7FBFF6846F3F77EFCA8
:10049000FEBD0000601500203EB5044690F828001F
:1004A0000128A06802D0F3F704F93EBD6946FAF7C7
:1004B000D5FEA068F3F714FC0290BDF80210B0F866
:1004C00058201144ADF80210BDF80610B0F86020B5
:1004D000891AADF80610BDF80010B0F854000144B8
:1004E000208A801E0844ADF80000401CADF80400CE
:1004F00002A8F3F74BFC6946A068FBF76BF83EBD1A
:1005000008C883F07F4308C1521EF9D1704770B507
:100510004FF07F4408C8DEB203F47F4545EA064544
:10052000C3F30746354324EA03031D4320C1521E8B
:10053000F0D170BDFEB504460E4615462046FFF7C5
:10054000ADFA0D4951F8243000FB063100FB0532AD
:100550000A4B002053F82430CDE9003002900748C0
:10056000001F50F824302046FCF7C4FD034808382B
:1005700040F82450FEBD000030320108B0130020C6
:100580002DE9FE4F04460E4617469846DDE90CA5B8
:10059000DDF838902046FFF781FA114951F8242000
:1005A000104951F8241000FB01220E480D49001D8E
:1005B0000C3150F8240051F8243007FB006606FB8C
:1005C00003210AFB008606FB0322401B2B460290F8
:1005D000CDE900902046FCF78DFDBDE8FE8F0000C0
:1005E00030320108A813002008B509480068816965
:1005F00021F0010181610020009006482823152286
:1006000001681C38F6F78EFDBDE80840F8F7A2BF78
:10061000A04D0020BC4E002008B509480068816943
:1006200041F0010181610020009006482923152234
:1006300001681C38F6F776FDBDE80840F8F78BBF77
:10064000A04D0020BC4E00202DE9FE4F04468846F8
:1006500092461F46DDE90D960C9D2046FFF71EFAD7
:10066000124A1149114B52F8242051F8241000FB72
:1006700002110E48001D0C3350F8240053F82430AA
:100680000AFB008202FB031206EBD671C5EB610187
:10069000401B2B4602902046CDE900913946FCF7DD
:1006A00029FDBDE8FE8F000030320108A8130020AC
:1006B0002DE9FE4F04460E4692469846DDE90D9719
:1006C0000C9D2046FFF7EAF9124A1149114B52F8E6
:1006D000242051F8241000FB02110E48001D0C3399
:1006E00050F8240053F824300AFB006202FB031682
:1006F0007F1BA0EB050A2046FFF786FB8DE8210251
:1007000053463A4631464046FCF714FDBDE8FE8F9D
:1007100030320108A81300202DE9FC4704460E469C
:1007200017461D46DDE90A89F4F782F8012826D02C
:10073000AD1B6D1CA8EB070808F101082046FFF768
:10074000ADF9194A1749184B52F8242051F82410D2
:1007500000FB02111448001D0C3350F8240053F81C
:10076000243007FB006202FB0311401B4346CDE926
:1007700000092A462046FCF703FDBDE8FC8700225D
:1007800020461921F8F73AFD43462A4639463046B5
:10079000F8F706FA02B02046044A1921BDE8F047EE
:1007A000F8F72CBD30320108A81300201907010802
:1007B00070B505460E460024F088082806D00124AE
:1007C000A4B12846BDE87040F8F7B2BA252110461A
:1007D000F8F726FA40B1F06820B100790028EFD090
:1007E0000124EDE70124EBE70124E9E7054C2A6841
:1007F000A8682168FFF78BFE29682068FCF7F2FCE7
:10080000206870BD941300202DE9F04192B0064697
:10081000012E7DDA6D4D0024286900286ED1F1F794
:1008200079FBF8F799FE6A49086840F08060086033
:10083000086800F08060019065482038026842F046
:1008400080620260026822F080620260604A143AAC
:10085000136843F400031360126802F4000201926B
:100860005B4A343A136843F400031360136823F4BB
:10087000000313600A6842F000620A60096801F030
:1008800000610191016841F000610160016821F09F
:1008900000610160002203215820F7F751F9582028
:1008A000F7F740F9002203215A20F7F749F95A20B7
:1008B000F7F738F96420029005200390049402A908
:1008C0004448F6F72FFB434942481C31F6F7FEF93E
:1008D0004148F6F725FF40480021F6F7DDFF582094
:1008E000F7F720F93B4858380068016841F4007177
:1008F00001605A20F7F716F9012028613046F8F711
:10090000E3F948B13046F8F70DFA0546304600E005
:1009100059E0F8F7F3F906E03046F8F7EFF9054645
:100920003046F8F7FFF905940695079408900F955F
:1009300010903046FFF768FA0990FF200A900B9458
:100940008DF844408DF845408DF846404FF4C06026
:100950000C9007200D90214850F826000E9005A914
:100960001D483246F6F7F4FD3046F8F745F90828F9
:1009700004DC19483146F6F732FE1DE013481849E9
:100980000C3050F82600884216D10024154FDFF8AD
:10099000588020467D68A84748F82400641CFF2C36
:1009A000F7D911494FF480720B483346F6F76EFDC4
:1009B00009483146F6F713FE0648F6F7E1FB012138
:1009C0000220F9F79DF812B0BDE8F08194130020E1
:1009D00044380240A04E0020A04D002030320108D3
:1009E0006832010850320108A049002032483149DC
:1009F00001600121C1600421816000211C3001607F
:100A000041600162C16141620222C26040F6FF7230
:100A1000826141614FF448720261522282624FF456
:100A2000C372C2624FF4EE6202630C2242638263BD
:100A3000C2634FF4F07202644FF400424264102229
:100A40008264C1645202026552104265521082658E
:100A50005210C2655210026652104266A0F58E70A6
:100A6000164A02601205426052088260C16001614C
:100A700080F8361080F83510802180F834103E213F
:100A800041610B2181614FF4B571C1611721016290
:100A900040F28A41416240F2F711816240F2B65160
:100AA000C16240F2032101630349054858390860D7
:100AB00070470000006C0140A04E0020006801401B
:100AC00000B002402DE9F84F81460F4690469A4605
:100AD000DDF828B00C9C002623E0144D2246484641
:100AE0006968FFF70DFDA96822463846FFF708FD43
:100AF00000940E9BA968D5E90020FCF7B7FB286895
:100B000022464146FFF7FCFC04EB0A0009EB800992
:100B100004EB0B0007EB80070B98204408EB8008E0
:100B2000761C0D988642D8D3BDE8F88F9413002028
:100B300030B401F47F43C1F30744C9B2234343EA0D
:100B40000141024630BC0148F6F7E2BCA04D00204E
:100B5000002903D001460348F6F75EBD014601486F
:100B6000F6F720BDA04D002030B401F47F44C1F35E
:100B70000745C9B22C4344EA0141064C44F822100F
:100B80002146034630BC4FF4807201F58060F6F7D1
:100B90007DBC0000A0490020C1F1FF0102460148D0
:100BA000F6F7B9BEA04D002003460148F6F7D5BEC2
:100BB000A04D002003460148F6F7FABEA04D0020E4
:100BC00030B40A4C084B54F8204053F8203002FB54
:100BD0000411064A083252F8202001FB023130BCD1
:100BE00002460348F6F775BE30320108AC13002008
:100BF000A04D00200A4B842202EBC01000291A6885
:100C000004D0115841F00101115003E0115821F0B6
:100C1000010111501868416A41F0010141627047B9
:100C2000A04D00207FB50546F3F75AF81E4C009002
:100C3000616881B10846F3F753F80290466902A84B
:100C4000F3F7A4F800984169891B002907DC616863
:100C5000416065601EE00021656041601AE06468E3
:100C60002046F3F73DF80190446864B12046F3F75D
:100C700037F80390466903A8F3F788F800984069AD
:100C8000801B00280ADC009844600198456001A898
:100C9000F3F77CF86846F3F779F87FBD019844686C
:100CA00001A8F3F773F8DBE7FC160020704730B5B6
:100CB00091B0054604A9FAF7D1FA2846F3F710F8DF
:100CC00010A909AACDE9002108AB029007AA06A93C
:100CD000FFF775F8BDF91600BDF91210401A079913
:100CE000401A0999441A029890F87810490708D4D4
:100CF000406FA04201DD012100E000212846FAF703
:100D000087FF0299486FC1F88440C867BDF9140095
:100D1000BDF91020801A069A801A089A841A91F850
:100D20007800800708D4086FA04201DD012100E0AF
:100D300000212846FAF75EFF0298016FC0F8904044
:100D4000C0F888107C30F9F7D8FF02988830F9F79E
:100D5000D4FF02980DF1340C7C300EC88CE80E00E4
:100D600007C80AAB83E8070002A8F3F70FF80AAA3E
:100D70000DA92846F9F757FF11B030BD884200DDB4
:100D8000084670472DE9F0478AB004460020914696
:100D90008A4601900290039006AE4FF0030804903B
:100DA00022E02046F2F79CFF4A4651460090F4F7B5
:100DB00005FA00984A4651460830F4F7FFF90098C2
:100DC000D0E907576846F2F7E1FF4A465146284600
:100DD000FFF7D8FFCDF80480CDE906A901A9204688
:100DE0000496FBF7BFFB3C46002CDAD10AB0BDE805
:100DF000F087002280690621F8F732BB0022806963
:100E00000521F8F72DBB38B5CC680546002C28D055
:100E100029466068FBF705FA78B10121284600F001
:100E2000F5FE29466068FBF7EBF9002819D0284643
:100E3000F2F756FF009061680EE00021284600F0AE
:100E4000E5FE29462068FBF7DBF9002809D0284693
:100E5000F2F746FF00902168C0F880106846F2F76C
:100E600095FF38BDFEB5F2F73BFF0090406EF3F7FB
:100E700017F80546002417E0406E2146F3F71CF8EA
:100E8000F2F72EFF019070B106683046F2F728FFA6
:100E9000029028B1476802A8F2F778FF3046B847B9
:100EA00001A8F2F773FF641C0098AC42E4DB806E8B
:100EB000F2F7F6FF054600240EE0806E2146F2F7B9
:100EC000FBFFF2F70DFF019028B10068F2F750FE2A
:100ED00001A8F2F75BFF641C0098AC42EDDB406EAA
:100EE000F2F7B6FF0098806EF2F7B2FF6846F2F7AD
:100EF0004DFFFEBD38B50446F2F7F2FE0090406AA1
:100F000020B1F2F735FE0099002048626846F2F7FA
:100F10003DFF2046F2F72CFE38BD000010B5084C0E
:100F2000A068F2F73DFEE068F2F73AFE2069F2F7BA
:100F300037FE00202061E060A0606061A06110BD0C
:100F4000D813002070B50A4C00250B4E656374223F
:100F5000336829460748984708223368002104F17E
:100F600048009847034860616570256270BD0000C5
:100F70000C140020F44F0020E415002010B5044CA0
:100F8000A068F2F70DFE0020A060606010BD0000B8
:100F9000C814002070B51B4D002405F160026C7070
:100FA000EC632046A2F10801C5F8184042F8204041
:100FB00041F82040401C0228F8D3AC62EC62EC619E
:100FC000124E6C62AC631822336800210E489847B9
:100FD0000C49002048316C6341F82040401C022835
:100FE000FAD3102233680021094898471022336849
:100FF0000021084898473368BDE87040102200215E
:10100000054818476015002068500020E4150020AE
:10101000F0500020005100201051002010B5034C6A
:101020002069F2F7BDFD0020206110BD00160020F0
:10103000024800210160416081607047FC16002079
:101040002DE9F04194B00E468046F2F749FE09A919
:101050000CAA0B90CDE9002105AB08AA0AA9FEF75E
:10106000AEFE0FA8FAF756F80FA90B98F9F77EFD18
:10107000DDE90F01CDE90301DDE90820BDF80E101F
:1010800002441144ADF80E100C9ABDF8121002443F
:10109000891AADF812100A9ABDF80C1002441144D6
:1010A000ADF80C10059ABDF810101044081AADF8F0
:1010B0001000DDE90301CDE9110111A8FAF7DAFD0D
:1010C0004046FAF79CF820B10B984C49406B884297
:1010D00005D00B98406BF4F721F9F2F787FF0B98D6
:1010E000D0F8942012B10021404690470B9890F818
:1010F0006C1041B10C9A0599CDE900124146089B4C
:101100000A9AFDF7B9FE0FA903A8099AF5F7CCFAD8
:1011100003A8FAF7AFFD0B98FF22816BB2EB116FBA
:1011200009D00C99059ACDE9002102964146089B09
:101130000A9AFDF751FB0B98D0F8942012B10121C7
:101140004046904711A8FAF795FD0B98406EF2F7CC
:10115000A7FE0546002419E00B982146406EF2F7E1
:10116000ABFEF2F7BDFD079078B107683846F2F79D
:10117000B7FD0E9030B102683146384690470EA850
:10118000F2F704FE07A8F2F701FE641CAC42E3D3B9
:1011900003A8FAF76FFD0B98806EF2F781FE054603
:1011A000002419E00B982146806EF2F785FEF2F7D5
:1011B00097FD079078B107683846F2F791FD0D90DA
:1011C00030B102683146384690470DA8F2F7DEFD8F
:1011D00007A8F2F7DBFD641CAC42E3D30020FAF76A
:1011E00049FD0B98D0F8942012B102214046904757
:1011F0000BA8F2F7CBFD14B0BDE8F081785634FFB0
:101200002DE9F04188B0F2F76BFD0590406A0028A7
:101210005AD0F2F765FD0646079005988068F2F708
:101220005FFD069030F8544F03A98788B0F8088016
:10123000858905988068FAF711F8BDF80C00BDF8AB
:101240001020204400B2ADF80C00BDF80E10394457
:10125000ADF80E10A2EB08010AB2ADF81020BDF8EF
:101260001210491B0CB20599ADF812400D6A0B69BA
:10127000651B069C54F8807FE4682F441D1B91F881
:101280002830012B26D0541B641CA04204DD001B17
:10129000044406EB40062D1A002D0FDD8869F4F793
:1012A00048F8059A0121881E92F829208DE8070048
:1012B0003B46224629463046F3F7FCF806A8F2F7EB
:1012C00065FD07A8F2F762FD05A8F2F75FFD08B01B
:1012D000BDE8F0810446DFE7F8B50E460546F2F7B3
:1012E000FFFC00903046F9F731FA04463046F9F732
:1012F00097FFFE28009808D0C0F88C402846FAF7DF
:10130000A9F96846F2F742FDF8BDC0F88040F5E75C
:1013100038B50446F2F7E4FC0090C16D89B120466F
:10132000F8F7E7FF0099C86D00280ADD0A6D086E1E
:10133000824202DB4FF0010201E04FF000020BDCC1
:101340000BE000990A6D086E824202DC4FF0010248
:1013500001E04FF0000200DA08651AB12046FBF701
:10136000ACFF04E000983221406EFAF77FFA68463D
:10137000F2F70CFD38BD0000F8B50E460746CD6803
:10138000F2F7AEFC0090B0F87C406846F2F7FEFC45
:10139000F068002817D0287AB0B1200702D4384668
:1013A000FAF74CFB3846F9F79DFCE0060BD5E00553
:1013B00009D50023200606D40A482946B0F90020A2
:1013C0003846FAF7DDFAF8BD3846F2F789FC0090A6
:1013D00030F87C1F21F4807101806846F2F7D6FC5A
:1013E000F8BD0000E41400202DE9F04FCD6891B065
:1013F0008046002D7DD0287A4FF4807B002840461F
:1014000078D0F2F76DFC0190046D826C04A940461F
:1014100090470198426DC16CB0F832A08F1A5FEA14
:101420000A7003D5D5E90010C5E9000101982D68BF
:101430000026816D03290FD0059AAA4220DB761E73
:10144000022951D0406E10B14046FBF736FF01999A
:101450000220641E886547E04046FBF72EFF0C988B
:10146000059900EBD070A5EB6000401A401E784350
:101470000B99F4F75DFD04460198046601A86CE041
:10148000069AAA4203DD406D241A46422CE0079AD0
:10149000AA4214DB0B9800280DDD0C98059900EB8F
:1014A000D070A5EB6000451A6D1E07FB05F00B9987
:1014B000F4F73EFD044601990320886514E0089A7C
:1014C000AA4202DD466D34440EE0099AAA420BDBC3
:1014D0000126012908D0406E10B14046FBF7EDFE11
:1014E00001990120641C886501980C99D0F85C90E2
:1014F00001E07DE057E001EBD171059AA5EB6101B8
:10150000891A0B9A491E3AB107FB01F01146F4F70C
:101510000FFD0199086604E0816D012909D00021C1
:10152000016601A8F2F732FCD6B1B9F1000F03D081
:101530001CE0C16C491EF3E745464FF4C872002316
:1015400040F2D2414046F9F7E7FB07462846F2F75A
:10155000C7FB00904766C6656846F2F717FC05E0D2
:10156000B9F1000F02D04046FBF7A7FE012140462B
:10157000FAF7E8F921464046F9F7FEF85FEACA5063
:1015800036D445464046F2F7ABFB009090F8284031
:101590006846F2F7FBFB59462846F9F78DFAA00793
:1015A00026D5012121E0F2F79BFB0190448E01A892
:1015B000F2F7ECFBE0051BD5454659464046F9F7E6
:1015C000CDF92846F2F78CFB0090C06D10B128468B
:1015D000FBF773FE0098002190F82840816568466B
:1015E000F2F7D4FBA00703D502212846FAF79CF8AE
:1015F00011B0BDE8F08F2DE9F14F98B01898F2F7CF
:101600006FFB0C90416B1291C16D066D8D68F1F707
:10161000EFFA07460C98B0F958B00CA8F2F7B6FBF1
:101620001898F9F701FF0B901898F9F714FF044682
:101630002A6801211898904780462A680321189843
:1016400090470E902A6800211898904709902A68C0
:101650000221189890470546189800900020FAF744
:1016600083FC002848D00B980B99A0F10109099838
:10167000A4F1010A074407EB0B00A0F1010B0E983F
:10168000651B0C1A781E169006A904A8641ECDE9E5
:101690000A016D1E0020059004900B200190CDE9F9
:1016A000069A6846B047CDE9064BCDE90487AB45BD
:1016B00000DB07950E2001906846B047CDF81080FA
:1016C0000998CDE905041698079005200190684611
:1016D000B047DDE90A121898F1F7BCFA0220F3F7D7
:1016E000BFFE1298F3F742FE122001906846B04701
:1016F000FAF7EEFB0028CDD119B0BDE8F08FF0B5B8
:1017000095B00646F2F7ECFA0C9090F86810C76CAA
:1017100001F00101056E0E91416BF8F7C2FD044620
:101720000CA8F2F733FB0EA80B9069463046F9F788
:1017300007FD0B20CDE90360BDF900000790BDF95E
:1017400002000890BDF904000990BDF906000A9056
:1017500003A8A847DDE90001CDE9130113A901227F
:101760000846F4F7A1FF13A8FAF784FA0520CDE99B
:1017700003600E980028BDF90000079008D0BDF95D
:1017800002000890BDF904102044CDE9091007E0DB
:10179000BDF902102044CDE90810BDF906000A90F9
:1017A00000200F9003A8A8470E980028BDF900005C
:1017B00005D00790BDF90200641C204404E0641CBD
:1017C00020440790BDF902000890BDF9040009907B
:1017D000BDF906000A9001200F9003A8A8473046E3
:1017E000F2F77EFA0C90F8F71AFD0D90F8B1384632
:1017F000F3F7BCFDDDE90C026946F8F713FD0CA810
:10180000F2F7C4FA0D9810901220CDE90360BDF9EB
:1018100000000790BDF902000890BDF9040009908E
:10182000BDF906000A9003A8A8470DA800E00CA87F
:10183000F2F7ACFA0020FAF71DFA15B0F0BD70B55A
:101840009AB00646F2F74CFA1290046C816D054688
:10185000179190F832006946C0F3C00016903046E8
:10186000FBF728F812A8F2F791FA14A92846F9F71D
:101870009AF90996BDF952000E90BDF956001090E4
:1018800016A8119008200A9000980D9001980F90CA
:1018900009A8A04710200A900198401C0D900298BA
:1018A000401E0F9009A8A04711200A900398401CE1
:1018B0000D900498401E0F9009A8A04713200A908D
:1018C00002980D9003980F9009A8A04709200A904C
:1018D00004980D9005980F9009A8A047DDE905012F
:1018E000884207D00C200A9005980F91401C0D905B
:1018F00009A8A0471AB070BD10B50446F2F75EFA09
:10190000806AC00301D5034900E003492046BDE8D1
:1019100010400847354E0008ADC300082DE9FC41D2
:101920001F4C80462068806CF2F7DAF90090404640
:10193000F2F7D6F90146019000980830F3F798FCC9
:1019400028B32068DDE90021D0E9135601F1080031
:101950000832F4F7AFFD6846F2F718FA114FC7F8EE
:101960002C8001992068B1F90020C264B1F90210FD
:10197000016501A8F2F70AFA4046FFF7BDFF002013
:10198000F8622068C0E913560120BDE8FC81684672
:10199000F2F7FCF901A8F2F7F9F90020F5E70000E9
:1019A00020140020601500202DE9FC410546F2F7C7
:1019B00097F9009090F8281089073DD5C46939E05F
:1019C0002046F2F78DF9019090F82810C943890755
:1019D0002BD100990831F3F74BFC30B30098D0E9D4
:1019E00002676846F2F7D2F901A8F2F7CFF920466C
:1019F000FFF794FF70B12046F2F7E0F9019020461E
:101A0000FFF7D2FF2046F2F7D9F901902846F2F706
:101A1000D5F900902846F2F763F900902046F2F7D6
:101A20005FF901900098C0E902670198046A01A873
:101A3000F2F7ACF9002CC3D16846F2F7A7F9BDE87C
:101A4000FC81000010B50E4C6168206B814209D802
:101A5000401E2063FDF774FC216B491C216308B113
:101A6000002010BD60680422401E6060606A616BE7
:101A700002EBC0028A586262012201F8302010BDD8
:101A8000284F0020084910B54A680424521C4A60B7
:101A90004B6B04EBC0044A6A1A514B6B002203F8EB
:101AA0003020486210BD0000284F0020F0B5866845
:101AB000DDE90574356A02FB05105D1A15F10105B3
:101AC000D6F800C03CF810C0401C24F802CB6D1EB4
:101AD000F6D11046521CB842ECDBF0BD10B50446FE
:101AE0004068FEF74DF910280DD2084963680A686E
:101AF000D21A0A6001EBC002D4E90201443200B1FB
:101B0000416009B1086010BD106010BD284F002071
:101B10007CB5050026D0144C2068A84206D1F2F707
:101B2000DFF8009080682060684612E0044694B1B7
:101B30002046F2F7D5F801908068A8420DD1F2F75F
:101B4000CFF801990090806888606846F2F71EF926
:101B500001A8F2F71BF900207CBD044601A8F2F7AA
:101B600015F9E4E701207CBDFC1600202DE9F05FAB
:101B7000DFF894808346D8F83840D8F80C10601EFF
:101B80000F182046D0E90015B9BB6619BE4236D2FF
:101B9000D6E9001989B3D8F8343013F83130012B65
:101BA0002DD1D8F82C20914201D1012100E0002153
:101BB0008A46FFF793FF3068D8F83410042202EB0E
:101BC000C0004A460C5031462046EEF7C4FBBAF13D
:101BD000000F05D0D8F83410321B891AC8F8341019
:101BE00004EB09012846FAF789FDBBF1000F05D087
:101BF000834503D80020BDE8F09F00E04D462C440B
